:020000040801F1
:100000009057002025020108F96F01085965010881
:10001000F56F01081B1A010835AF01080000000048
:1000200000000000000000000000000021A0010806
:100030009B30010800000000C1710108A5A701085C
:1000400069B00108B1710108C1A90108B98C0108A2
:10005000A15C0108B98A0108CD5A0108D15A0108EA
:100060001D5B0108695B01086D5B0108052F010834
:10007000072F0108092F01080B2F01080D2F010878
:100080000F2F0108112F01087314010847AE010852
:1000900049AE0108251A0108271A0108B95B0108B1
:1000A000C3A90108C9A90108C7A90108C5A9010870
:1000B000CBA90108CDA90108CFA901085F650108F6
:1000C0005D65010863650108616501081BA0010801
:1000D0001DA00108D5AB0108D9AB01087DAC010812
:1000E000CF5A0108898B010845AE0108D7A901083C
:1000F000DDA90108DBA90108D9A9010875140108C7
:10010000D55C010819A00108D1A901081FA00108A8
:10011000D1AB0108D3AB0108D3A90108D5A90108C7
:10012000132F0108152F0108172F0108192F010897
:1001300000F002F800F067F80AA090E8000C824492
:100140008344AAF10107DA4501D100F05CF8AFF26F
:10015000090EBAE80F0013F0010F18BFFB1A43F0A5
:100160000103184720780200407802000A444FF04B
:10017000000C10F8013B13F0070408BF10F8014B06
:100180001D1108BF10F8015B641E05D010F8016B4B
:10019000641E01F8016BF9D113F0080F1EBF10F8AF
:1001A000014BAD1C0C1B09D16D1E58BF01F801CBD2
:1001B000FAD505E014F8016B01F8016B6D1EF9D555
:1001C0009142D6D37047000000230024002500266A
:1001D000103A28BF78C1FBD8520728BF30C148BFAA
:1001E0000B607047692900F06180002070471FB5DF
:1001F0009DE8030000F0F8FC00F082FE1FBD10B582
:1002000000F0E7FE10BD00F01BFF1146FFF7EFFF07
:100210000DF0BAFA01F082F803B4FFF7F0FF03BC67
:100220000BF05CFB0348004703480449044A054BB4
:100230007047000031010108904D002090570020C8
:10024000905200209052002070470FB4014610B524
:1002500004AA039800F0A2FB10BC5DF814FB70B573
:10026000044685690068C10601D5302600E02026D5
:10027000C00707D070BDD4E9012130469047206AFD
:10028000401C20626D1EF6D570BD70B504468569B0
:100290000078C00707D170BDD4E901212020904724
:1002A000206A401C20626D1EF6D570BD2DE9F0411C
:1002B0000646002410687529314616A510D0AFF304
:1002C0000080002802DA404213A507E031688A075F
:1002D00001D512A502E0490704D511A5012401E0CA
:1002E000AFF3008000210A2206F1240709E0B0FBE9
:1002F000F2FCB0FBF2F302FB1C00303078541846DD
:10030000491C0028F3D123462A463046BDE8F04177
:1003100000F0EBBA000000002D0000002B000000F0
:10032000200000002DE9F05F894604464FF0000AE6
:10033000DFF824B1FB44C0F820A02046E1688847DC
:1003400000287DD0252806D0D4E901219047206AD5
:10035000401C2062F1E700255F462046E16888479F
:100360002028064607DB312E05D2B81910F8200CDC
:1003700008B10543F1E7A80701D525F00405C4F845
:100380001CA00027C4F818A02A2E09D030460BF074
:1003900093FA38B304EB8708303EC8F8186019E0C8
:1003A00059F8041B204604EB87029161E1688847F5
:1003B000012F064618D1E069002820DA25F0200533
:1003C0001DE0D8F8180000EB800006EB4000303844
:1003D000C8F818002046E168884706460BF06CFA1A
:1003E0000028EED1012F0AD02E2E08D12046E16838
:1003F00088477F1C0646022F45F02005C4DBA06914
:10040000002803DA404245F00105A061E80701D069
:1004100025F01005A6B1A6F14100192802D8203612
:1004200045F400654A463146204625604D46FFF7B3
:10043000D9FE60B1012807D0ED1D25F0070000E0CE
:1004400007E000F1080978E705F1040975E730468F
:100450007AE7206ABDE8F09F0B4E02002DE9F041DB
:1004600017460D4604460646012913DD38460CF0B2
:10047000EFFB411C0CD0C0B20A2804F8010B02D0DB
:100480006D1E012DF2DC002020703046BDE8F081A9
:10049000B44201D10020F9E7384600F091FA002873
:1004A000F1D00026EFE700002DE9F0410C460746A9
:1004B0001646104600F06EF82078611C61280AD0BC
:1004C000722802D077283CD102E00125002405E003
:1004D0000225042402E0082448F2020511F8010B69
:1004E0002B2806D0622809D011F8010C74280AD0F4
:1004F0000BE045F0030544F00204EFE745F0040586
:1005000044F00104EAE744F01004384621460BF0B9
:10051000FBF9411C15D00021316171604FF400716D
:10052000F560F1617061200704D530460222002198
:1005300000F04AFA306D40F0010030653046BDE809
:10054000F0810020FBE72DE9F0410D460646104CF6
:10055000206DC10704D0410804D020F00104F7E762
:1005600022460EE0542000F06AF907000ED0206DFC
:1005700047F00101084354212065384600F0F4F8A3
:100580003A4629463046BDE8F0418DE70020D6E7DF
:10059000344C00202DE9F04704464FF000094FF09D
:1005A000FF37C568D4E90486A80707D0204600F0C5
:1005B000BBFA30460BF087F9002802DA3846BDE86E
:1005C000F087280502D5404600F068F94C21204606
:1005D00000F0CAF8206D20F0010020654846EEE7E3
:1005E00010B5431C02E010F8011B71B18107FAD16C
:1005F0004FF0013202C88C1A8C4314EAC211F9D0B0
:10060000C01A0A0603D0C01E10BDC01A10BD0A04CD
:1006100001D0801E10BD0902FCD0401E10BD421E3C
:1006200012F8013F002BFBD111F8013B002B02F81F
:10063000013BF9D17047032A40F2308010F0030CDF
:1006400000F0158011F8013BBCF1020F624498BF25
:1006500011F801CB00F8013B38BF11F8013BA2F1C2
:10066000040298BF00F801CB38BF00F8013B11F03D
:10067000030300F02580083AC0F0088051F8043BDD
:10068000083A51F804CBA0E80810F5E7121D5CBF4A
:1006900051F8043B40F8043BAFF30080D20724BF7D
:1006A00011F8013B11F801CB48BF11F8012B24BF11
:1006B00000F8013B00F801CB48BF00F8012B704760
:1006C00010B5203AC0F00B80B1E81850203AA0E8ED
:1006D0001850B1E81850A0E81850BFF4F5AF5FEA21
:1006E000027C24BFB1E81850A0E8185044BF18C9D4
:1006F00018C0BDE810405FEA827C24BF51F8043B7B
:1007000040F8043B08BF7047D20728BF31F8023BCE
:1007100048BF11F8012B28BF20F8023B48BF00F862
:10072000012B70474FF000020429C0F0128010F036
:10073000030C00F01B80CCF1040CBCF1020F18BFBD
:1007400000F8012BA8BF20F8022BA1EB0C0100F050
:100750000DB85FEAC17C24BF00F8012B00F8012B23
:1007600048BF00F8012B70474FF0000200B5134658
:1007700094469646203922BFA0E80C50A0E80C50C1
:10078000B1F12001BFF4F7AF090728BFA0E80C5072
:1007900048BF0CC05DF804EB890028BF40F8042B6B
:1007A00008BF704748BF20F8022B11F0804F18BFD8
:1007B00000F8012B704700004FF0013C50F8042B6B
:1007C00051F8043B9A4221D1A2EB0C03934313EA64
:1007D000CC1317D150F8042B51F8043B9A4215D191
:1007E000A2EB0C03934313EACC130BD150F8042B68
:1007F00051F8043B9A4209D1A2EB0C03934313EA4C
:10080000CC13DBD04FF00000704700BFD01A01BA04
:10081000B1FA81F101F0180122FA01F0CB40C1F1E7
:100820002001DBB2C0B2C01A2CFA01F3D11A9143F5
:1008300011EAC311E6D1704770477047704770B531
:10084000064600F0B5F9056806F10B0020F0070434
:10085000B4429CBF002070BD2B466A68BAB11068D4
:10086000A04210D304F1080188423CBF5068586090
:1008700007D35168101941601168091B0160586065
:100880001460101D70BD13465268002AE7D121463E
:10089000284600F095F90028DED170BD70B50446F9
:1008A000051F00F085F90068002C14BF446870BD76
:1008B000002C18BFAC423CBF20466468F8D30168E6
:1008C0000A18AA4218BF456003D12A680546114498
:1008D000016028684119A1421CBF6C6070BD61684D
:1008E000696021680844286070BD2DE9F0470D4615
:1008F00099469246044600F124080168880604D50A
:10090000E06921F01001216000E00120A84201DD32
:10091000471B00E00027A1697A1902EB0900081AB9
:10092000A0612078C00602D42046FFF798FC00267C
:1009300008E0D4E901211AF806009047206A401C1B
:10094000761C20624E45F4DB2078C0060AD520468E
:10095000FFF785FC06E0D4E9012130209047206AAA
:10096000401C2062381EA7F10107F4DC07E0D4E93F
:10097000012118F805009047206A401C2062281EBB
:10098000A5F10105F3DC2046FFF77FFC2078000687
:1009900002D50220BDE8F0870120FBE7074B70B5C8
:1009A0000D467B4400F05BF90446284600F008F849
:1009B00010B14FF0FF3070BD204670BD47C300003E
:1009C000007B00F0800070472DE9F0410446164698
:1009D0000D464769007B80072ED038460AF08BFF12
:1009E00050BB3EB3012E02D0022E25D104E020469A
:1009F00000F065FA05441DE038460AF071FFE16831
:100A0000002841F01001E16005DA204600F058F8B6
:100A10000120BDE8F081C9030BD56268E16A91420B
:100A200000D81146A26911442269891A814200DD69
:100A300008460544002D01DA0220EAE7E16A606811
:100A4000E268814206D29103E06203D522F40031CC
:100A500041F01002A6690027AE4213DCE16A814230
:100A600001D90B4600E0034603EB060C2369ACEB0F
:100A7000030CAC4506DD814201D98C4600E084467A
:100A80009C4505D1A760276042F02000A5620DE0DB
:100A9000AD1BE669AE1B8142A66000D90846C01AAC
:100AA000281A20605819606022F02000034908408D
:100AB000E060002084F84870ABE70000BFCFD7FFAC
:100AC000C16821F4001141F08001C1600021816002
:100AD000016070472DE9F047814614460E464FF0FD
:100AE000FF383248D5685769054209D03846A169B0
:100AF0000AF049FF002811DB2C48C0430540E5609F
:100B00002B463246494638460AF04BFFA16920F091
:100B10000042B21A11440028A16103D02046FFF719
:100B2000CFFF4046BDE8F08770B504460569C06A4E
:100B30006168884200D80846E16821F42011E1602C
:100B4000C90312D5A84208D02246411B2846FFF708
:100B5000C1FF10B14FF0FF3070BD0020E562C4E965
:100B60000150E06820F48030E060002070BD10B5D6
:100B70000446C06820F02000E060A16AA0698842B5
:100B80000DD02046FFF7D0FFE06820F4405040F041
:100B90001000E060A06AA0612069E062606044F239
:100BA0004001E0688843E06010BD000010000200D2
:100BB00000487047384D00207047704770477047B5
:100BC00038B504460A4600206946AFF30080002885
:100BD00008BF38BD02460099204600F05BFA0120AC
:100BE00038BD012000F0AABBF8B5AFF30080054680
:100BF00000200C46102000BF0646A819A0420DD9BF
:100C0000324669460020AFF30080070008BF00F0BD
:100C100095FB0098A04218BF0546C419FFF7C8FF0E
:100C200005600746F01D20F007004619284600F031
:100C30000AF8B44208BFF8BDA21B31463868BDE8C7
:100C4000F84000F027BA00210160C0E901107047A8
:100C50001020704701694A1C02610878704700B58E
:100C60008FB0CDE901310021059105497944CDE9E5
:100C7000031011466846FFF755FB0FB000BD00009A
:100C8000E5FFFFFF70B50D4601461446D368506975
:100C90002A460AF065FE002807DA411C07D0E16801
:100CA00020F0004041F48041E160281A70BD2046E8
:100CB000FFF706FF4FF0FF3070BDC16800220260F1
:100CC00021F4805141F0400111F4C06FC16001D0A6
:100CD0008260704702694168891AC269891A816015
:100CE00070472DE9F0470446C06840F48000E0609A
:100CF000010312D520F40020E060810606D4E26AE8
:100D000061688A4200D80A46511A216040F40010F6
:100D1000E06094F82500BDE8F08720F40010E06062
:100D2000800602D52046FFF722FFE06842F28101EB
:100D30004FF0FF390140012903D02046FFF7C0FEE4
:100D4000B6E02168002600290ADAC94340F4805041
:100D50002160C4E902606068411C61600078DAE7E4
:100D600044F2400108420CD020F4A04040F0400082
:100D70002660E06021696068401AE169401AA0605D
:100D800096E0216991B9C00310D4E069FFF757FDDF
:100D90002061B0B1E06840F4006010F4407FE06092
:100DA00002D140F48070E06020696060E068D4F8AF
:100DB00014A0C1061AD5C0030ED52046FFF7B4FE15
:100DC00014E004F1240020610120E061E06820F4D7
:100DD000407040F48060E6E721696068401AA169CC
:100DE000014450460AF0CFFD0028A6DBE068C003AE
:100DF0002AD56168E06A884200D808462169451A08
:100E0000E069471B1BD02046D4F81880FFF78CFE02
:100E100008EB05015046C4F818800AF0B4FD00281C
:100E20008BDBE06840F40030E060000202D5A0698E
:100E30002844A061E1692069C91B45180DE02046DE
:100E4000FFF772FEE769F5E725696168D4E90607EF
:100E5000491BE56208446560A061E06820F010006D
:100E600010F4C06FE06002D0204600F03BFAE0686A
:100E700040F48050C4E90260000205D52069E062B8
:100E800060606FF0010046E7224639462846FFF7CA
:100E9000F9FE411C0CD02918E16258B1401E2060B7
:100EA000681C6060E06840F40030E060287832E759
:100EB000484630E765602046FFF7FFFEF8E710B5CB
:100EC0000146C268900703D0900607D5886A0AE0F9
:100ED00000F0DCF801210160881E10BD8B694868B4
:100EE00018440B69C01A91F848301BB191F84910A9
:100EF000401A10BD1103FCD50028FADD401E10BDBC
:100F000010B542485421FFF72FFC41485421FFF708
:100F10002BFC40485421FFF727FC3F493B483C4A03
:100F20003F4B08603D490A603A491960531C03650C
:100F3000481C1065012008653B48344A39A17844B3
:100F4000FFF7B2FA20B9384878440A3800F0EFF9D0
:100F500037482F4A35A17844FFF7A6FA20B934481C
:100F600078440A3800F0E3F932482A4A2FA178443D
:100F7000FFF79AFA20B92F4878440A3800F0D7F9D9
:100F800040232248DC000021224600F088F920B1ED
:100F900025487844543800F0CAF91D4822464023B9
:100FA000002100F07CF920B121487844543800F049
:100FB000BEF9184822461023002100F070F90028DD
:100FC00006D01C487844BDE81040563800F0AFB950
:100FD00010BD104870B5006D20F001040B48FFF7FC
:100FE000D9FA0B48FFF7D6FA0A48FFF7D3FA09E017
:100FF000206D20F001052046FFF7CCFA2046FFF7D0
:101000004DFC2C46002CF3D170BD0000344C002068
:10101000884C0020DC4C0020080400200C04002038
:101020001004002072000000F63901007700000073
:10103000E4390100D339010000487047304D0020E9
:101040007546FFF7F9FFAE4605006946534620F0A6
:101050000700854618B020B5FFF7E6F8BDE8204048
:101060004FF000064FF000074FF000084FF0000B64
:1010700021F00701AC46ACE8C009ACE8C009ACE817
:10108000C009ACE8C0098D467047000000487047B1
:10109000304D0020034640688C46002818BF884227
:1010A0003CBF03464068F8D318681844884207D00C
:1010B0000CF1030020F00700001D411A521A0146EE
:1010C000081D0A60FFF7EABB2DE9F04705460C460C
:1010D000C86820F4201040F48000C860800602D563
:1010E0000846FFF744FDE06841F282014FF0FF3906
:1010F0000140022903D02046FFF7E2FCB5E000F4EE
:101100002041B1F5004F0FD1C00306D56168E06AF8
:10111000884200D80846606006E02069E0626060AE
:1011200060690AF0DDFBA061A0680022EEB2002831
:101130000DDAE1688B050AD4C043A06041F4903019
:101140002260E0606068411C61600670A5E0E068B4
:101150009046226040F40050E060206968BB6069FE
:101160000AF0C9FB012704F12405A0B1A08910F4FD
:10117000407F08D0E069FFF762FB206118B1E068AA
:1011800040F4006016E0E7612561E06820F44070FB
:1011900040F480600EE0E069FFF751FB0028206119
:1011A000F1D0E06840F4006010F4407FE06002D1CC
:1011B00040F48070E06020696060E06825696FF04D
:1011C000010AC1051FD56168E06A884200D8084657
:1011D000411B04D022462846FFF77CFCF0BBE068A8
:1011E000010203D5E562C4E9015854E0691CE162DB
:1011F0006160E16940F48030491EC4E90210304664
:101200002E70BDE8F087010202D500F480320AE0BA
:101210006068411C61600670E0680A2E40F480300E
:10122000E06006D00022E16A6068814203D90B4683
:1012300002E00122F7E70346A7895B1B7F0503D481
:10124000E7699F4200DDE2B1814200D80146E562D4
:101250000F1AC4E90158002B09DD00E005E0224621
:1012600019462846FFF736FC08B14846C9E747B19A
:10127000A069E5626560C01BA061E06840F01000F5
:10128000E060E068000208D56168A069E562491B7A
:1012900008446560A0615046B3E73046B1E770B5D9
:1012A000C468A50713D0650211D4B2F5807F09D0B8
:1012B000B2F5007F06D0B2F5806F08D1012300F1AE
:1012C000240106E05D1E6FF07F46B54201D3012088
:1012D00070BD0161C361416024F470611143C1605C
:1012E000002070BD70B5054640F202260A4C0FE0A2
:1012F00094F85000C00708D0AC4206D0E06836EA47
:10130000000002D1204600F021F8206D20F00104F9
:10131000002CEDD170BD0000344C002010B5044607
:10132000AFF300802046BDE81040FEF775BF10B552
:1013300000F044F8BDE8104000F03AB810B500F0F5
:1013400057F8BDE8104000F033B8000070B504460F
:10135000C068810713D0800601D5A56A04E0A169A1
:10136000606808442169451A2046FFF7DDFB00222A
:10137000064629462046FFF727FB304670BD002071
:1013800070BD70B510B1BDE87040DFE70025074CB7
:101390006E1E07E02046FFF7D9FF00B13546206DED
:1013A00020F00104002CF5D1284670BD344C0020FB
:1013B000002801D00AF092BA7047000010B501462B
:1013C00002A000F03DF8012010BD00005349475233
:1013D000545245443A2052656469726563743A20F8
:1013E00063616E2774206F70656E3A200000000004
:1013F00010B5012805D0002103A000F021F801203C
:1014000010BD09A1F8E7000053494752544D454D1E
:101410003A204F7574206F662068656170206D6595
:101420006D6F7279000000003A2048656170206D90
:10143000656D6F727920636F727275707465640088
:1014400070B505460C460A2000E06D1C0AF0BCFA97
:1014500035B128780028F8D102E0641C0AF0B4FA0B
:1014600014B120780028F8D1BDE870400A200AF0B5
:10147000ABBA704770470029816802D041F0010182
:1014800001E021F0010181607047000010B50020EB
:10149000214908600120087148714FF4602088607C
:1014A0000020C860032008741C4800F059F8072386
:1014B00001220F21194800F077F8072302220821A2
:1014C000164800F071F8072303220921134800F0A1
:1014D0006BF80121114800F02DF801210F4800F0B0
:1014E0001FF801210D48FFF7C6FF0C4800F096F8E1
:1014F00000BF0A4800F02DF80028FAD1074800F094
:101500009CF800BF054800F01DF80028FAD1012121
:10151000024800F088F810BDE80D002000240140CA
:101520000029816802D041F4807101E021F48071CA
:10153000816070474268491E22F4604242EA4131AC
:1015400041607047014600208968490700D50120A5
:101550007047014600208968090700D501207047BF
:1015600010B542680E4B0C791A400B6842EA04220F
:101570001343436082680B4B1A40D1E90243234373
:101580004C7942EA440213438360C26A097C22F424
:101590007002491EC9B242EA0151C16210BD000089
:1015A000FFFEF0FFFDF7F1FF70B5072509290AD905
:1015B000C468A1F10A0606EB4606B540AC43B34049
:1015C0001C43C46007E0046901EB4106B540AC432D
:1015D000B3401C4304611F23072A09D2446B521EE7
:1015E00002EB820293409C4391400C43446370BDE4
:1015F0000D2A09D2046BD21F02EB820293409C4356
:1016000091400C43046370BDC46A0D3A02EB820240
:1016100093409C4391400C43C46270BD816841F08B
:101620000801816070470029816802D041F4A0015F
:1016300001E021F4A00181607047816841F004015C
:101640008160704710B51848007858B301211748D9
:1016500004F0E3FD30BB65211548006809F054FE35
:1016600000241CE0002240F22551124809F083FBBF
:1016700066220F480168002001F010FC0C48006849
:1016800008F0EAFB01F02AFC012240F2255109484A
:1016900009F071FB002004490870601CC4B2032CDF
:1016A000E0DB00BF10BD0000080100200008014081
:1016B00004010020004400401148006811490968F5
:1016C0000844401C00EB40000F4901EB800080689B
:1016D000A8B10C480068042805DA0A480068401CD4
:1016E0000849086008E006480068182804DA044839
:1016F0000068401C024908600120044908707047D6
:101700004C03002060010020540C00206F010020D9
:101710000C480068002808DD0A480068401E094996
:1017200008600120084908700BE00848006800289C
:1017300007DD06480068401E044908600120024990
:1017400008707047600100206F0100204C030020EA
:1017500000B502460B46184600F010F802EB820175
:1017600000EB410000BD0146092903DD01F137000E
:10177000C0B2704701F13000C0B2FAE7014630292B
:1017800001DB392901DD002001E001F00F00704785
:101790000149405A70470000006C0040014A8152E4
:1017A00070470000006C00402DE9F84300244EA172
:1017B0004E48FEF7C8FE4E490860084600680028FB
:1017C0007ED04FF480614B4804F035FD01204A493A
:1017D00008704AA146480068FEF737FD642007F00C
:1017E0000DFB642190FBF1F201FB1205084607F0A6
:1017F00005FB642190FBF1F090FBF1F201FB120676
:10180000084607F0FBFA42F2107190FBF1F73346FD
:101810003A4641A1364800950068FEF716FD474854
:1018200000683C2190FBF1F201FB1205434800687F
:1018300090FBF1F62B46324641A12D480068FEF799
:1018400004FD692007F0DAFA0546682007F0D6FAA9
:10185000642190FBF1F6682007F0D0FA642190FB38
:10186000F1F201FB120733463A463AA120480095AF
:101870000068FEF7EAFC00BF204604F071FA8046DB
:10188000204605F009FA50B1404604F053FD0546E4
:101890002B46424636A116480068FEF7D6FC04F0F7
:1018A00071FE00F02DFD611C0C46084605F00EFA95
:1018B0000028E1D030A10E480068FEF7C6FC00E029
:1018C00010E04FF4FA502E49086001E004F05AFE8F
:1018D0002B4800680028F9D10749087004480068BF
:1018E000FEF758FEBDE8F883770000005C5003085F
:1018F000F0030020000C0140080100202A2A204D9E
:1019000069737454696D65206261636B75702066DC
:10191000696C652E0A0000002A2A2050726F6772D7
:10192000616D2056657273696F6E3A2025692E25A8
:101930003032692E253032690A0000003000002064
:101940002A2A2054696D653A20253032693A2530BB
:1019500032690A002A2A20446174653A202530320F
:10196000692D253032692D253034690A00000000C8
:1019700025693D25690A00002A2A20456E640A006F
:1019800018000020F0B506460C461746BC420BD1A5
:10199000C4EBC400104951F82000B04201D12046E8
:1019A000F0BD4FF0FF30FBE7E01900EBD0714D10B8
:1019B000C5EBC500084951F82000B04205DA3A46A7
:1019C000691C3046FFF7DEFFEAE72A46214630462B
:1019D000FFF7D8FFE4E700005CEB010810B5002436
:1019E0000FE004F5CA70002109F0C2FB04F5E370B2
:1019F000002109F0BDFB04F5FC70002109F0B8FBE3
:101A0000641C322CEDD3002140F2931009F0B0FB9E
:101A10000021662009F0ACFB10BD00BFFEE70146C7
:101A200001207047704770470120704710B50121B1
:101A3000224804F0F2FB00283FD10BF019F90028EE
:101A40003BD11F49A1F804011E480BF025F810B93D
:101A500007F04EFD31E008F03DFD0022042108466C
:101A600008F054FD01220621042008F04FFDFFF785
:101A70009BFE00201249A1F8040113A00BF00CF802
:101A800090B901210A2009F073FB01210B2009F014
:101A90006FFB01210C2009F06BFB022207210420BF
:101AA00008F034FD00BFFEE700210A2009F060FBCA
:101AB00005F00CFA01200649087010BD000801402D
:101AC000044B00205C5003084D545F562A00000070
:101AD0006F0100202DE9FC5F4FF0000B3B480068D0
:101AE000C0EBC0003A4951F82090484604F05EF936
:101AF0000090484604F01EFC0546009804F026F9C4
:101B00000746009804F018F98046009804F00AF996
:101B10000190009805F0CEF88246BAF5284F3DD1E5
:101B2000642095FBF0F695FBF0F100FB115465B3D2
:101B30000D2E26D2DFE806F0250714081B091C0A23
:101B40000B1D0C1E0D0000BF00BF00BF00BF00BF7B
:101B500000BF012C01DB1F2C01DD4FF0010B13E056
:101B6000012C01DB1D2C01DD4FF0010B0CE000BF4F
:101B700000BF00BF012C01DB1E2C01DD4FF0010B6B
:101B800002E04FF0010B00BF00BFBBF1010F0ED10F
:101B900001224846019909F0FFFA08E0BD4201DB45
:101BA000454504DD01224846019909F0F5FA074848
:101BB0000068401C054908600846006805F086F882
:101BC00010B1002001490860BDE8FC9F2000002002
:101BD0005CEB010810B50121294804F01EFB90BB05
:101BE000682007F00BF9044640F2E6322548016808
:101BF000204609F005FB00BF07F05AFC04F0C2FCC8
:101C0000214800680F2190FBF1F201FB120080B91E
:101C10004FF480611D4804F007FB28B14FF4806148
:101C20001A4804F008FB04E04FF48061174804F000
:101C300004FB154800680028DED142F668116420D4
:101C400009F096FA1AE0FFE700BFFFF743FF04F040
:101C500099FC4FF480610D4804F0E6FA28B14FF486
:101C600080610A4804F0E7FA04E04FF48061074815
:101C700004F0E3FA044800680028E6D110BD000033
:101C8000000801403000002020000020000C01402E
:101C90007047000010B503480078012801D107F013
:101CA000B9FB10BD6E01002010B506F0A1FCA8B173
:101CB00008F0B0FD60B90C480068A0B901200A49DD
:101CC000086040F27D1007F099F8084908600AE0C2
:101CD0000020054908600549086004E00020024929
:101CE00008600249086010BDA00000209C00002090
:101CF0002DE9F041074640F2831007F07FF8804657
:101D0000002623E03146384604F0BCFB0546314648
:101D1000384604F0C4FB0446A5420ADA04F0D2FABD
:101D2000A84206DB04F0CEFAA04202DA3046BDE853
:101D3000F081A54209DD04F0C5FAA04203DB04F0FE
:101D4000C1FAA84201DB3046F1E7761C4645D9DBF3
:101D50004FF0FF30EBE7000010B50B2007F04EF816
:101D6000012817D108F0B6FB03220421084608F029
:101D7000CDFB04220621104608F0C8FB00201849BC
:101D8000086000BF07F094FB04F0FCFB14480068F7
:101D90000028F7D100210B2009F0EAF90C2007F008
:101DA0002DF8012812D100200AF062FF70B900203E
:101DB0000C49A1F804010C480AF06EFE30B9052266
:101DC0000621042008F0A2FB07F092FB00210C2062
:101DD00009F0CEF905F07AF801200449087010BD29
:101DE00020000020044B00205C5003086F010020FD
:101DF00070B501257BE0284604F0E2FA0446062C83
:101E000073D2DFE804F0030B141D262F284608F0D8
:101E100052FA2146284608F027FA66E000212846B3
:101E200008F02AFA2146284608F01EFA5DE0002153
:101E3000284608F0D9FA2146284608F015FA54E059
:101E40000021284608F03EFA2146284608F00CFA00
:101E50004BE00021284608F07BFA2146284608F08E
:101E600003FA42E0284604F089FA50B9284606F001
:101E7000DFFC0021284608F095F90121284608F0EA
:101E8000D7F9284604F042FF70BB284604F0AEFAAA
:101E900005281CD2DFE800F003070C1116002846C5
:101EA00008F009FA13E00121284608F0E5F90EE0F0
:101EB0000121284608F098FA09E00121284608F097
:101EC00001FA04E00121284608F042FA00BF00BFF1
:101ED0000021284608F0ACF9284604F087FA0646A7
:101EE0003146284608F0ACF900BF00BF6D1C4FF426
:101EF000BD7006F083FFA842BFF67DAF70BD000045
:101F000010B54FF4C27006F079FF04464FF4BF706D
:101F100006F074FF2049096888420BDD1E480168FD
:101F20004FF4BF7009F024F91C48016840F27F109B
:101F300009F01EF94FF4C07006F060FF16490968F9
:101F400088420BDA144801684FF4C07009F010F9A8
:101F50001248016840F2811009F00AF9DCB10F481B
:101F60000068844217D10C4801684FF4BF7009F033
:101F7000FFF80A48016840F27F1009F0F9F80648B6
:101F800001684FF4C07009F0F3F80448016840F2AA
:101F9000811009F0EDF810BD38000020300000205D
:101FA00010B54348046843480068844204D041485F
:101FB00004600120404908603D4844683F4800688B
:101FC000844204D03D48046001203B490860384801
:101FD00084683B480068844204D03948046001208A
:101FE00035490860012004F009FA044635480068C4
:101FF000844204D03348046001202F490860022045
:1020000004F0FCF9044630480068844204D02E48AD
:102010000460022028490860032004F0EFF9044618
:102020002A480068844204D02848046001202249DC
:102030000860042004F0E2F9044625480068844260
:1020400004D02348046001201B490860214800682F
:1020500008F0E4FF2049086020480068012804D106
:102060000846006880F0010008601D4800680128EB
:1020700006D11948006840F400601749086005E07F
:102080001548006820F4006013490860154800688E
:10209000012806D11048006840F480500E490860BD
:1020A00005E00D48006820F480500B49086010BD21
:1020B000F40B0020700000201803002074000020A2
:1020C00090000020780000207C000020800000208C
:1020D0008400002088000020600000208C00002088
:1020E000940000209800002010B504463A4800EB08
:1020F0000410006810B1012866D14CE03748006830
:1021000037490968884245D006F072FA28B106F0CE
:102110006FFAE8B306F076FAD0B304F002FAA04200
:1021200038DD2F48006800EB40002E4951F82000B0
:10213000294901EB0411496808602948006800EB4F
:102140004000284901EB80004068234901EB04115D
:10215000896808602248006800EB4000214901EBD3
:10216000800080681C4901EB0411C96808601C48A4
:102170000068401C142190FBF1F201FB1200184989
:1021800008600120144901EB04110860164900E0C1
:1021900000E008601EE0104800EB0410C068006812
:1021A00088B900200C4901EB0411496808600A490C
:1021B00001EB041189680860074901EB041108600C
:1021C00001200949086005E00020034901EB0411E2
:1021D000086000BF00BF10BDE4000020E000002048
:1021E000DC000020280E00201803002010B5FFF7A7
:1021F0005BFD002403E02046FFF776FF641C022C01
:10220000F9DB10BD70B50025002414E004EB440098
:10221000114901EB8000806801280BD104EB4401D7
:102220000D4A52F8211001F2851006F0E7FD012851
:1022300000D10125641C192CE8DB35B9074800687A
:1022400040F001000549086005E00448006820F0FE
:1022500001000249086070BD540C0020600000209D
:1022600010B50221234803F0D8FF30B1224800689E
:1022700040F001002049086005E01F48006820F098
:1022800001001D49086004211A4803F0C6FF30B15F
:102290001948006840F002001749086005E0164838
:1022A000006820F00200144908608021114803F002
:1022B000B4FF30B11048006840F004000E490860D7
:1022C00005E00D48006820F004000B49086010216B
:1022D0000A4803F0A2FF30B10748006840F0080048
:1022E0000549086005E00448006820F0080002493C
:1022F000086010BD000801406C0000200010014083
:102300002DE9F84F002000909DE07E480068401EB7
:102310007C49086006F0B6FC7B4908600846006806
:102320007A4988420EDB0120009077480068401A05
:102330007549086006F04EFD7348006806F02AFDF6
:1023400006F048FD7248006820B171480068401EE0
:102350006F4908606F48006820B16E480068401EF1
:102360006C4908606C48006820B16B480068401EEA
:10237000694908606948006820B168480068401EE3
:10238000664908606648006820B165480068401EDC
:10239000634908606348006820B162480068401ED5
:1023A000604908606048006820B15F480068401ECE
:1023B0005D4908605D48006820B15C480068401EC7
:1023C0005A4908604FF000080CE0594850F82800BE
:1023D00030B1574850F82800401E554941F82800B0
:1023E00008F10108B8F10A0FEFDB52480068002835
:1023F00005DD50480068401E4E49086005E00A208F
:102400004C49086001204C4908604C48D0F800B0A5
:1024100006F038FC3C21B0FBF1F906F033FC3C211E
:10242000B0FBF1F201FB120045490860B9F5B46F49
:1024300001DB40F29F59CB4502D04048C0F80090E4
:102440000120404908702F48006800287FF45DAFE4
:102450000098002853D0692006F0D0FC0546E91703
:1024600005EB91718910A5EB810141B9642195FBC0
:10247000F1F201FB125111B14FF01D0A01E04FF0D2
:102480001C0A682006F0BAFC0646642196FBF1F4AB
:1024900096FBF1F201FB1260471C0D2C18D2DFE80D
:1024A00004F0170712081709170A0B170C170D006D
:1024B00000BF00BF00BF00BF00BF00BF1F2F01DD76
:1024C000641C012709E0574501DD641C012704E075
:1024D0001E2F01DD641C012700BF00BF0C2C04DD92
:1024E0000124691C692008F043FE04EBC40000EBE2
:1024F000041007EB80063146682008F039FEBDE87D
:10250000F88F000004000020D0000020805101005E
:102510006C0300200C030020C4000020B800002041
:10252000280100209C0000204400002050000020D2
:102530002C0C0020CC0000201803002030000020CC
:1025400034000020C000002010B53448046804F0B6
:10255000010008B106F0F0FD04F0020010B106F031
:1025600023FE01E006F018FE04F0040010B106F0AE
:102570002DFE01E006F020FE04F0080010B106F088
:1025800039FE01E006F02CFE04F0100010B106F058
:1025900045FE01E006F038FE04F0200010B106F020
:1025A00051FE01E006F044FE04F0400010B106F0D8
:1025B0005DFE01E006F050FE04F0800010B106F070
:1025C00069FE01E006F05CFE04F4807010B106F0D4
:1025D00075FE01E006F068FE04F4007010B106F02C
:1025E00081FE01E006F074FE04F4806010B106F094
:1025F0009BFD01E006F090FD04F4006010B106F0D0
:10260000C1FD01E006F0B4FD04F4805010B106F005
:10261000A7FD01E006F09CFD10BD00006000002059
:1026200000B51448006840F2FE7188431149086003
:1026300000220CE0104901EB02114968086808F01B
:10264000EDFC0C49096808430A490860521C022A3B
:10265000F0DB0A48006830B10648006840F40060CA
:102660000449086005E00348006820F4006001495F
:10267000086000BD60000020E4000020A0000020F1
:102680000146A1F13000C1B2092901DDC81FC1B264
:1026900001F00F00704700000021002009E0084A07
:1026A000525C00EB800302EB4302A2F130004A1CB3
:1026B000D1B2034A525C0AB10829F0DB704700002E
:1026C000710100202DE9FE4F4FF000080024002783
:1026D000A14600250026A246A34600200290FC4801
:1026E0000078002878D009F071F9FA4901EB001060
:1026F0000068019003F05AFBF749086009F066F999
:10270000F44901EB00100068009003F04FFB0190CA
:1027100004F0D0FAB0F5A04F73D014DCB0F5605FD0
:1027200070D009DCB0F5005F22D0B0F5205F3BD05F
:10273000B0F5405F37D16BE0B0F5804F70D0B0F5A9
:10274000904FF7D104E1B0F5384F6AD009DCB0F50D
:10275000B04F67D0B0F5104F75D0B0F5284FE9D124
:1027600084E2B0F5504F6FD0B0F5983FE2D1D9E197
:1027700014E0D748005D2C2803D0D548005D2D28F3
:1027800002D14FF0010807E0D148005D05EB85015B
:1027900000EB4100A0F13005601CC4B2CC48005DE4
:1027A00008B1082CE5DBD9E221E0C948005D2D28FD
:1027B00002D14FF0010818E0C548005D2C2801D176
:1027C000012712E04FB1C248005D06EB860100EB25
:1027D0004100A0F1300608E0E2E2BD48005D05EBF3
:1027E000850100EB4100A0F13005601CC4B2B8487F
:1027F000005D08B1082CD8DB092E04DD4FF001087C
:1028000005E0E3E03CE005EB850006EB4005A5E2D2
:1028100025E0AF48005D2D2805D14FF001081CE0F0
:1028200062E0E6E127E1AA48005D2C2801D10127FA
:1028300013E057B1A648005D06EB860100EB4100AE
:10284000A0F1300609E094E15FE2A148005D05EBEC
:10285000850100EB4100A0F13005601CC4B29C482A
:10286000005D08B1082CD4DB632E02DD4FF00108B7
:1028700005E005EBC50000EB051006EB80056DE2F9
:1028800020E09348005D2D2802D14FF0010817E0A9
:102890008F48005D2C2801D1012711E047B18C48F9
:1028A000005D06EB860100EB4100A0F1300607E079
:1028B0008748005D05EB850100EB4100A0F1300584
:1028C000601CC4B28248005D08B1082CD9DBB6F5A3
:1028D0007A7F02DB4FF0010805E005EB4500C0EB15
:1028E000C51006EBC00539E220E07948005D2D28CF
:1028F00002D14FF0010817E07548005D2C2801D186
:10290000012711E047B17248005D06EB860100EB3C
:102910004100A0F1300607E06D48005D05EB850140
:1029200000EB4100A0F13005601CC4B26848005DB6
:1029300008B1082CD9DB42F20F70864202DD4FF05D
:10294000010804E040F27120684306EB001505E23F
:102950005F48007870B35E4800782D282AD05C4824
:102960000078A0F130055A48407800B358484078C4
:1029700005EB850100EB4100A0F13005544880785B
:1029800090B153488078A0F130065148C07840B1EA
:102990004F48C07806EB860100EB4100A0F13006FD
:1029A0000AE04FF0010807E04FF0010804E04FF0A3
:1029B000010801E04FF001083B2E02DD4FF0010855
:1029C00003E0C5EB051006EB8005C7E14FF00108F9
:1029D0003F480078F0B33E4800782D284AD03C4864
:1029E0000078A0F1300A3A48407898B338484078E7
:1029F0000AEB8A0100EB4100A0F1300A34488078EC
:102A000040B333488078A0F1300B3148C07808B328
:102A10002F48C0780BEB8B0100EB4100A0F1300B8D
:102A20002B480079B0B12A48007930380290284804
:102A3000407978B126484179029800EB800001EB9B
:102A4000400030380290BBF13B0F13DC02983B286A
:102A500010DC00E00EE0BAF1170F0BDC4FF00008BD
:102A60004FF461600AFB00F0CBEB0B1100EB81012E
:102A700002980D1872E1164800782D2802D14FF007
:102A80000109012419E01248005D2C2801D1012719
:102A900011E047B10E48005D06EB860100EB4100F6
:102AA000A0F1300607E00A48005D05EB850100EB68
:102AB0004100A0F13005601CC4B20548005D08B1BA
:102AC000082CE0DB092E09DD4FF0010829E00000A9
:102AD000710100209C2C002040030020B9F1010F5F
:102AE00006D105EB850006EB4000C0F52F7505E02B
:102AF00005EB850006EB400000F52F7540F27B10DA
:102B000006F07CF968B1A5F57F7000EBC00101EB20
:102B100000102D2101EB40005A2190FBF1F000F54F
:102B20002F751BE1AB4800782D2802D14FF0010929
:102B3000012410E0A748005D2C2802D14FF00108C5
:102B400009E0A448005D05EB850100EB4100A0F120
:102B50003005601CC4B29F48005D08B1082CE9DB59
:102B6000B9F1010F02D1C5F52F7501E005F52F75FB
:102B7000F4E0984800782D2802D14FF001081FE0BA
:102B800019E09448005D2C2801D1012711E047B1DC
:102B90009048005D06EB860100EB4100A0F1300695
:102BA00007E08C48005D05EB850100EB4100A0F1DA
:102BB0003005601CC4B28748005D08B1082CE0DB1A
:102BC000092E02DD4FF0010812E005EB850006EB4F
:102BD000400540F27B1006F011F948B105EBC50045
:102BE00000EB05102D2101EB40005A2190FBF1F57F
:102BF000B4E0784800782D2802D14FF00109012473
:102C000019E07448005D2C2801D1012711E047B17B
:102C10007048005D06EB860100EB4100A0F1300634
:102C200007E06C48005D05EB850100EB4100A0F179
:102C30003005601CC4B26748005D08B1082CE0DBB9
:102C4000092E02DD4FF001080FE0B9F1010F06D1A6
:102C500005EB850006EB4000C0F52F7505E005EBA0
:102C6000850006EB400000F52F7577E059480078A5
:102C70002D2802D14FF0010846E0564841780078EF
:102C8000303800EB800001EB4000A0F130055148E6
:102C9000C1788078303800EB800001EB4000A0F173
:102CA00030060D2E26D2DFE806F0250714081B0992
:102CB0001C0A0B1D0C1E0D0000BF00BF00BF00BF93
:102CC00000BF00BF012D01DB1F2D01DD4FF001080A
:102CD00013E0012D01DB1C2D01DD4FF001080CE09C
:102CE00000BF00BF00BF012D01DB1E2D01DD4FF035
:102CF000010802E04FF0010800BF00BF06EBC6006C
:102D000000EB061005EB800528E0324800782D28FE
:102D100002D14FF0010820E02E48007830386421BD
:102D200048432C494978303901EB810100EB4100DF
:102D3000284989780844A0F1300526480179C078EF
:102D4000303800EB800001EB4000A0F1300605EBCD
:102D50004500C0EBC51006EBC00500BF00BFB8F1D1
:102D6000000F33D108F032FE1B4901EB0010006860
:102D7000009003F01BF8019002F0E8FFA8420DDC80
:102D800008F024FE144901EB00100068009003F0E5
:102D90000DF8019002F0D0FFA84202DA4FF00108CE
:102DA00014E008F013FE0C4901EB0010006801224A
:102DB0002946019008F0F0F908F008FE064901EBF9
:102DC0000010006810B9284607F0F4F94046BDE845
:102DD000FE8F0000710100209C2C002030B50024E3
:102DE000002351E0184603F029FF01284AD1284862
:102DF0000068CD214843274901EB8000143000EBE7
:102E000003100568244800EB0410056020480068A2
:102E1000CD2148431F4901EB8000143000EB031023
:102E200040681D4901EB0411486019480068CD2134
:102E30004843184901EB8000143000EB0310806810
:102E4000154901EB0411886011480068CD21484301
:102E5000104901EB8000143000EB0310C0680E49EC
:102E600001EB0411C8600C4800EB04100068401C22
:102E700030B932230121601E074A02EB0010816045
:102E8000601CC4B2581CC3B2322BABDB30BD000097
:102E9000E8020020EC5C02089C2C002070B506467D
:102EA0000C46154600200C490860012006F07CFF06
:102EB000304606F0D1FF2C2006F076FF204606F0C3
:102EC000CBFF2C2006F070FF284606F0C5FF02203D
:102ED00006F06AFF70BD00003001002010B503202D
:102EE00006F062FF0548006807F042F8042006F08B
:102EF0005BFF00200249087010BD00003001002077
:102F00003C0100207047704770477047704770471A
:102F1000704770477047704770470029016802D0BA
:102F200041F0010101E021F0010101607047000062
:102F300010B5114800F028F81048114908601148F0
:102F40004860002088600320C8600020086180205D
:102F50004861400088618000C8612020086200024A
:102F6000486200208862044800F07AF80121024893
:102F7000FFF7D3FF10BD0000080002404C240140C1
:102F8000FC0D0020800D0020016821F0010101608E
:102F90000021016041608160C1602D4B2C49C21A43
:102FA0008039984243D018DC2A4BA0EB03029842A8
:102FB00035D00ADC284A801829D014282BD028289C
:102FC00024D1486840F4706034E0142A2BD0282AB9
:102FD0001CD1486840F470002CE02048B2F56C7FAA
:102FE0002ED009DCB2F5627F26D0B2F5677F0DD115
:102FF000016841F0F00108E0B2F5717F24D0B2F52C
:10300000767F03D1016841F4702101607047486800
:1030100040F00F000EE0486840F0F0000AE0486819
:1030200040F4704006E0486840F4702002E04868D0
:1030300040F0706048607047016841F00F01E4E7BC
:10304000016841F47061E0E7016841F47041DCE738
:103050008000024044000240F8FFFDBF040402402B
:1030600030B5036847F6F07293430C6A8A682243CE
:10307000D1E904452C4322438C692243CC69224385
:103080004C6A22438C6A22431A430260CA68426037
:103090000A6882604968C16030BD7047002000E066
:1030A000401C41F288318842FADB7047002000E082
:1030B000401CB0F57A7FFBDB70470000F8B50024B8
:1030C0004748007850B104F0D1FA0021084603F0D7
:1030D00039FA0122A821002004F06AFA00204149AF
:1030E000086065E0404800683E490968084400EB14
:1030F00040003E4901EB8000806808B9012457E098
:1031000038480168891C052003F01CFA344800780F
:1031100068B30120334D00902D68354E3668B542B6
:1031200001D1012500E000252B462F4D2D682D4EA5
:103130003668354405EB45052C4E06EB8505AA6837
:10314000294D2D68274E3668354405EB4505274E39
:1031500006EB85056968244D2D68224E3668354496
:1031600005EB4505214E56F8250007F0C1FF1D4A25
:1031700012681F4B1B689A4201D1012200E0002215
:103180001146194A1268174B1B681A4402EB420297
:10319000164B03EB8202906803F0E8FE11480068CA
:1031A000401C1049086008460068052800DB01241F
:1031B000002C97D00A48007868B10A48006850B9D6
:1031C000012C08D104210F2003F0BCF90022A92111
:1031D000104608F0DDF8002001490870F8BD000035
:1031E0006F010020500300204C030020540C0020ED
:1031F0006001002038B53E480078002877D00020D4
:103200003B49087001222D2104F0C6FA022100205A
:1032100003F098F90020374B00901B68364C246867
:10322000234403EB4303354C04EB83039A68314B8F
:103230001B68314C2468234403EB43032F4C04EBFD
:10324000830359682B4B1B682B4C2468234403EBE6
:1032500043032A4C54F82300002307F049FF0421BC
:10326000084603F06FF90022C521104608F090F8D7
:103270000521042003F066F90022C421104608F05D
:1032800087F80621022003F05DF900228D2101203C
:1032900005F0C6F90621122003F054F900228E2110
:1032A000012005F0BDF90621222003F04BF9002290
:1032B0008F21012005F0B4F90621482003F042F9DE
:1032C00000228A21012005F0ABF90621582003F0E5
:1032D00039F900228B21012005F0A2F9062168208E
:1032E00003F030F900228C21012005F099F938BD56
:1032F0006F0100204C03002060010020540C0020CE
:103300002DE9F041F848056840F2831005F076FD9C
:1033100004464FF4C17005F071FDF4490860022CB9
:1033200015DB0120F2490860F2490860F2490860A3
:10333000F2490860F2490860F2490860F249086001
:10334000F2490860F2490860F249086014E0002080
:10335000E7490860E7490860E7490860E74908600D
:10336000E7490860E7490860E7490860E7490860FD
:10337000E7490860E7490860032C15DB0120E649AE
:103380000860E6490860E6490860E6490860E649E1
:103390000860E6490860E6490860E6490860E649D1
:1033A0000860E649086014E00020DB490860DB495A
:1033B0000860DB490860DB490860DB490860DB49DD
:1033C0000860DB490860DB490860DB490860DB49CD
:1033D0000860042C15DB0120D9490860D949086030
:1033E000D9490860D9490860D9490860D9490860B5
:1033F000D9490860D9490860D9490860D9490860A5
:1034000014E00020CE490860CE490860CE4908602B
:10341000CE490860CE490860CE490860CE490860B0
:10342000CE490860CE490860CE490860052C15DBFE
:103430000120CD490860CD490860CD490860CD49DB
:103440000860CD490860CD490860CD490860CD4984
:103450000860CD490860CD49086014E00020C249E9
:103460000860C2490860C2490860C2490860C24990
:103470000860C2490860C2490860C2490860C24980
:103480000860C2490860062C15DB0120C0490860AD
:10349000C0490860C0490860C0490860C049086068
:1034A000C0490860C0490860C0490860C049086058
:1034B000C049086014E00020B5490860B5490860BB
:1034C000B5490860B5490860B5490860B549086064
:1034D000B5490860B5490860B5490860B549086054
:1034E0004FF4BD7005F08AFC0446022C03DB01207A
:1034F000B149086002E00020AF490860032C03DBFB
:103500000120AE49086002E00020AC490860042CAC
:1035100003DB0120AA49086002E00020A8490860F6
:10352000052C03DB0120A749086002E00020A54923
:103530000860062C03DB0120A349086002E000209C
:10354000A1490860072C03DB0120A049086002E0C4
:1035500000209E490860082C03DB01209C4908607C
:1035600002E000209A490860092C03DB01209949F8
:10357000086002E00020974908600A2C03DB012064
:103580009549086002E000209349086040F29110DC
:1035900005F034FC012801DD012000E000208F4906
:1035A00008606C2005F02AFC012806D0022817D0FC
:1035B00003281ED0052840D12FE00120884908604B
:1035C00000204B490860544908605D49086066491D
:1035D00008606F490860834908608349086034E0E7
:1035E00001207F4908607F49086000207E4908600B
:1035F0002BE001207A49086000203D4908604649D7
:1036000008604F4908605849086061490860754979
:10361000086001207449086017E0002070490860C4
:10362000334908603C490860454908604E490860D4
:10363000574908606C49086007E001206849086044
:10364000694908606749086000BF00BF872005F02E
:10365000D5FB012806D0022817D003281ED0052844
:1036600040D12FE001206149086000202149086015
:103670002A490860334908603C49086045490860A8
:103680005B4908605B490860BEE00120574908605B
:1036900057490860002057490860B5E001205349A8
:1036A00008600020124908601B490860244908602E
:1036B0002D490860364908604D49086001204D4990
:1036C0000860A1E00020494908600A4908601349E0
:1036D00008601C490860254908602E490860454972
:1036E000086091E088E00000000300207C010020D9
:1036F000840100209C010020B4010020CC010020A6
:10370000E4010020FC010020140200202C02002013
:10371000440200205C02002088010020A00100205B
:10372000B8010020D0010020E801002000020020A4
:103730001802002030020020480200206002002011
:103740008C010020A4010020BC010020D401002035
:10375000EC010020040200201C02002034020020A2
:103760004C0200206402002090010020A8010020EB
:10377000C0010020D8010020F00100200802002034
:1037800020020020380200205002002068020020A1
:1037900094010020AC010020C4010020DC010020C5
:1037A000F40100200C020020240200203C02002032
:1037B000540200206C020020980200209C0200208D
:1037C000A0020020A4020020A8020020AC020020D9
:1037D000B0020020B4020020B80200202403002020
:1037E0008001002070020020BC020020980100200F
:1037F00074020020C00200200120FB490860FB4940
:103800000860FB49086000BF00BFA22005F0F6FA7F
:10381000012806D0022817D003281ED0052840D141
:103820002FE00120F34908600020F3490860F349C4
:103830000860F3490860F3490860F3490860F349F8
:103840000860F349086034E00120EA490860EF4964
:1038500008600020EE4908602BE00120E54908607F
:103860000020E5490860E5490860E5490860E54948
:103870000860E5490860E54908600120E4490860FE
:1038800017E00020DB490860DB490860DB4908607D
:10389000DB490860DB490860DB490860DC490860F7
:1038A00007E00120D3490860D8490860D84908607A
:1038B00000BF00BFBD2005F0A1FA012806D00228F4
:1038C00017D003281ED0052840D12FE00120D14970
:1038D00008600020D0490860D0490860D0490860DD
:1038E000D0490860D0490860D0490860D0490860D4
:1038F00034E00120C7490860CC4908600020CC4969
:1039000008602BE00120C34908600020C24908601C
:10391000C2490860C2490860C2490860C2490860DB
:10392000C24908600120C249086017E00020B94977
:103930000860B9490860B9490860B9490860B949DF
:103940000860B9490860BA49086007E00120B14938
:103950000860B6490860B649086000BF00BFD820BB
:1039600005F04CFA012806D0022817D003281ED0F3
:10397000052840D12FE00120AE4908600020AE4963
:103980000860AE490860AE490860AE490860AE49BB
:103990000860AE490860AE49086034E00120A549DE
:1039A0000860AA4908600020A94908602BE00120AE
:1039B000A04908600020A0490860A0490860A0490B
:1039C0000860A0490860A0490860A049086001207B
:1039D0009F49086017E000209649086096490860F2
:1039E00096490860964908609649086096490860BB
:1039F0009749086007E001208E49086093490860F4
:103A00009349086000BF00BFF32005F0F7F90128D3
:103A100006D0022817D003281ED0052840D12FE059
:103A200001208C49086000208B4908608B490860A0
:103A30008B4908608B4908608B4908608B49086096
:103A40008B49086034E0012082490860874908609A
:103A50000020874908602BE001207E490860002093
:103A60007D4908607D4908607D4908607D4908609E
:103A70007D4908607D49086001207D49086017E0A4
:103A800000207449086074490860744908607449EA
:103A9000086074490860744908607549086007E067
:103AA00001206C490860714908607149086000BFD5
:103AB00000BF4FF4877005F0A1F9012806D0022855
:103AC0000DD0032814D0052836D125E001206949FE
:103AD00008600020684908606849086034E00120F7
:103AE00064490860644908600020644908602BE06C
:103AF0000120604908600020614908606149086050
:103B00006149086061490860614908605A49086074
:103B100001205A49086017E00020564908605849BA
:103B20000860584908605849086058490860584971
:103B300008605249086007E001204E4908604E497C
:103B400008604E49086000BF00BF40F2291005F030
:103B500055F9012806D0022817D003281ED00528C1
:103B600040D12FE001204B49086000204A490860FD
:103B70004A4908604A4908604A4908604A49086059
:103B80004A4908604A4908609CE0012041490860B0
:103B90004649086000204649086093E001203D49FD
:103BA000086000203C4908603C4908603C490860C6
:103BB0003C4908603C4908603C49086001203C4998
:103BC00008607FE0002033490860334908603349CA
:103BD0000860334908603349086033490860344954
:103BE00008606FE066E00000980100207402002089
:103BF000C0020020B0010020B4010020B801002064
:103C0000BC010020C0010020C40100207802002077
:103C1000C4020020C8010020CC010020D0010020F7
:103C2000D4010020D8010020DC0100207C0200200B
:103C3000C8020020E0010020E4010020E80100208B
:103C4000EC010020F0010020F4010020800200209F
:103C5000CC020020F8010020FC010020000200201E
:103C600004020020080200200C0200208402002030
:103C7000D00200201002002088020020D402002080
:103C800014020020180200201C0200202002002044
:103C900024020020280200202C02002030020020F4
:103CA00034020020380200203C0200208C02002058
:103CB000D80200200120F7490860F7490860F74959
:103CC000086000BF00BF4FF4A27005F097F801280C
:103CD00006D0022817D003281ED0052840D12FE097
:103CE0000120EF4908600020EE490860EE490860B5
:103CF000EE490860EE490860EE490860EE49086048
:103D0000EE49086034E00120E5490860EA490860AE
:103D10000020EA4908602BE00120E149086000200A
:103D2000E0490860E0490860E0490860E04908604F
:103D3000E0490860E04908600120E049086017E0B8
:103D40000020D7490860D7490860D7490860D7499B
:103D50000860D7490860D7490860D849086007E07B
:103D60000120CF490860D4490860D449086000BFE9
:103D700000BF40F25F1005F041F8012806D002288C
:103D800017D003281ED0052840D12FE00120CC49B0
:103D900008600020CB490860CB490860CB49086027
:103DA000CB490860CB490860CB490860CB49086023
:103DB00034E00120C2490860C74908600020C749B3
:103DC00008602BE00120BE4908600020BD49086062
:103DD000BD490860BD490860BD490860BD4908602B
:103DE000BD4908600120BD49086017E00020B449C2
:103DF0000860B4490860B4490860B4490860B4492F
:103E00000860B4490860B549086007E00120AC4982
:103E10000860B1490860B149086000BF00BFB04800
:103E200000681F2874D2DFE810F01F0043024D0223
:103E30007300C1022C035A03D003D103FC032704EF
:103E400052047300730073007300730073007300F7
:103E5000F7012902EE0073007300730073007A0209
:103E600083008D002F03A5034FF416709D49086051
:103E700000209D4908709D49087003F085F9472886
:103E800047D006DC1B2838D01E2848D02E284DD11C
:103E90001AE04D2807D0872825D08D2846D101204B
:103EA0008F49086042E0672004F0A8FF0446601CC8
:103EB0000446032800DD00242146672007F058F956
:103EC00001208B49086031E040F27B1004F096FF3E
:103ED000C0F10106314640F27B1007F049F901209C
:103EE0008349086022E000208249086015207C494F
:103EF000086001207E49086018E000207E490860C3
:103F00007E4908607E4908601320754908600DE00D
:103F100004E200207B4908604FF47A7506E0152022
:103F2000774908601B206E49086000BF00BFF9E3B5
:103F300001230022AF21AE2000F028FC1C2068499C
:103F40000860EFE304F0A6FF0746172F08D0472FBD
:103F500002D0872F50D100BF00206149086050E097
:103F6000FEF79AFB0646012E42DB4FF4BD7004F0CB
:103F700045FFB0423CDB0B2E2FD2DFE806F02E06C9
:103F80000A0E12161A1E22262A0005205949086018
:103F900023E00C20574908601FE0132055490860B2
:103FA0001BE01A205349086017E02120514908609E
:103FB00013E028204F4908600FE02F204D4908608A
:103FC0000BE036204B49086007E03D204949086076
:103FD00003E044204749086000BF00BF0020484973
:103FE000086004203E49086001204149086002E061
:103FF0001B203B49086004E00021384602F098FC91
:1040000000BF00BF8EE3002000F0ACFE04F042FFD2
:104010000746472F0AD004DC172F11D02D2F09D1C6
:104020000AE0872F03D08D2F04D104E000BF0020C9
:104030002B490860EEE000BF384606F009FFE9E0D2
:10404000314800782D4909780844C6B20C2E12D2A6
:10405000DFE806F006125C697683909DAAB7C4D1AA
:10406000002025490860254908601520244908607A
:1040700013201B490860CBE003201E49086015206F
:104080001F4908600420164908600120184908608B
:10409000BEE00000280200208C020020D802002090
:1040A0004002002044020020480200204C02002070
:1040B000500200205402002090020020DC02002068
:1040C000580200205C0200206002002064020020F0
:1040D000680200206C02002094020020E002002010
:1040E000000300206C0300206E0100206C01002002
:1040F00018030020E80200204C030020600100208B
:1041000008030020F0020020EC0200200520F849FE
:1041100008601520F74908600420F749086001206D
:10412000F649086074E00C20F14908601520F14957
:1041300008600420F04908600120F049086067E049
:104140001320EB4908601520EA4908600420EA4979
:1041500008600120E94908605AE01A20E449086033
:104160001520E44908600420E34908600120E34980
:1041700008604DE02120DE4908601520DD49086017
:104180000420DD4908600120DC49086040E0282067
:10419000D74908601520D74908600420D64908602F
:1041A0000120D649086033E02F20D149086015204E
:1041B000D04908600420D04908600120CF49086038
:1041C00026E03620CA4908601520CA490860042044
:1041D000C94908600120C949086019E03D20C44967
:1041E00008601520C34908600420C3490860012005
:1041F000C24908600CE04420BD4908601520BD4953
:1042000008600420BC4908600120BC49086000BF68
:1042100000BF00BF00BF85E2FEF750FF04F03AFE8A
:10422000472810D004DC172816D02D2824D104E00C
:1042300087280DD08D281FD102E0FDF73DFA1BE045
:10424000FDF766FA18E0AB480068AB49086013E078
:104250000020A94908600FE0A9480068A949096839
:10426000084400EB4000A84901EB8000806810B1D1
:104270001420A149086000BF00BF53E2FEF7BAFF57
:1042800004F008FE172807D047280BD087280DD147
:1042900000209949086009E006F088FE132096493D
:1042A000086003E013209449086000BF00BF39E2B2
:1042B000012300221D211E2000F068FA02208E49F1
:1042C00008602FE204F0E6FD0746172F08D0472FBD
:1042D00002D0872F1CD100BF0020874908601CE056
:1042E000FEF7DAF9064640F60A30864202D08748E1
:1042F000864209D101207E4908601A207E49086063
:1043000001208349087002E000207B49086004E036
:104310000121384602F00CFB00BF00BF02E2012081
:1043200000F020FD04F0B6FD074600207949087032
:10433000472F0AD004DC172F13D02D2F34D10CE0D7
:10434000872F03D08D2F2FD106E000BF00207149A9
:1043500008706949086027E000BF384606F078FD1C
:1043600022E06D480078674909780844C6B216B162
:10437000012E17D109E002205D4908601A205D492D
:10438000086004205C4908600CE04B205849086034
:104390001A205849086004205749086001205D49E7
:1043A000087000BF00BF00BF00BFBBE150480068FD
:1043B00000F0EEFB04F06EFD06464B2E4CD006DC02
:1043C000172E18D02D2E09D0472E58D10AE04E2E88
:1043D0002ED0872E0BD08D2E51D100BF304606F047
:1043E00037FD4CE0434800684349086047E000203F
:1043F0004149086043E007F0E9FA484901EB001041
:10440000D0F80080404601F0D1FC074602F044FCA1
:1044100068B10420424908600520374908603948DE
:104420000068404908603C4800683F49086026E051
:1044300000BF2F480068CD2148433C4901EB800074
:1044400040682B4908600846006802F04FFC0028CD
:10445000EFD04FF47A7512E000BF25480068CD21F7
:104460004843324951F82000214908600846006855
:1044700002F03CFC0028F0D04FF47A7500BF00BF7A
:1044800050E102F0ABF84DE101F0B6F8172804D086
:10449000472803D0872820D11BE000BF20480068B0
:1044A000154908601E4805681E48006815490860DF
:1044B0001D480068184908600D480068CD22504327
:1044C0001A4A02EB800001228168002003F064F99F
:1044D00003E000200849086000BF00BF22E100F0AF
:1044E000ABFF172824D0472823D0872840D13BE0B2
:1044F000E802002008030020000300201803002029
:104500004C03002060010020540C0020C6D53C0064
:104510006E0100206C010020EC0200209C2C002089
:10452000040300207403002078030020EC5C0208E0
:1045300000BF8A4800688A49086088480568894839
:104540000068894908608948006889490860894885
:104550000068CD225043884A02EB80000122816826
:10456000002003F019F903E000207D49086000BF36
:1045700000BFD7E000F0EEF9172804D0472803D099
:10458000872820D11BE000BF744800687449086088
:10459000724805687348006873490860734800688A
:1045A0007349086073480068CD225043724A02EB99
:1045B000800001228168002003F0EEF803E0002073
:1045C0006749086000BF00BFACE000BF00F020F901
:1045D000172804D0472803D0872820D11BE000BF2C
:1045E0005E4800685E4908605C4805685D48006890
:1045F0005D4908605D4800685D4908605D48006885
:10460000CD2250435C4A02EB8000012281680020E9
:1046100003F0C2F803E000205149086000BF00BF6A
:1046200080E000F0FAF8172804D0472803D0872844
:1046300020D11BE000BF494800684949086047484D
:104640000568484800684849086048480068484983
:10465000086048480068CD225043474A02EB80007A
:1046600001228168002003F097F803E000203C4914
:10467000086000BF00BF55E000F0DEFC172804D042
:10468000472803D0872820D11BE000BF33480068AB
:10469000334908603148056832480068324908608B
:1046A000324800683249086032480068CD225043E1
:1046B000314A02EB800001228168002003F06CF88F
:1046C00003E000202649086000BF00BF2AE001F097
:1046D0008BF8172804D0472803D0872820D11BE067
:1046E00000BF1E4800681E4908601C4805681D4838
:1046F00000681D4908601D4800681D4908601D4884
:104700000068CD2250431C4A02EB800001228168E0
:10471000002003F041F803E000201149086000BFC9
:1047200000BF00BF00BF1548006858B900200C4901
:104730000860134908600120124908704FF4167090
:104740000E49086006480068854205D000200E49E1
:10475000086001200B490870BDE8F08104030020C7
:104760000003002074030020600100207803002073
:10477000EC020020E8020020EC5C02086C03002040
:10478000F00200206F0100200C030020F8B5044661
:104790000F4615461E4607F0DFFA0122214600208B
:1047A00002F0FAFF0321042001F0CCFE002239467A
:1047B000104606F0EDFD3EB9062000231A462946B4
:1047C0000090184603F098FE0421084601F0BAFE56
:1047D00000220821022003F023FF002209210220E9
:1047E00003F01EFF00220921022003F019FF00221E
:1047F0000921022003F014FF00220B21022003F004
:104800000FFF04F01FFE0521082001F09BFEF8BDFC
:1048100010B5022000F006F810BD10B5032000F01E
:1048200001F810BD2DE9F04105466F0004F032FBA0
:10483000064600204149087041480078062814DAED
:1048400040480068B0F5FA7F05DA00225F210120B8
:1048500003F0E6FE04E000222021012003F0E0FE48
:10486000394800780B3838490870304608F050FF56
:1048700058B333480078B8425CDA304609F0D4FBCC
:104880002F490A780978491C2D4B19702F498854F3
:10489000304609F0C9FB044600222146012003F0FE
:1048A000BFFE29480078284908702548007802286A
:1048B00005D02348007804283CD1022D3ADD224857
:1048C00000780B302049087034E0172E02D0272ED4
:1048D0002FD104E0FDF7F6FE00B1022629E01848CA
:1048E0000478012C24DBBC4222DC0078401E1449F1
:1048F000087000211548124A127881541448025D4C
:104900000B21082007F073F90F4908700C48007854
:10491000052804DA00222021012003F081FE601E18
:104920000B490A5C0B21082007F061F90649087061
:1049300000BF00BF3046BDE8F08100006F010020DD
:104940006D0100201400002065010020710100208D
:104950004403002070B57F480078C1004FF07F40CD
:10496000C8407D4908607B480078C1004FF08070E6
:1049700008417A49086077480078C1004FF000503C
:1049800008417749086073480078C1004FF0FE4045
:1049900008417449086004F07DFA04460020724919
:1049A00008706C480078042874DA70480068000EBB
:1049B0006F4908706D480068000C6E4908706B48BC
:1049C0000088000A6C490870684800786B490870D4
:1049D00060480078C0EB0010083069490860082082
:1049E0006849087068480068B0F5FA7F07DA084639
:1049F000007863490968884201D1012000E0002065
:104A000002465B480178012003F00AFE5D48007809
:104A1000001D5C4908705C480068B0F5FA7F07DA51
:104A20000846007856490968884201D1012000E013
:104A3000002002464F480178012003F0F1FD514863
:104A40000078001D4F4908704F480068B0F5FA7FA4
:104A500007DA084600784A490968884201D10120EE
:104A600000E00020024644480178012003F0D8FD10
:104A700044480078001D4349087043480068B0F579
:104A8000FA7F08DA084600783D490968884202D171
:104A9000012001E00AE000200246384801780120A8
:104AA00003F0BEFD36480078364908704B2C33D0F1
:104AB00004DC172C07D02D2C49D137E04E2C21D007
:104AC0008D2C44D10DE0172406F080FF2F4901EB17
:104AD00000100122056825480168284606F05CFBA5
:104AE00035E0224800681C49096808401D490968EA
:104AF000884206DA1D4800681849096808441B49BD
:104B0000086024E013480078002804DD114800788C
:104B1000401E104908701AE00E480078032804DA95
:104B20000C480078401C0B49087010E00F480068E2
:104B30000949096808400A490968884206DD0B48A6
:104B4000006806490968401A0849086000BF00BFAC
:104B5000204670BD6D010020580300205C0300203A
:104B600060030020640300206F0100203803002050
:104B70005403002055030020560300205703002053
:104B80006803002065010020140000209C2C0020F8
:104B90002DE9F0410746002669480760694800781A
:104BA00090B1FEF71BF966480068CD225043664A73
:104BB00002EB800001228168002002F0EDFD002060
:104BC000624908606249086000205E4908706148D7
:104BD0000068002877D000205E49086001213A2053
:104BE00001F0B0FC5948006850B1002287211046FE
:104BF00003F016FD00228821104603F011FD09E0A4
:104C000000222021104603F00BFD00222021104637
:104C100003F006FD07213A2001F094FC00E0761C29
:104C20004D4800EB061080680028F8D0474800681F
:104C3000001DB0420CD0052E0ADB00228521104653
:104C400003F0EEFC00228621104603F0E9FC09E0A7
:104C500000228921104603F0E3FC0022892110463E
:104C600003F0DEFC02203D49087038480578002436
:104C700062E0394800EB05100068401C002858D05D
:104C800001203749087032480068844201D1012070
:104C900000E0002002462021002003F0C1FC042097
:104CA0002F4908702A480068844201D1012000E0A1
:104CB00000200146284602F067FC2548006884422F
:104CC00002D1012001E039E00020034601222946FB
:104CD000002002F09DFE204901EB0511086801F05B
:104CE00065F8804601F0C0FFD0281AD072201C4918
:104CF000087017480068844201D1012000E00020BC
:104D000002462021002003F08BFC114800688442F9
:104D100001D1012000E0002002462946002002F0D7
:104D20008FFB681CC5B20D480078401C0B49087009
:104D300000E00524601CC4B2052C9ADBBDE8F081BC
:104D4000E80200206F010020EC5C0208EC02002069
:104D500060010020180300209C2C00206601002028
:104D60006501002070B50646002568480660684861
:104D70000078A0B1FEF732F864480068CD225043B5
:104D8000644A02EB800001228168002002F004FDE9
:104D900000205F4908706049086060490860604809
:104DA0000068002879D000205D49086001213A2080
:104DB00001F0C8FB5848006850B100228721104616
:104DC00003F02EFC00228821104603F029FC09E0A4
:104DD00000222021104603F023FC0022202110464F
:104DE00003F01EFC07213A2001F0ACFB00E06D1C33
:104DF0004C4800EB051080680028F8D04648006851
:104E0000001DA8420CD0052D0ADB0022852110468A
:104E100003F006FC00228621104603F001FC09E0A5
:104E200000228921104603F0FBFB00228921104655
:104E300003F0F6FB02203C490870002463E036488A
:104E400000682044374901EB00100068401C00282E
:104E500056D001203549087030480068844201D19D
:104E6000012000E0002002462021002003F0D8FBB2
:104E70002A480068844201D1012000E00020024657
:104E80002021002003F0CCFB032028490870234890
:104E90000068844202D1012001E036E00020024691
:104EA0001D48006820441F4B03EB001041680020A0
:104EB00006F06EFA0BE019480068844201D1012027
:104EC00000E0002002462021002003F0A9FB174843
:104ED00000787828EFDB7720144908700F480068C5
:104EE000844201D1012000E0002002462021002060
:104EF00003F096FB0C480078401C0B49087000E05A
:104F00000524601CC4B2052C99DB70BDE8020020AA
:104F10006F010020EC5C0208EC0200206001002020
:104F2000180300209C2C0020660100206501002051
:104F300010B50446062C22D2DFE804F02103090F45
:104F4000151B0022B821104606F022FA1DE00022AF
:104F5000B921104606F01CFA17E00022BA211046CB
:104F600006F016FA11E00022BB21104606F010FAF6
:104F70000BE00022BC21104606F00AFA05E00022F0
:104F8000B821104606F004FA00BF00BF10BD10B5EE
:104F900004460B2C4DD2DFE804F04C060D141B2206
:104FA0002930373E4500002240F28711104602F0BA
:104FB00032FC3EE000224FF4C471104602F02BFC9C
:104FC00037E0002240F28911104602F024FC30E064
:104FD00000224FF4C571104602F01DFC29E00022AA
:104FE00040F28B11104602F016FC22E000224FF432
:104FF000C671104602F00FFC1BE0002240F28D113A
:10500000104602F008FC14E000224FF4C77110466D
:1050100002F001FC0DE0002240F28F11104602F078
:10502000FAFB06E000224FF4C871104602F0F3FBD1
:1050300000BF00BF10BD000070B503F02BFF044699
:105040000020F8490870F8480078052814DAF74875
:105050000068B0F5FA7F05DA00225F21012003F035
:10506000DFFA04E000222021012003F0D9FAF04801
:1050700000780B38EE4908704B2C7DD00EDC2B2CC1
:105080007BD006DC172C16D01D2C19D0272C16D15E
:1050900053E12D2C72D02E2CF9D1F0E08B2C72D054
:1050A00004DC4D2C6CD04E2CF1D18BE08D2C45D0F6
:1050B0008E2CECD123E0FDF705FB00B10224ADE11D
:1050C000D9480078052819DA3021D74802780078C5
:1050D000401CD54B1870D74881540022012003F0A2
:1050E0009FFAD3480078001DD1490870CE48007857
:1050F000032803D1084600780F3008708EE1CA48B3
:105100000078052819DA3121C74802780078401C58
:10511000C54B1870C74881540022012003F080FA63
:10512000C3480078001DC2490870BF4800780328B2
:1051300003D1084600780F3008706FE1BA48007854
:1051400005281FDA3221B84802780078401CB64B97
:105150001870B84881540022012003F061FAB44865
:105160000078001DB2490870AF480078032809D1C3
:10517000084600780F3004E062E0BEE09EE002E006
:105180003FE008704AE1A8480078052819DA332181
:10519000A54802780078401CA34B1870A54881549C
:1051A0000022012003F03CFAA1480078001DA0492C
:1051B00008709D480078032803D1084600780F3016
:1051C00008702BE198480078052819DA34219648B0
:1051D00002780078401C944B187096488154002245
:1051E000012003F01DFA92480078001D90490870D4
:1051F0008D480078032803D1084600780F300870E6
:105200000CE189480078052819DA352186480278AA
:105210000078401C844B187086488154002201207D
:1052200003F0FEF982480078001D814908707E482D
:105230000078032803D1084600780F300870EDE0AD
:1052400079480078052819DA3621774802780078FD
:10525000401C754B1870774881540022012003F0E0
:10526000DFF973480078001D714908706E480078B6
:10527000032803D1084600780F300870CEE06A4852
:105280000078052819DA3721674802780078401C31
:10529000654B1870674881540022012003F0C0F963
:1052A00063480078001D624908705F480078032851
:1052B00003D1084600780F300870AFE05A480078F4
:1052C000052819DA3821584802780078401C564BD6
:1052D0001870584881540022012003F0A1F9544865
:1052E0000078001D524908704F480078032803D108
:1052F000084600780F30087090E04B480078052889
:105300001ADA3922484801780078401C464B187058
:105310004848425400223921012003F081F94448D1
:105320000078001D424908703F480078032803D1E7
:10533000084600780F30087070E03B480578062D6D
:105340006AD2DFE805F069533D271103364800783B
:10535000401E3549087000203649334A1278885477
:1053600053203349087057E02F480078401E2E49DB
:10537000087000202F492C4A1278885453202C4959
:10538000087000228921012003F04AF944202849AD
:10539000087041E024480078401E2349087000202E
:1053A0002449214A12788854442021490870002257
:1053B0008921012003F034F926201D4908702BE0D3
:1053C00019480078401E1849087000211948164AEB
:1053D0001278815426201649087000228921012064
:1053E00003F01EF917201249087015E00E480078E6
:1053F000401E0D49087000200E490B4A127888544F
:1054000017200B49087000228921012003F008F9B8
:1054100008200749087000BF00BF00BF00BF20463A
:1054200070BD00006F0100206D01002014000020FD
:1054300065010020710100202DE9F0416A480078E3
:1054400080B101206949087000206749087006F0A2
:10545000BDFA674901EB00100668304600F06AFFAC
:105460006449086003F016FD044606F0AFFA60498F
:1054700001EB00100768384600F098FC064601F082
:1054800019FC05460521082001F05CF85748007812
:1054900000285CD0002055490870B5F5004F35D084
:1054A0000ADCDDB1B5F5D04F10D0B5F5E04F1DD019
:1054B000B5F5F04F4AD121E0B5F5584F2ED0B5F5EE
:1054C000684F33D0B5F59C3F40D137E000231A46F2
:1054D00048480168012001F074FE37E000231A46B5
:1054E00044480168012002F067F92FE000231A46C2
:1054F00040480168012002F059FA27E000231A46CB
:105500003C480168012001F08CFE1FE000231A4690
:1055100038480168012002F0E9F917E000231A4633
:1055200034480168012002F071FA0FE000231A46A6
:1055300030480168012002F03AFA07E000231A46D9
:105540002C480168012001F06BFE00BF00BF172C42
:1055500038D02D2C04D0472C41D08D2C40D118E0D0
:1055600006F034FA224901EB00100768384600F0D3
:105570001DFC064600F0EAFB1E490968884204DA71
:105580001C480068401E1B4908600120174908702C
:1055900026E006F01BFA164901EB001007683846B2
:1055A00000F004FC064600F0C7FB12490968884277
:1055B00004DD10480068401C0E49086001200B49BA
:1055C00008700DE006F002FA094901EB0010012213
:1055D000066808480168304605F0DEFD00E000BFBF
:1055E00000BF2046BDE8F0816F0100203C03002091
:1055F0009C2C00203803002070B57648007880B1DC
:1056000001207549087000207249087006F0DEF923
:10561000724901EB00100568284600F08BFE7049C6
:10562000086003F037FC04460521082000F08AFFDB
:105630006948007810B1002067490870172C73D0B2
:105640002D2C04D0472C70D08D2C55D155E06548B9
:10565000006830B101280AD002281ED003284AD1A0
:1056600030E001205E4908605B49087043E05C4817
:105670000068042802D005280DD106E0052058490D
:10568000086001205449087005E001205449086071
:105690005149087000BF00BF2DE051480068022842
:1056A00008D003280CD102204D49086001204A4946
:1056B000087005E001204A4908604749087000BFAA
:1056C00000BF18E006F082F9444901EB00100668BB
:1056D000304600F06BFB054600F038FB4049096896
:1056E000884204DA3E480068401E3D4908600120B7
:1056F0003949087000BF00BF68E03A48006830B11F
:1057000001280AD0022821D003284FD135E00120FA
:10571000334908603049087048E031480068012882
:1057200004D0052810D108E042E04EE005202C49C5
:10573000086001202849087006E004202849086014
:1057400001202549087000BF00BF2FE024480068F1
:10575000012802D002280ED106E00220204908606C
:1057600001201D49087006E003201D490860012042
:105770001949087000BF00BF18E006F027F9174963
:1057800001EB00100668304600F010FB054600F003
:10579000D3FA13490968884204DD11480068401CA7
:1057A0000F49086001200C49087000BF00BF0DE0E0
:1057B00006F00CF9094901EB0010012205680848C0
:1057C0000168284605F0E8FC00E000BF00BF204665
:1057D00070BD00006F0100203C0300209C2C0020C5
:1057E000380300201C03002010B50020B1490870C8
:1057F000B1480078082814DAB0480068B0F5FA7F9C
:1058000005DA00225F21012002F00AFF04E00022F5
:105810002021012002F004FFA94800780B38A84994
:10582000087003F037FB04462E2C6ED010DC1E2CC3
:105830006CD006DC172C1AD01B2C68D01D2C1AD16A
:105840001AE0272C76D02B2C75D02D2CF7D1ADE07B
:105850008B2C47D006DC4B2C6ED04D2C6ED04E2CB2
:10586000EDD155E08D2C2BD08E2CE8D116E0FCF735
:1058700029FF00B102241AE18F48007808280CDAC9
:1058800030218D4802780078401C8B4B18708D4871
:1058900081540022012002F0C3FE08E1864800780E
:1058A00008280CDA3121844802780078401C824BA9
:1058B0001870844881540022012002F0B1FEF6E005
:1058C0007D48007808280CDA32217B48027800787D
:1058D000401C794B18707B4881540022012002F053
:1058E0009FFEE4E07448007808280DDA33227248FD
:1058F00001780078401C704B1870724842540022A6
:105900003321012002F08CFED1E03CE08AE071E01E
:105910006948007808280CDA342167480278007852
:10592000401C654B1870674881540022012002F02A
:1059300077FEBCE087E04BE013E0FFE75E480078CD
:1059400008280DDA35225C4801780078401C5A4B53
:1059500018705C48425400223521012002F060FE9C
:10596000A5E05548007808280CDA3621524802781C
:105970000078401C504B187052488154002201207E
:1059800002F04EFE93E04C48007808280DDA3722EA
:10599000494801780078401C474B187049484254E8
:1059A00000223721012002F03BFE80E042480078CF
:1059B00008280CDA3821404802780078401C3E4B19
:1059C0001870404881540022012002F029FE6EE048
:1059D0003948007808280CDA3921374802780078ED
:1059E000401C354B1870374881540022012002F0CA
:1059F00017FE5CE030480078082812DA3248007858
:105A000078B92C222C4801780078401C2A4B187059
:105A10002C48425401202C49087000222E2102F00B
:105A2000FFFD44E02448007860B92D212248027827
:105A30000078401C204B187022488154002201201D
:105A400002F0EEFD33E01C48007800282EDD1A48F5
:105A50000078401E184908701A480978405C2C28C4
:105A600002D100201849087000201649124A127805
:105A7000885411480078072809DA002220210120E3
:105A800002F0CEFD0E4800780B380D4908700C4826
:105A900000780B380A49087000222021012002F00A
:105AA000BFFD074800780B380549087000BF00BFEC
:105AB000204610BD6F0100206D0100201400002061
:105AC00065010020710100207001002070477047BF
:105AD00010B5022000F09CF8B8B102210B4800F08C
:105AE0009CFB60B90A4800680A49884207DA0A48FC
:105AF000007820B906480068401C054908600A2063
:105B000005490870022000F07DF810BD0008014032
:105B10001404002040420F000000002010B50420B3
:105B200000F076F8B8B104210B4800F076FB60B9BC
:105B30000A4840680A49884207DA0A48007820B9CA
:105B400006484068401C054948600A20054908701D
:105B5000042000F057F810BD000801401404002094
:105B600040420F00010000207047000010B51020D7
:105B700000F04EF8B8B110210B4800F04EFB60B9B0
:105B80000A48C0680A49884207DA0A48007820B9FA
:105B90000648C068401C0549C8600A2005490870CD
:105BA000102000F02FF810BD001401401404002054
:105BB00040420F000300002010B5802000F028F8BC
:105BC000B8B180210B4800F028FB60B90A48806812
:105BD0000A49884207DA0A48007820B906488068EE
:105BE000401C054988600A2005490870802000F0A3
:105BF00009F810BD000801401404002040420F00C5
:105C000002000020014908607047000014040140B0
:105C1000064A014600201268044B0A4014331B68F0
:105C20000B4202D0002A00D001207047000401403E
:105C300030B583791949026853B30B6893430B60FD
:105C40000A1D13680468A343136002790A441368A9
:105C5000046823431360114A083213680468A3439D
:105C60001360131D1C680568AC431C604479102C3C
:105C700005D021440A68006802430A6030BD1168FB
:105C8000046821431160196800680143196030BD40
:105C90000079084401689143016030BD000401406F
:105CA0007047000004490A6822F010020A600A687E
:105CB00002430A60704700000020024004490A685D
:105CC00002F038020A600A6802430A607047000066
:105CD00000200240704710B5044640F27B1003F0EC
:105CE0008DF808B9204610BDA4F52F70C0EB001048
:105CF00000EB4000192101EB4000322190FBF1F054
:105D000000F57F70EFE7000010B504E000222021CD
:105D1000104602F085FC024800787828F6DD10BDB8
:105D2000650100200146C1EBC100024A02EB800080
:105D3000406970475CEB01080146C1EBC100024AB3
:105D400002EB8000006970475CEB01080146C1EB83
:105D5000C100024A02EB8000C06870475CEB01089A
:105D60000146C1EBC100024A52F820007047000012
:105D70005CEB010810B50446002300E05B1CC3EB9C
:105D8000C300094901EB80008068A04207D0C3EB43
:105D9000C30051F820004FF6FF718842EED118463B
:105DA000FFF7DEFF10BD00005CEB010870B5044694
:105DB0004FF0FF3625460648854206DA4FF49E72BC
:105DC00000212846FBF7DEFD0646304670BD000088
:105DD00078D4030008B50121480202F07DFD0121BD
:105DE000084602F061FD0121084602F075FD01211F
:105DF000042002F071FD0121082002F06DFD012157
:105E0000102002F069FD0121202002F065FD012132
:105E1000402002F061FD0121480402F051FD012102
:105E2000880402F04DFD0121082000F0CFF9012186
:105E3000AE4800F0CBF98620ADF8000004208DF8C4
:105E4000030003208DF802006946A94800F070F9AC
:105E50004FF40070ADF8000003208DF80200182008
:105E60008DF803006946A24800F062F94FF48060A3
:105E7000ADF8000004208DF8030069469C4800F04E
:105E800057F90120ADF8000003208DF8020004202E
:105E90008DF803006946964800F04AF92020ADF8D5
:105EA000000003208DF8020010208DF803006946E1
:105EB0008F4800F03DF94FF4D050ADF800000320BA
:105EC0008DF8020010208DF803006946884800F024
:105ED0002FF94FF47050ADF8000010208DF803003A
:105EE00003208DF802006946824800F021F9402025
:105EF000ADF8000003208DF8020014208DF8030097
:105F000069467C4800F014F98220ADF800000320B7
:105F10008DF8020004208DF803006946754800F0F2
:105F200007F90320ADF8000000208DF80300694652
:105F3000704800F0FDF82020ADF8000000208DF83A
:105F4000030069466C4800F0F3F84FF47070ADF848
:105F5000000010208DF803006946674800F0E8F85B
:105F60001020ADF8000004208DF803006946624857
:105F700000F0DEF84FF20F00ADF8000003208DF8BE
:105F8000020048208DF8030069465C4800F0D0F814
:105F90002020ADF8000003208DF8020018208DF8B5
:105FA00003006946554800F0C3F84020ADF80000F2
:105FB00003208DF8020004208DF8030069464F4845
:105FC00000F0B6F84FF48070ADF8000003208DF8B3
:105FD000020018208DF803006946484800F0A8F830
:105FE0004FF40070ADF8000003208DF8020004208B
:105FF0008DF803006946414800F09AF84FF4496073
:10600000ADF8000003208DF8020010208DF8030089
:1060100069463A4800F08CF80120ADF800001420E1
:106020008DF8030003208DF802006946344800F023
:106030007FF88020ADF8000010208DF803000320C9
:106040008DF8020069462E4800F072F84FF47F4048
:10605000ADF8000003208DF8020028208DF8030021
:106060006946274800F064F80121002000F04CF850
:10607000022024490860002008710C20487101208A
:1060800088710846FFF7D4FD0221002000F03CF89B
:1060900004201C490860002008710C204871012070
:1060A00088710846FFF7C4FD0721002000F02CF896
:1060B000802014490860002008710C2048710120DC
:1060C00088710846FFF7B4FD0421022000F01CF897
:1060D00010200C490860002008710C204871012034
:1060E00088710846FFF7A4FD08BD000030001400C9
:1060F00000080140000C0140001001400014014064
:1061000000180140AC00002010B58A0721F00304FC
:106110000649130F21440F228C689A4094438C60E7
:106120008A68984002438A6010BD00000000014068
:10613000F0B5CB78002503F00F02DB0601D58B7894
:106140001A430B884FF00F0E13F0FF0F4FF0010CA6
:1061500019D004680E880CFA05F31E409E420ED139
:10616000AF000EFA07F6B44302FA07F7CE783C43C5
:10617000282E00D14361CE78482E00D103616D1CDA
:10618000082DE7D304600B88FF2B1DD94468002538
:1061900005F108060CFA06F30E881E409E420FD148
:1061A000AF000EFA07F624EA060602FA07F43443B3
:1061B000CE78282E00D14361CE78482E00D10361DD
:1061C0006D1C082DE4D34460F0BD0000F0B5104D07
:1061D0006B68440D260184B2C0F30157B440C0F38C
:1061E0000342032F05D0C0020AD503209040834309
:1061F00007E0686823F0706220F07060686002E079
:10620000A34343F0706201B122436A60F0BD000015
:1062100000000140806880B270470246002092680A
:106220000A4200D00120704702460020D2680A428C
:1062300000D0012070474161704701617047C16023
:106240007047000070B506463546472D00DA4725F1
:106250001A48854200DD0546D2220021284603F077
:106260004BF8441E012C00DA0124601C00EB4000B6
:10627000134951F8200004EB4401114A52F821104F
:10628000401A04EB440102EB81014968691A484352
:10629000611C01EB410102EB8101496804EB4402FE
:1062A000074B03EB82025268891A90FBF1F004EB72
:1062B00044011A4652F82110084470BD54220E00C1
:1062C000080E020804480068C0EB00100349096882
:1062D00001EB8000704700003000002034000020F7
:1062E0000146481E014A52F8200070472C0C00203D
:1062F00010B503460A46184600F00CF9044610464D
:1063000000F0BDF8204410BD10B504460748844293
:1063100009DA2046FFF74AFDC0EBC000044901EB53
:106320008000806810BD0020FCE7000078D40300E6
:106330005CEB010870B504460E48844218DA20462A
:10634000FFF734FD054600F09BFC30B12046FFF717
:10635000DBFF054602F022FE70BD2046FFF726FD5A
:10636000C0EBC000044901EB800040680068F3E71F
:106370000020F1E778D403005CEB01080146481ED9
:10638000014A52F820007047400F002070B50446C3
:106390000D4629462046FFF7ABFF00F17006304658
:1063A00002F02CFD70BD70B504460D46294620460E
:1063B000FFF79EFF00F17106304602F01FFD70BD31
:1063C00070B50446204600F0A5F800F16C0528469B
:1063D00002F014FD70BD70B50446204600F09AF836
:1063E00000F18605284602F009FD70BD0146481EF1
:1063F000014A52F820007047180F00200146002083
:10640000002201291BDB062919DC072911D2DFE84C
:1064100001F0100406080A0C0E00012209E0022215
:1064200007E0042205E0082203E0102201E0202218
:1064300000BF00BF024B1B68134003B90120704727
:106440006C00002002461146002900DA0021B1F557
:10645000805F01DB40F6FF714FF47A704843C1F56D
:10646000805390FBF3F0704770B50446204600F06F
:1064700051F800F16D05284602F0C0FC70BD0146E0
:106480008800704770B504460D4629462046FFF740
:106490002FFF00F16E06304602F0B0FC70BD70B503
:1064A00004460D4629462046FFF722FF00F16F06FD
:1064B000304602F0A3FC70BD10B54FF4C17002F07D
:1064C0009DFCB8B110480468B4F5967F03DB40F238
:1064D0001450844207DD0D48006820B901210020D6
:1064E00003F0F2FD0EE00A4804600121002002F0F2
:1064F00025FF07E04FF42F700549086001210020B7
:1065000002F01CFF10BD0000F40B0020C4000020AE
:10651000380000200146481E00EBC00000EB4000A0
:10652000704710B540F2911002F068FC10BD0146B2
:1065300001F114006422504340F6FF7290FBF2F028
:1065400070470000024B1970024B18707047000032
:10655000660100206501002000BFFEE7704770471C
:106560007047704710B501210148FFF766FE10BD66
:106570000018014002494CF6CC400860704700000A
:106580000030004002494AF6AA2008607047000027
:106590000030004001494860704700000030004072
:1065A00001498860704700000030004001490860E0
:1065B000704700000030004010B545F25550FFF71D
:1065C000F5FF0520FFF7E6FF40F6C410FFF7E8FFF0
:1065D000FFF7D8FFFFF7CEFF10BD000070B5CD4824
:1065E0000078002843D0CC480068CD225043CB4AE5
:1065F00002EB800001228168002001F0CDF8032128
:106600000220FFF79FFF02F01DFF05F0DFF90446AF
:10661000002100F0B9FF05F0D9F9C4B2002301222E
:106620002146184601F0F4F905F0D0F9C4B2002271
:106630002146104600F004FF04210846FFF782FFC0
:1066400000220821022001F0EBFF00220921022094
:1066500001F0E6FF00220921022001F0E1FF002203
:106660000921022001F0DCFF0020AA49087005F092
:10667000ADF9AB4901EB001005682846FFF796FB22
:10668000044600F017FBC0F30A0100297ED1C012B6
:106690002B287BD2DFE800F01618191A7A7A7A7A5A
:1066A0007A677F7A7A1B1C1D1E1F7A7A2551177A0A
:1066B0007A269E272820212223247A7A7A3D7A2955
:1066C0007A7AE60000BF00BF00BF00BF00BF00BF76
:1066D00000BF00BF00BF00BF00BF00BF00BF00BFC2
:1066E00000BF00BF00BF00BF00BF00220A21022080
:1066F00001F096FF05F06AF9894901EB0010046882
:106700002046FFF717FE8749086006208649086083
:10671000FDE000220A21022001F082FF05F056F977
:106720007F4901EB001004682046FFF703FE7D4916
:1067300008601D207C490860E9E000220B2102204E
:1067400001F06EFF05212120FFF7FCFE00223A2117
:10675000012001F065FF05210820FFF7F3FE072067
:1067600071490860D3E000220B21022001F058FF9C
:1067700005212120FFF7E6FE00223A21012001F049
:106780004FFF05210820FFF7DDFE00E0B2E0082002
:1067900065490860BBE000220B21022001F040FFA8
:1067A00005212120FFF7CEFE00223A21012001F031
:1067B00037FF05214220FFF7C5FE00223A210120C4
:1067C00001F02EFF05210820FFF7BCFE09205649E5
:1067D00008609CE000220B21022001F021FF05212E
:1067E0000820FFF7AFFE00228921012001F018FFE9
:1067F0004E480078001D4D49087000228921012073
:1068000001F00EFF49480078001D48490870002239
:106810008921012001F004FF44480078001D43490C
:10682000087000222D21012001F0FAFE3F48007877
:10683000001D3E49087000228921012001F0F0FE70
:106840003A480078001D394908700022892101204A
:1068500001F0E6FE05210820FFF774FE0A20324908
:10686000086054E005F0B2F82D4901EB001004680F
:106870002046FFF75FFD2B49086000220B21022014
:1068800001F0CEFE05210820FFF75CFE25480068D8
:10689000010E0022012001F0C3FE24480078001DF3
:1068A0002249087000221F480068C0F307410120F8
:1068B00001F0B6FE1D480078001D1C49087000223A
:1068C00018480088C0F30721012001F0A9FE1748ED
:1068D0000078001D15490870124801780022012037
:1068E00001F09EFE05210820FFF72CFE1E200E4918
:1068F00008600CE000220B21022001F091FE05212E
:106900000820FFF71FFE0B200749086000BF00BFEB
:1069100070BD00006F010020E8020020EC5C02085E
:106920009C2C00203803002000030020650100207B
:1069300070B505460C46B548007808287BDCB3489E
:106940000078082814DAB2480068B0F5FA7F05DA52
:1069500000225F21012001F063FE04E000222021DB
:10696000012001F05DFEAB4800780B38A9490870A2
:106970004B2D7BD00CDC2B2D79D004DC1D2D14D0BD
:10698000272D2AD114E12D2D72D02E2DF9D1C3E05F
:106990008B2D57D004DC4D2D6BD04E2DF1D16FE0F7
:1069A0008D2D34D08E2DECD118E098480078082831
:1069B00013DA3021954802780078401C934B187008
:1069C0009548815424B90022012001F029FE04E0F9
:1069D00000222A21012001F023FE15E18B480078D6
:1069E000082813DA3121894802780078401C874B47
:1069F00018708948815424B90022012001F010FE4A
:106A000004E000222A21012001F00AFEFCE07F4878
:106A10000078082815DA32227C4801780078401C7A
:106A20007A4B18707C48425434B90022322101203C
:106A300001F0F6FD05E0E8E000222A21012001F046
:106A4000EFFDE1E071480078082818DA33226F483A
:106A500001780078401C6D4B18706F4842544CB957
:106A600000223321012001F0DBFD08E03BE085E05E
:106A70006BE01FE000222A21012001F0D1FDC3E0DC
:106A800062480078082814DA3422604801780078D7
:106A9000401C5E4B1870604842542CB900223421CF
:106AA000012001F0BDFD04E000222A21012001F0B7
:106AB000B7FDA9E055480078082813DA3521534876
:106AC00002780078401C514B18705348815424B907
:106AD0000022012001F0A4FD04E000222A2101206F
:106AE00001F09EFD90E049480078082813DA36212D
:106AF000464802780078401C444B18704648815440
:106B000024B90022012001F08BFD04E000222A219B
:106B1000012001F085FD77E03C480078082813DA71
:106B200037213A4802780078401C384B18703A48B0
:106B3000815424B90022012001F072FD04E00022FA
:106B40002A21012001F06CFD5EE030480078082821
:106B500013DA38212D4802780078401C2B4B18702E
:106B60002D48815424B90022012001F059FD04E090
:106B700000222A21012001F053FD45E0234800783E
:106B8000082814DA3922214801780078401C1F4B6C
:106B90001870214842542CB900223921012001F0FB
:106BA0003FFD04E000222A21012001F039FD2BE005
:106BB00016480078002826DD14480078401E134946
:106BC000087000201449114A127888540F48007840
:106BD000072809DA00222021012001F021FD0D48BB
:106BE00000780B380B4908700A4800780B380949BF
:106BF000087000222021012001F012FD05480078D4
:106C00000B380449087000BF00BF70BD6D01002043
:106C100014000020650100207101002010B5102132
:106C20000448FFF70AFB4FF480610348FFF703FBBA
:106C3000012010BD00080140001001400146084835
:106C40000068CD225043074A02EB8000143000EB6D
:106C50000110C068006808B1012070470020FCE7FF
:106C6000E8020020EC5C02080146C1EBC100034AC7
:106C700002EB8000008B00F4FE6070475CEB0108C3
:106C80000146C1EBC100034A02EB8000007EC0F365
:106C9000400070475CEB01080146C1EBC100044AAB
:106CA00002EB8000007E00F0010080F001007047E0
:106CB0005CEB01080146C1EBC100034A02EB800016
:106CC000806900F4FF2070475CEB01080146C1EBCE
:106CD000C100054A52F820004FF6FF72904201D1E0
:106CE000012070470020FCE75CEB01080146CD2045
:106CF0004843054A02EB8000C068006808B10120E3
:106D000070470020FCE70000EC5C0208024600200F
:106D1000002111E00A4B03EB01135B681B689342EF
:106D200007D1074B03EB0113DB681B680BB9012389
:106D300000E000231846491C08B90229EADB704725
:106D4000E400002030B502460B4801680B48036898
:106D50000EE001EB41000A4C54F82000904201D1B2
:106D6000012030BD481C142490FBF4F504FB1501F0
:106D70009942EED10020F4E7DC000020E000002082
:106D8000280E002038B500250820ADF8000010209E
:106D90008DF8030003208DF8020069464A48FFF78A
:106DA000C7F908214848FFF746FAFCF77FF946483B
:106DB000FFF730FA04130820ADF8000048208DF8E2
:106DC000030069464048FFF7B3F90F2C76D1042041
:106DD000ADF8000010208DF8030003208DF80200AC
:106DE00069463948FFF7A4F904213748FFF723FA29
:106DF000FCF75CF93448FFF70DFA04130420ADF8F2
:106E0000000048208DF8030069462F48FFF790F9ED
:106E10000F2C4FD10220ADF8000010208DF8030098
:106E200003208DF8020069462748FFF781F9022107
:106E30002548FFF700FAFCF739F92348FFF7EAF98C
:106E400004130220ADF8000048208DF803006946C5
:106E50001D48FFF76DF90F2C27D10120ADF8000078
:106E600010208DF8030003208DF8020069461648B3
:106E7000FFF75EF901211448FFF7DDF9FCF716F979
:106E80001148FFF7C7F904130120ADF800004820AE
:106E90008DF8030069460C48FFF74AF90F2C00D122
:106EA0000FE0E0B240F010050BE0E0B240F020054A
:106EB00007E003E0E0B240F0400502E0E0B240F05D
:106EC0008005284638BD00000014014070B500F070
:106ED00035F8002417E0002511E0A107080E294627
:106EE00003F084F9002606E000222146012004F088
:106EF000B1F9701CC6B2402EF6DB681CC5B2082D75
:106F0000EBDB601CC4B2022CE5DB00F023F870BDA3
:106F100010B548F220010748FFF78DF94FF4804182
:106F20000448FFF78AF940210348FFF784F9FFF787
:106F3000CDFF10BD000C01400008014010B53E22FD
:106F40000021084604F086F93E220121002004F0C9
:106F500081F910BD10B53F220021084604F07AF9EE
:106F60003F220121002004F075F910BD70B50546DF
:106F70000C466E201C490870012D28D11B48006862
:106F8000C8280CDA00201A490870E2B2FE2101F08C
:106F900047FBE2B22021002001F042FB23E013482E
:106FA0000068B0F5FA7F1EDD10480068B0F52F7F4D
:106FB00019DA01200E490870E2B2F821002001F030
:106FC0002FFBE2B22021002001F02AFB0BE0022D72
:106FD00009D1E2B2F721002001F022FBE2B2FD214B
:106FE000002001F01DFB70BD650100201400002091
:106FF0004B03002000BFFEE77047000010B54FF4C0
:107000008031C80200F0A0F84FF4E06000F092F880
:10701000284800F051F826202649087000204870C2
:1070200001208870C870084600F046F827202149E2
:1070300008700020487001208870C870084600F071
:107040003BF803201B49087000204870022088701C
:107050000120C870084600F02FF807201549087075
:107060000020487088700120C870084600F024F89D
:107070000820104908700020487088700120C870EE
:10708000084600F019F80A200A49087000204870E4
:1070900088700120C870084600F00EF817200549D6
:1070A00008700020487088700120C870084600F001
:1070B00003F810BDA5000020F0B50F22C3780178B9
:1070C00001244FF0E0263BB3184B1B6803F4E06348
:1070D000C3F5E0631D0AC5F10403EA4045789D400D
:1070E000837813402B431A018B07DF0E21F0030333
:1070F0000F49BA405D182968FF23BB4099431A40E5
:1071000011432960007800F01F018C40400906EB14
:107110008000C0F80041F0BD01F01F008440480924
:1071200006EB8000C0F88041F0BD00000CED00E0EF
:1071300000E400E00249084302490860704700008B
:107140000000FA050CED00E0024A1140014302483C
:107150000160704780FFFF1F08ED00E00120002163
:107160000AE0084A02EB0112D26812680AB9012249
:1071700000E000221046491C022901DA0028F0D163
:1071800070470000E400002010B50848006820B9EE
:1071900001200649086003F023FC03F04BF903F0DB
:1071A000C9F901F077FE0446204610BD0C0300200B
:1071B00070470000014908627047000000000E425D
:1071C00070472DE9F04180460C4615461E4604F1F5
:1071D000950003F099FA074685B104E03246202174
:1071E000404601F01DFA38467F1C0628F6DB324681
:1071F00004F19501404604F0CBF80FE0324604F16B
:107200009501404604F0C4F804E03246202140468F
:1072100001F006FA38467F1C0628F6DBBDE8F0814F
:10722000704770472DE9F04107460D4690461E46CF
:1072300080240C4800780C380A4908700EE005EAF2
:10724000040028B132463021384601F0E9F904E063
:1072500032463121384601F0E3F96410002CEED1BA
:10726000BDE8F081650100202DE9F04106460C469D
:1072700090461D460020244908702A4620213046A9
:1072800001F0CEF90A2094FBF0F00A2190FBF1F214
:1072900001FB12003030C7B22A463946304601F0B1
:1072A000BFF90A2094FBF0F100FB11403030C7B267
:1072B0002A463946304601F0B3F92A462D21304698
:1072C00001F0AEF94FF47A7094FBF0F00A2190FBD4
:1072D000F1F201FB12003030C7B22A46394630467F
:1072E00001F09EF9642094FBF0F00A2190FBF1F28A
:1072F00001FB12003030C7B22A463946304601F051
:107300008FF9BDE8F0810000640100202DE9F0470D
:107310000746884691461E46474800783038464919
:107320000870464D2C6804F00F00FAF71CFA8246EC
:1073300032465146384601F073F9C4F30320FAF798
:1073400012FA824632465146384601F069F9C4F3D2
:107350000340FAF708FA824632465146384601F0B1
:107360005FF9C4F30360FAF7FEF9824632465146EC
:10737000384601F055F932462D21384601F050F9D2
:107380002D1D2C6804F00F00FAF7EDF98246324605
:107390005146384601F044F9C4F30320FAF7E3F903
:1073A000824632465146384601F03AF9C4F303406A
:1073B000FAF7D9F9824632465146384601F030F99B
:1073C000C4F30360FAF7CFF9824632465146384695
:1073D00001F026F932462D21384601F021F92D1D04
:1073E0002C6804F00F00FAF7BEF982463246514687
:1073F000384601F015F9C4F30320FAF7B4F98246D0
:1074000032465146384601F00BF9C4F30340FAF70F
:10741000AAF9824632465146384601F001F9C4F3D2
:107420000360FAF7A0F9824632465146384601F029
:10743000F7F8BDE8F087000065010020E8F7FF1FBE
:107440002DE9F04105460C46164671204C4908705E
:107450004C4901EB04110868FEF7A8FC8046FFF7D1
:1074600003FC074607F00F0000286ED138111628DC
:107470007DD2DFE800F07C0B1C22287C7C2E343A85
:1074800040464C52585E647C7C6B7C7140F27B10B1
:1074900001F0B4FC28B932460021284603F078FFF9
:1074A00004E032461021284603F072FF65E03246C0
:1074B0000121284603F06CFF5FE032460221284696
:1074C00003F066FF59E032460321284603F060FFCF
:1074D00053E032460421284603F05AFF4DE032467D
:1074E0000521284603F054FF47E03246062128468E
:1074F00003F04EFF41E032460721284603F048FFE3
:107500003BE032460821284603F042FF35E0324690
:107510000921284603F03CFF2FE032460A21284685
:1075200003F036FF29E032460B21284603F030FFF6
:1075300023E032460C21284603F02AFF1DE03246A4
:107540000D21284603F024FF17E010E032460E21FB
:10755000284603F01DFF10E03246F021284601F0D6
:107560005FF83246F521284601F05AF805E0324628
:107570000F21284603F00CFF00BF00BFBDE8F081DB
:10758000650100209C2C002070B504460D4607487C
:1075900000EB04102A464168002003F0F9FE2A4659
:1075A0000F21002003F0F4FE70BD00009C2C002091
:1075B0002DE9F04105460C4616460027672001F0EC
:1075C0001DFC06283FD2DFE800F0030C16202A3409
:1075D00004EB4401234A52F83100F9F701F8074659
:1075E00031E004EB44011F4A02EBC1014868F8F79F
:1075F000F7FF074627E004EB44011A4A02EBC101FA
:107600008868F8F7EDFF07461DE004EB4401154AD2
:1076100002EBC101C868F8F7E3FF074613E004EB8B
:107620004401104A02EBC1010869F8F7D9FF074687
:1076300009E004EB44010B4A02EBC1014869F8F789
:10764000CFFF074600BF00BF07EB4700C0F1400077
:107650000549087032462146284603F099FEBDE8E8
:10766000F08100006C4902086501002010B500217E
:107670000846FEF767FF00220221084600F0D0FF0F
:1076800000212020FEF75EFF00220321022000F0EF
:10769000C7FF00214020FEF755FF002203210220F2
:1076A00000F0BEFF00216020FEF74CFF0022042105
:1076B000022000F0B5FF04210020FEF743FF002266
:1076C0000521022000F0ACFF04212020FEF73AFF44
:1076D00000220621022000F0A3FF04214020FEF733
:1076E00031FF00220621022000F09AFF04216020D1
:1076F000FEF728FF00220721022000F091FF10BDB5
:1077000010B50020224908702249087000220D217E
:10771000022000F085FF20201D49087000220E2164
:10772000022000F07DFF40201949087000220E2140
:10773000022000F075FF60201549087000220F211B
:10774000022000F06DFF002011490870042011494B
:10775000087000221021022000F062FF20200C4956
:10776000087000221121022000F05AFF4020084931
:10777000087000221121022000F052FF602004490D
:10778000087000221221022000F04AFF10BD000004
:10779000650100206601002070B504460D461646BE
:1077A000FFF764FF00210846FEF7CCFE324629466B
:1077B0002046FFF7FDFE70BD2DE9F04180460C46E6
:1077C00015461E4604F1170002F09EFF074685B1DC
:1077D00004E032462021404600F022FF38467F1C5C
:1077E0000628F6DB324604F11701404603F0D0FDCF
:1077F0000FE0324604F11701404603F0C9FD04E0F2
:1078000032462021404600F00BFF38467F1C0628F8
:10781000F6DBBDE8F0812DE9F04106460D4617463E
:10782000284601F0EBFA0446210E3A46304600F0B5
:10783000F7FE3A46C4F30741304600F0F1FE3A46FF
:10784000C4F30721304600F0EBFEE1B23A46304681
:1078500000F0E6FEBDE8F0812DE9F04107460C4658
:1078600015461E4605B332462021384600F0D8FEA4
:1078700032462021384600F0D3FE210E32463846EB
:1078800000F0CEFE3246C4F30741384600F0C8FE91
:107890003246C4F30721384600F0C2FEE1B2324658
:1078A000384600F0BDFE1FE0210E3246384600F09B
:1078B000B7FE3246C4F30741384600F0B1FE324607
:1078C000C4F30721384600F0ABFEE1B23246384639
:1078D00000F0A6FE32462021384600F0A1FE3246D6
:1078E0002021384600F09CFEBDE8F0817047000082
:1078F0002DE9F04106460C4690461D4600202949D8
:107900000870294894FBF0F00A2190FBF1F201FB8A
:1079100012003030C7B22A463946304600F080FEA9
:1079200042F2107094FBF0F00A2190FBF1F201FB9F
:1079300012003030C7B22A463946304600F070FE99
:107940004FF47A7094FBF0F00A2190FBF1F201FB06
:1079500012003030C7B22A463946304600F060FE89
:107960002A462D21304600F05BFE0A2094FBF0F001
:107970000A2190FBF1F201FB12003030C7B22A4617
:107980003946304600F04CFE0A2094FBF0F100FB33
:1079900011403030C7B22A463946304600F040FE2A
:1079A000BDE8F08164010020A086010070472DE948
:1079B000F04180460C4615461E4604F1110002F0C7
:1079C000A3FE074685B104E032462021404600F080
:1079D00027FE38467F1C0628F6DB324604F11101EB
:1079E000404603F0D5FC0FE0324604F11101404659
:1079F00003F0CEFC04E032462021404600F010FEA9
:107A000038467F1C0628F6DBBDE8F0817047000091
:107A10002DE9F84F06460D4617469846A84901EB52
:107A200005110868FEF7C2F98246FFF743F981465F
:107A3000A34901EB05110868FEF77CFC04464C20C5
:107A4000A0490870C9F30A00002823D14FEAE920B1
:107A50002B281FD2DFE800F0AC1E1E1E161F303789
:107A60003E454C5D1EA2B6C0CA1E7E261E9B1EE869
:107A70001E1EF8D41EDE1E1E1E1EF7F61E1E56F516
:107A80001E1EF400062043463A462146009030462A
:107A900000F032FD11E143463A462146304600F0FF
:107AA000C9FC0AE140208749087043463A4621460E
:107AB000304600F065F900E143463A46214630463B
:107AC00000F056FCF9E043463A462146304600F0C5
:107AD000A5FAF2E043463A462146304600F0F4F873
:107AE000EBE043463A462146304600F041FAE4E0F6
:107AF00044207449087043463A462146304600F017
:107B0000B3F9DAE043463A462146304600F0E8FA57
:107B1000D3E040F27B1001F071F930B943463A46A8
:107B20002146304600F054FB13E0A4F52F70C0EB63
:107B3000001000EB4000192101EB4000322190FBC6
:107B4000F1F000F57F7A43463A465146304600F060
:107B50003FFBB2E040F27B1001F050F930B94346F0
:107B60003A462146304600F065FC0FE0C4EB0410B5
:107B700000EB4000192101EB4000322190FBF1FAAB
:107B800043463A465146304600F054FC95E04346A1
:107B90003A4621463046FFF767FB8EE04C204949C4
:107BA000087043463A4621463046FFF70AFB84E018
:107BB0004C204449087043463A4621463046FFF778
:107BC000FBFD7AE04C203F49087043463A46214687
:107BD0003046FFF7EBFE70E04C203A490870434610
:107BE0003A4621463046FFF71CFB66E04C203549FB
:107BF000087043463A4621463046FFF777FE5CE080
:107C00004C203049087043463A4621463046FFF73B
:107C1000FDFE52E04C202B49087043463A4621466F
:107C20003046FFF7C4FE48E040F27B1001F0E6F872
:107C300058B943463A462146304600F031FB18E039
:107C400034E02CE01DE015E022E0A4F52F70C0EB3D
:107C5000001000EB4000192101EB4000322190FBA5
:107C6000F1F000F52F7A43463A465146304600F08F
:107C700017FB22E043463A4621463046FFF7D2FA48
:107C80001BE043463A4621463046FFF73FFB14E0EF
:107C900043463A4621463046FFF72AFE0DE043466A
:107CA0003A4621463046FFF7BBFA06E043463A46DD
:107CB00021463046FFF7D0FD00BF00BFBDE8F88F7A
:107CC0009C2C0020650100202DE9F04106460C4661
:107CD00090461D4600202949087042F2107094FB1E
:107CE000F0F00A2190FBF1F201FB12003030C7B234
:107CF0002A463946304600F093FC2A462E2130466B
:107D000000F08EFC4FF47A7094FBF0F00A2190FBA7
:107D1000F1F201FB12003030C7B22A463946304634
:107D200000F07EFC642094FBF0F00A2190FBF1F25D
:107D300001FB12003030C7B22A463946304600F007
:107D40006FFC0A2094FBF0F00A2190FBF1F201FB9A
:107D500012003030C7B22A463946304600F060FC87
:107D60000A2094FBF0F100FB11403030C7B22A46E4
:107D70003946304600F054FCBDE8F0816401002033
:107D80002DE9F04106460C4617461D4600203449B1
:107D90000870344894FBF0F000F0FF082B463A4698
:107DA0004146002000F024FD42F2107094FBF0F0F8
:107DB0000A2190FBF1F201FB1200303000F0FF08C5
:107DC0002A464146304600F02BFC2A462E213046FA
:107DD00000F026FC4FF47A7094FBF0F00A2190FB3F
:107DE000F1F201FB1200303000F0FF082A46414654
:107DF000304600F015FC642094FBF0F00A2190FB63
:107E0000F1F201FB1200303000F0FF082A46414633
:107E1000304600F005FC2A462E21304600F000FCDA
:107E20000A2094FBF0F00A2190FBF1F201FB120012
:107E3000303000F0FF082A464146304600F0F0FBA3
:107E40000A2094FBF0F100FB1140303000F0FF08F5
:107E50002A464146304600F0E3FBBDE8F0810000D1
:107E600064010020A08601002DE9F04780460D4600
:107E700016461F462C4626B13A462021404600F0C1
:107E8000CFFB48F6A04094FBF0F00A2190FBF1F202
:107E900001FB1200303000F0FF093A4649464046E7
:107EA00000F0BEFB4FF4616094FBF0F00A2190FB00
:107EB000F1F201FB1200303000F0FF093A4649466A
:107EC000404600F0ADFB4FF4616094FBF0F100FB25
:107ED00011443A463A21404600F0A2FB4FF4167096
:107EE00094FBF0F00A2190FBF1F201FB120030301C
:107EF00000F0FF093A464946404600F091FB3C201D
:107F000094FBF0F00A2190FBF1F201FB12003030FB
:107F100000F0FF093A464946404600F081FB3A46E8
:107F20003A21404600F07CFB3C2094FBF0F100FB42
:107F300011400A2190FBF1F0303000F0FF093A4681
:107F40004946404600F06CFB3C2094FBF0F100FBFE
:107F500011400A2190FBF1F201FB1200303000F0D9
:107F6000FF093A464946404600F05AFBBDE8F08713
:107F70002DE9F04107460C4615461E4625B132460E
:107F80002021384600F04CFB4FF4167094FBF0F0C3
:107F90000A2190FBF1F201FB1200303000F0FF08E3
:107FA00032464146384600F03BFB3C2094FBF0F063
:107FB0000A2190FBF1F201FB1200303000F0FF08C3
:107FC00032464146384600F02BFB32463A213846CD
:107FD00000F026FB3C2094FBF0F100FB11400A214D
:107FE00090FBF1F0303000F0FF0832464146384651
:107FF00000F016FB3C2094FBF0F100FB11400A213D
:1080000090FBF1F201FB1200303000F0FF08324625
:108010004146384600F004FBBDE8F0812DE9F0410F
:1080200006460C4617461D4600202C49087042F2B1
:10803000107094FBF0F0642190FBF1F201FB120050
:1080400000F0FF082B463A464146304600F0D0FB90
:108050004FF47A7094FBF0F00A2190FBF1F201FBEF
:108060001200303000F0FF082A464146304600F04A
:10807000D7FA2A462E21304600F0D2FA642094FB2B
:10808000F0F00A2190FBF1F201FB1200303000F019
:10809000FF082A464146304600F0C2FA0A2094FB07
:1080A000F0F00A2190FBF1F201FB1200303000F0F9
:1080B000FF082A464146304600F0B2FA0A2094FBF7
:1080C000F0F100FB1140303000F0FF082A46414635
:1080D000304600F0A5FABDE8F08100006401002000
:1080E0002DE9F84307460D4690461E4600203749C5
:1080F00008702C46B4F52F7F0ADBA4F52F740620F8
:108100003346424621460090384600F0F5F95BE0E0
:1081100000202E490870C4F52F7442F2107094FBB1
:10812000F0F00A2190FBF1F201FB120000F0FF09D0
:10813000334642464946384603F0F0F94FF47A7028
:1081400094FBF0F00A2190FBF1F201FB120000F029
:10815000FF09334642464946384603F0DFF96420BA
:1081600094FBF0F00A2190FBF1F201FB120000F009
:10817000FF09334642464946384603F0CFF90A2004
:1081800094FBF0F00A2190FBF1F201FB120000F0E9
:10819000FF09334642464946384603F0BFF90B48CB
:1081A000007820B932462D21384600F039FA0A20ED
:1081B00094FBF0F100FB1140303000F0FF09324633
:1081C0004946384600F02CFABDE8F88364010020E7
:1081D0002DE9F04707460D4690461E462C46B4F55D
:1081E0002F7F08DBA4F52F743346424621463846DC
:1081F00000F020F94FE0002028490870C4F52F74E2
:108200004FF47A7094FBF0F00A2190FBF1F201FB3D
:10821000120000F0FF09334642464946384603F053
:108220007DF9642094FBF0F00A2190FBF1F201FB50
:10823000120000F0FF09334642464946384603F033
:108240006DF91648007820B932462D21384600F0E5
:10825000E7F90A2094FBF0F00A2190FBF1F201FB10
:108260001200303000F0FF0932464946384600F02F
:10827000D7F932462E21384600F0D2F90A2094FB75
:10828000F0F100FB1140303000F0FF093246494662
:10829000384600F0C5F9BDE8F08700006401002011
:1082A0002DE9F04707460D4690461E462C46B4F58C
:1082B0002F7F08DBA4F52F7433464246214638460B
:1082C00000F0B8F84FE0002028490870C4F52F747A
:1082D0004FF47A7094FBF0F00A2190FBF1F201FB6D
:1082E000120000F0FF09334642464946384603F083
:1082F00015F9642094FBF0F00A2190FBF1F201FBE8
:10830000120000F0FF09334642464946384603F062
:1083100005F91648007820B932462D21384600F07C
:108320007FF90A2094FBF0F00A2190FBF1F201FBA7
:108330001200303000F0FF0932464946384600F05E
:108340006FF932462E21384600F06AF90A2094FB74
:10835000F0F100FB1140303000F0FF093246494691
:10836000384600F05DF9BDE8F087000064010020A8
:108370002DE9F04106460C4617461D4600202C49C3
:10838000087042F2107094FBF0F00A2190FBF1F2B9
:1083900001FB120000F0FF082B463A4641463046EA
:1083A00000F026FA4FF47A7094FBF0F00A2190FB6B
:1083B000F1F201FB120000F0FF082B463A4641465D
:1083C000304600F015FA642094FBF0F00A2190FB8F
:1083D000F1F201FB1200303000F0FF082A4641465E
:1083E000304600F01DF92A462E21304600F018F9DB
:1083F0000A2094FBF0F00A2190FBF1F201FB12003D
:10840000303000F0FF082A464146304600F008F9B7
:108410000A2094FBF0F100FB1140303000F0FF081F
:108420002A464146304600F0FBF8BDE8F0810000E6
:10843000640100202DE9F04106460C4617461D4612
:1084400000202C49087042F2107094FBF0F00A21D1
:1084500090FBF1F201FB120000F0FF082B463A46B8
:108460004146304600F0C4F94FF47A7094FBF0F0C6
:108470000A2190FBF1F201FB120000F0FF082B46ED
:108480003A464146304600F0B3F9642094FBF0F0E0
:108490000A2190FBF1F201FB120000F0FF082B46CD
:1084A0003A464146304600F0A3F90A2094FBF0F02A
:1084B0000A2190FBF1F201FB1200303000F0FF08BE
:1084C0002A464146304600F0ABF82A462E21304677
:1084D00000F0A6F80A2094FBF0F100FB11403030C8
:1084E00000F0FF082A464146304600F099F8BDE802
:1084F000F0810000640100202DE9F04707460C469A
:1085000090461E46089D002037490870062D0FDB57
:10851000364894FBF0F00A2190FBF1F201FB1200C7
:1085200000F0FF09334642464946384600F060F9FC
:10853000052D10DB42F2107094FBF0F00A2190FB45
:10854000F1F201FB120000F0FF09334642464946B2
:10855000384600F04DF9042D10DB4FF47A7094FB8F
:10856000F0F00A2190FBF1F201FB120000F0FF098C
:10857000334642464946384600F03AF9032D0FDBB0
:10858000642094FBF0F00A2190FBF1F201FB120051
:1085900000F0FF09334642464946384600F028F9C4
:1085A000022D0FDB0A2094FBF0F00A2190FBF1F280
:1085B00001FB120000F0FF093346424649463846A7
:1085C00000F016F9012D0CDB0A2094FBF0F100FB02
:1085D0001140303000F0FF0932464946384600F07D
:1085E0001FF8BDE8F087000064010020A0860100AC
:1085F00010B54FF4BE7000F001FC08B1012010BDB1
:108600000020FCE70448006820B10448006808B96D
:10861000012070470020FCE7A00000209C00002003
:1086200070B506460C46154626B1012E07D0022E1F
:108630000FD109E02946204600F00EF809E029464E
:10864000204600F043F804E02946204600F08AF86E
:1086500000BF00BF70BD00002DE9F04105460E4689
:10866000002706B1FF27202D00DA202500241EE078
:1086700013480078802818DA1248017810480078EA
:1086800001F0B4FDA5F120000F4B03EBC000005D2D
:1086900080EA07020A4800788111012002F0DAFD21
:1086A00007480078401C06490870601CC4B2082CBA
:1086B000DEDB03480078801E01490870BDE8F081C8
:1086C0006501002066010020EC1B02082DE9F04145
:1086D00005460F464FF000080FB14FF0FF08202D60
:1086E00000DA202500242DE0002622E01A48007838
:1086F00080281CDA194800782044C1B21648007856
:1087000001F074FDA5F12000154B03EB401006EBC2
:108710000413C05C80EA08020F4800788111012030
:1087200002F098FD0C480078401C0B490870701C42
:10873000C6B2102EDADB08480078103806490870F7
:10874000601CC4B2022CCFDB034800780B30024916
:108750000870BDE8F081000065010020660100207E
:10876000F42202082DE9F04106460F464FF00008BA
:108770000FB14FF0FF0800242BE0002520E019483E
:10878000007880281ADA184800782044C1B21548C9
:10879000007801F02BFD154800EBC61005EB4413E3
:1087A000C05C80EA08020F4800788111012002F0C5
:1087B00051FD0C480078401C0A490870681CC5B27D
:1087C000202DDCDB07480078203806490870601C43
:1087D000C4B2042CD1DB034800781630014908707C
:1087E000BDE8F0816501002066010020143F020809
:1087F0002DE9F04107460C4615461E4614B90B48B4
:10880000007850B101200949087004F13000C1B26C
:1088100032463846FFF704FF05E025B132462021F5
:108820003846FFF7FDFEBDE8F0810000640100203E
:1088300010B504462046FEF785FA30BB13480068A1
:1088400000EB4000124941F820402046FDF7B8FDFA
:108850000E49096801EB41010D4A02EB81014860B4
:108860002046FDF7B8FD0949096801EB4101084AB6
:1088700002EB8101886005480068401C142190FBD0
:10888000F1F201FB12000149086010BDE000002078
:10889000280E0020034A516821F4404101435160F1
:1088A0007047000000100240044A0029516901D0BD
:1088B000014300E081435161704700000010024015
:1088C000044A0029D16901D0014300E08143D1610C
:1088D0007047000000100240044A0029916901D04D
:1088E000014300E0814391617047000000100240A5
:1088F00010B500F035F84FF4803000F0C3F800F008
:1089000029F91649087008460078012824D110205A
:10891000FDF7C8F90220FDF7D1F9002000F0A8F812
:10892000002000F0E5F84FF4806000F0D7F84FF435
:108930004040FFF7AFFF00214FF4803000F0E8F82F
:10894000012000F0DFF800BF392000F079F800289E
:10895000FAD0022000F0F4F810BD0000A4000020BE
:108960000B48016841F0010101604168094A11406A
:1089700041600168084A11400160016821F48021CA
:108980000160416821F4FE0141600021816070476F
:10899000001002400000FFF8FFFFF6FE224A10B56B
:1089A0005168224B11F00C0103D0042903D008298F
:1089B00003D0036015E01E4912E05168022301F460
:1089C000701103EB9141536813F4803F04D0536856
:1089D0009B0303D5174B02E0174B00E0144B5943A0
:1089E00001605168154B01F0F00109095C5C0168F8
:1089F000E1404160546804F4E064240A1C5D21FAFB
:108A000004F48460546804F46054E40A1B5DD940A3
:108A1000C1605268094B02F44042920B1B1F9A5CE2
:108A2000B1FBF2F1016110BD0010024000127A00AA
:108A300040787D0120BCBE0000093D008A5003083B
:108A40000246002053090949012B0BD0022B0BD001
:108A5000D1F8241002F01F02012393400B4200D0F2
:108A6000012070470968F5E7096AF3E70010024042
:108A7000034A516821F0F001014351607047000042
:108A8000001002400B490A6822F480320A600A682A
:108A900022F480220A60B0F5803F07D0B0F5802F25
:108AA00003D1086840F4A02008607047086840F4CB
:108AB0008030F9E7001002407047000006490022AC
:108AC0000A7001F82029012802D0042802D10520CB
:108AD00081F820007047000020100240034A5168CE
:108AE00021F4E06101435160704700000010024032
:108AF00003494A6822F4605242EAC0004860704765
:108B00000010024001490866704700000000424220
:108B1000034A5368084323F47C131843506070479A
:108B20000010024001490860704700003C044242C6
:108B300002490A6A02430A627047000000100240BC
:108B4000034A516821F0030101435160704700005E
:108B50000010024030B50B4C40F2FF153120FFF7FA
:108B60006FFF20706068401C6060207810B96068FA
:108B7000A842F3D13120FFF763FF002800D0012085
:108B800030BD0000FC0300207047000002490A8845
:108B900082430A80704700000428004010B54FF45B
:108BA0007A7400BF01214FF0C050FFF789FE012009
:108BB000FEF700FB0120FFF781FF2848046042F226
:108BC0001070844201DA04F5FA7400BF4120FFF707
:108BD00037FF18B9214800680028F7D14120FFF776
:108BE0002FFFE8B90020FFF769FF0020FEF7E2FA47
:108BF00000214FF0C050FFF763FE4FF4806118482A
:108C0000FDF71BFB4FF4FA701449086000BF1348CE
:108C100000680028FBD14FF480611148FDF70BFB81
:108C20004120FFF70DFF0028BCD04FF48070FFF704
:108C30007FFF0120FFF776FF00F0D4F800F0CAF8BC
:108C40000121084600F04AF800F0C4F847F6FF702A
:108C500000F0B0F800F0BEF810BD000018000020D1
:108C6000000C01400248018841F01001018070476A
:108C7000042800400248018821F01001018070475B
:108C800004280040034800880249091F098840EA77
:108C9000014070471C28004006490988054A0140E8
:108CA000121FC9B21288024202D009B101207047D6
:108CB000002070470428004010B50120FFF7ECFFAA
:108CC00048B100F087F80120FFF760FF0248006814
:108CD000401C0149086010BD04000020044A00291E
:108CE000118801D0014300E08143118070470000EA
:108CF0000028004010B501214FF0C050FFF7E0FD03
:108D00000120FEF757FA0420F8F742FD4AF2A55178
:108D100088422FD0FFF742FF00F05CF84AF6C0000F
:108D200000F038F800F056F84AF2A5510420F8F7A0
:108D300035FD00210820F8F731FD00210C20F8F75F
:108D40002DFD00211020F8F729FD00211420F8F74F
:108D500025FD00211820F8F721FD00211C20F8F73F
:108D60001DFD00212020F8F719FD00212420F8F72F
:108D700015FD0DE04120FFF763FE08B9FFF70EFF78
:108D800000F030F801210846FFF7A8FF00F022F8B4
:108D900010BD000000B50246FFF764FF0449100C47
:108DA0000880081D02805DF804EBFFF763BF000038
:108DB0001828004000B50246FFF754FF0449C2F3EB
:108DC00003400880081D02805DF804EBFFF752BFE6
:108DD00008280040024801888906FCD57047000039
:108DE000042800400448018821F00801018001881E
:108DF0000907FCD5704700000428004010B5044660
:108E0000204600F0CBF810BD70B540F29310FFF78C
:108E1000F5FF0546002D01DB322D00DB0025681E25
:108E2000051E00DA31252C46022218480168184830
:108E30000068FAF733F800BF04F5CA70FFF7DEFFE9
:108E4000064601F009F82C2000F0AEFF04F5E370AF
:108E5000FFF7D4FF064600F0FFFF2C2000F0A4FF30
:108E600004F5FC70FFF7CAFF064600F0F5FF641E2C
:108E7000002C00DA3124AC4202D02C2000F094FF08
:108E8000AC42D9D1FAF72AF870BD000010010020D9
:108E90001401002070B520480078D0B100BFFDF764
:108EA00071FF0446FAF7FAF8FDF76CFF0546FAF78A
:108EB000F5F8FDF767FF0646FAF7F0F8AC42EED199
:108EC000B442ECD10CB1002070BD002012490870F2
:108ED000FAE700BFFDF756FF04460CB90020F3E7A0
:108EE000FAF7DCF8FDF74EFF0546FAF7D7F8FDF77D
:108EF00049FF0646FAF7D2F8AC42EBD1B442E9D1C9
:108F00000548047034B14FF416700449086001201C
:108F1000034908602046D7E7BC0000206C0300200E
:108F20001803002070B504460D464FF480411848E0
:108F3000FDF783F924B980211648FDF77CF903E099
:108F400080211448FDF779F925B140211248FDF739
:108F500074F904E04FF400410D48FDF76EF920214B
:108F60000B48FDF76AF90B48FDF754F90646360A37
:108F700020210748FDF75FF940210748FDF75BF91D
:108F80004FF400410248FDF756F9304670BD00002D
:108F9000000C014000180140000801402DE9F04795
:108FA00006460027B500C5F30749ADB24FF00308E8
:108FB00000BF00242946484605F000FCF0B105F04A
:108FC000CFFAA12101EB4901C8B205F079FC0746AF
:108FD000A7B105F061F8044605F086F805F05CF8E5
:108FE00000EB042405F080F805F056F800EB0424AB
:108FF00005F07AF805F050F800EB042405F0C0FA0B
:1090000027B9A8F1010000F0FF0801E04FF00008C7
:10901000B8F1000FCDDC2046BDE8F08710B5184848
:10902000006820B1012807D0022817D109E01448B0
:10903000006804F0C9FC15E01148006804F0C4FCA5
:1090400010E010490E4A126831F81200FDF76FFA6D
:109050000D490B4A126841F8220003E0002008493C
:10906000086000BF00BF06480068401C0449086053
:1090700008460068022801DD0020086010BD0000DD
:10908000D4000020800D0020F40B0020F0B5024633
:109090000B4600240FE0174901EB021516490E6834
:1090A0000968491C144F3960A85DF8F767FB04EBA9
:1090B000840100EB41040F4800EB02100E490968DF
:1090C000405C984213D00B4800EB02100A49096833
:1090D000405C30280BDB074800EB021006490968AA
:1090E000405C392803DC044800681328D3DB2046A1
:1090F000F0BD0000402000202401002070B505468E
:109100000E46002404E0FF2000F09EFF2855641C5A
:10911000B442F8D3012070BD10B580210148FDF79D
:109120008AF810BD0014014010B580210148FDF7F8
:1091300084F810BD0014014010B580210348FDF7EC
:109140007CF880210148FDF776F810BD0010014041
:1091500010B510210148FDF76EF810BD0014014054
:1091600010B510210148FDF768F810BD001401404A
:1091700010B54FF400610248FDF75DF810BD000026
:10918000000C014010B54FF400610248FDF755F89E
:1091900010BD0000000C014010B540210148FDF752
:1091A0004AF810BD0010014010B540210148FDF7FC
:1091B00044F810BD0010014010B54FF48071024812
:1091C000FDF739F810BD00000010014010B54FF454
:1091D00080710248FDF731F810BD00000010014019
:1091E00010B54FF400610248FDF725F810BD0000EE
:1091F0000014014010B54FF400610248FDF71DF85E
:1092000010BD00000014014010B54FF40071024879
:10921000FDF711F810BD00000010014010B54FF42B
:1092200000710248FDF709F810BD00000010014070
:1092300010B54FF480610248FCF7FDFF10BD00003F
:109240000014014010B54FF480610248FCF7F5FFAF
:1092500010BD00000014014010B54FF40061024839
:10926000FCF7E9FF10BD00000008014010B54FF405
:1092700000610248FCF7E1FF10BD0000000801405A
:1092800010B54FF400510248FCF7D5FF10BD0000A7
:10929000000C014010B54FF400510248FCF7CDFF1F
:1092A00010BD0000000C014010B54FF48051024881
:1092B000FCF7C1FF10BD00000008014010B54FF4DD
:1092C00080510248FCF7B9FF10BD000000080140C2
:1092D00010B54FF480510248FCF7ADFF10BD0000FF
:1092E000000C014010B54FF480510248FCF7A5FF77
:1092F00010BD0000000C0140F0B507460C461646B4
:10930000B44201D12046F0BDA01900EBD0714D1040
:1093100005EB4500084901EB80004068B84205DDD7
:109320003246691C3846FFF7E7FFECE72A4621463C
:109330003846FFF7E1FFE6E7080E020870B502467F
:109340000020002317E000EB4004304D55F8244086
:10935000944206D100EB400405EB840464688C421F
:1093600006D000EB4004294D05EB8404A4680CB939
:10937000012300E0401C192801DA002BE3D0E3B3FD
:1093800000EB4004214D05EB8404A468022C3BD182
:1093900023E0441C04EB44041C4D55F8244000EB2E
:1093A00040051A4E46F82540441C04EB440435465B
:1093B00005EB8404646800EB400506EB85056C60F2
:1093C000441C04EB4404354605EB8404A46800EB1C
:1093D000400506EB8505AC60401C1828D9DB00244D
:1093E00000EB4005094E46F8254000EB400506EB32
:1093F00085056C6000EB400500E005E006EB8505A7
:10940000AC600124024D2C7070BD0000540C002093
:109410006F010020002010E0002100EB4002084B0B
:1094200003EB8202916000EB400243F8221000EB54
:10943000400203EB82025160401C1928ECDB7047AC
:10944000540C00200021074A1170002004E0002184
:10945000054A1154411CC8B20828F8DB0021034A10
:10946000117070476D010020710100207001002013
:10947000002014E0002100EB40020A4B43F82210C8
:1094800000EB400203EB8202516000EB400203EB71
:1094900082029160044A1160044A1160401C142841
:1094A000E8DB7047280E0020DC000020E0000020F0
:1094B00070B50E480068FCF753FC04460B48006882
:1094C000FCF730FC054601222946204601F064FEE7
:1094D00006490968491C054A08461160FDF7F6FB74
:1094E00010B100200149086070BD0000200000207C
:1094F00070B539A13948F7F726F8394908600846A8
:109500000068002867D04FF480613648FCF795FE6C
:1095100001203549087000F0DDFF032204210846D0
:1095200000F0F4FF05220621042000F0EFFF2AE0FE
:10953000002400252D48005D2A2822D008E02B4871
:10954000005D05EB850100EB4100A0F13005641CD6
:109550002648005D3D28F2D1641C002608E023481F
:10956000005D06EB860100EB4100A0F13006641CB3
:109570001E48005D0A28F2D100223146284601F03B
:109580000BFEFCF7FFFF16481E2102681748F6F78E
:1095900065FF0028CCD1FCF7F5FF11480068F6F70D
:1095A000F9FFFCF7EFFF12490C4803F0ADFBFCF7A5
:1095B000E9FF41F288300F49086001E0FCF7E2FF63
:1095C0000C4800680028F9D107490870FDF77EFCB7
:1095D00001200949087070BD720000005C5003084A
:1095E000F0030020000C014008010020144C002072
:1095F00071500308180000206F01002070B5E5E0ED
:1096000000F0ACFB044674480078062870D2DFE80E
:1096100000F00314384C70B3012C0DD1C8206F49F1
:10962000086001206C49087000206D4908606D4990
:109630000860204600F0DEFBC7E0204600F0DAFBC1
:109640002C2C16D101266520FFF7D8FB064665486D
:109650000068B04202D06348006818B902205E4931
:10966000087002E000205C49087000205E49086034
:1096700006E021465B480068F8F76AF85949086037
:10968000A3E0204600F0B6FB2C2C06D10320524963
:10969000087000205549086006E0214652480068DD
:1096A000F8F756F8504908608FE0204600F0A2FB1A
:1096B000022C15D104204849087000204C4908604C
:1096C0004C490860002508E000214B48484A1268D0
:1096D00000EB02104155681CC5B2102DF4DB06E00A
:1096E000214642480068F8F733F8404908606CE0CA
:1096F00067E0204600F07EFB032C06D105203649AA
:10970000087000203D49086035E02C2C20D13848F5
:109710000068401C3649086008460068642803DB7E
:1097200008460068401E0860002032490860002595
:1097300008E0002030492E4A126801EB021148551A
:10974000681CC5B2102DF4DBC8202449086012E063
:1097500029482749096800EB011026490968445443
:1097600024480068401C2349086008460068122805
:1097700001DD1220086028E0042C13D11F48006886
:1097800017490968884209D14FF416701C490860CE
:1097900000F038F800201049087011E000200E4950
:1097A00008700DE015480068000114490860204663
:1097B000F8F766FF1149098889B208430F49086024
:1097C00003E000200449087000BF00BF00F0DEFA8B
:1097D00000287FF415AF70BD3B0100202C01002054
:1097E0003001002010010020140100201801002089
:1097F0001C01002020010020402000203401002016
:10980000280100202DE9F047FC4800680E2878D098
:1098100009DC0C2849D2DFE800F048174849788B6A
:10982000CC484848FEFD65286CD006DC0F286AD07D
:10983000102869D0642838D1B2E1662876D067282C
:1098400075D06828F7D129E20222ED480168ED4879
:109850000068F9F723FB002400BF0020EA490860F4
:1098600000212046FFF712FC80464046FCF79EFA96
:10987000002806DB4046FCF75DFD054600F0ECFAEB
:1098800005E02D2000F090FA312000F08DFADF483D
:109890000068844202DA2C2000F086FA641CDB485F
:1098A00000688442D9DDF9F719FB16E20222D44898
:1098B0000168D4480068F9F7F1FAD5480078D5492D
:1098C0000978884206D12D2000F06EFA312000F090
:1098D0006BFA13E0CF4805780CE0681CC5B2142D74
:1098E00000DB0025CC4951F8250000F0B5FA2C200A
:1098F00000F05AFAC6480078A842EED1F9F7EEFA1D
:10990000EBE109E196E134E146E1C1480078C14963
:1099100008700222BA480168BA480068F9F7BEFA2E
:10992000302000F041FAF9F7D9FAD6E192E195E159
:1099300000250222B2480168B2480068F9F7AEFA81
:10994000B648007830B92D2000F02EFA312000F012
:109950002BFA1BE016E0B24951F8350000F07CFA12
:109960002C2000F021FAAE4901EBC501486800F057
:1099700073FA681CC5B2A9480078854202DA2C2027
:1099800000F012FAA54800788542E4DBF9F7A6FA60
:10999000002508E00020A24941F8350001EBC5018F
:1099A0004860681CC5B2782DF4DB00209B49087024
:1099B00093E1002502229248016892480068F9F775
:1099C0006DFA9848007830B92D2000F0EDF931207B
:1099D00000F0EAF91BE016E0934951F8350000F079
:1099E0003BFA2C2000F0E0F98F4901EBC5014868F3
:1099F00000F032FA681CC5B28A480078854202DA63
:109A00002C2000F0D1F9874800788542E4DBF9F793
:109A100065FA01E07FE010E0002508E000208249BF
:109A200041F8350001EBC5014860681CC5B2782DCE
:109A3000F4DB00207B4908704FE10024A1467B48FD
:109A40000078002854D100BF002600206E4908602D
:109A50003D212046FFF71AFB80466B480068401CFA
:109A6000694908604046FCF7A1F9002839DB404607
:109A7000FCF79CF940B900212046FFF707FB06469A
:109A8000304600F097FB2EE04046FCF78FF91B288C
:109A900029D000212046FFF7F9FA06464046FCF798
:109AA00085F90546FDF7F8F8E8B14046FCF77EF980
:109AB0000546FCF74BF9B04202DD49F0020912E01D
:109AC0004046FCF773F90546FCF736F9B04202DA76
:109AD00049F0040907E000223146404601F05CFBF2
:109AE00001E049F00109641C484800688442ABDD8C
:109AF0004348006870B11422414801684148006839
:109B0000F9F7CCF94949097809EBC10000F0A4F94B
:109B1000F9F7E4F9E1E0E0E00024002717E0002095
:109B20003949086000212046FFF7B0FA404941F862
:109B30003700641C00203449086000212046FFF7EC
:109B4000A5FA3B4901EBC7014860641C7F1C2F4804
:109B500000688442E3DB09E00020354941F8370022
:109B6000002238467F1C01EBC0004260192FF3DB56
:109B7000B3E000202449086000210846FFF786FA78
:109B800080464046FCF7D6FB012804D10122022181
:109B9000404601F001FBA0E000201B4908609CE06A
:109BA00000201949086000210846FFF76FFA804637
:109BB00000201549086000210120FFF767FA0646DA
:109BC000FA2E00DDFA2602220D4801680D480068D1
:109BD000F9F764F9C24600250AE01AF8010B00F013
:109BE0003BF9701EA84202DD2C2000F0DDF86D1C50
:109BF000B542F2DBF9F772F96FE0000018010020BE
:109C00001001002014010020240100201C0100206C
:109C10002500002024000020240400203901002019
:109C2000740400203A010020340800203C01002088
:109C3000680F002000202A49086000210846FFF72D
:109C400025FA284908600846006810B10120264915
:109C5000087042E00020244908703EE000202049BE
:109C6000086000210846FFF711FA18B1A0F2E730AA
:109C700090B902E0FFF7C8F80EE0F7F7AFFE022256
:109C80001A4801681A480068F9F708F9002000F03E
:109C9000E3F8F9F723F900BF00BF1EE002221348E2
:109CA000016813480068F9F7F9F8122000F0D4F8B9
:109CB0002C2000F079F86420FFF7A0F8054600F0AA
:109CC000CBF82C2000F070F86520FFF797F80546D8
:109CD00000F0C2F8F9F702F900BF00BFBDE8F08755
:109CE00024010020040100200801002010010020B0
:109CF0001401002010B500201149086011490860C6
:109D00001149086011490860114908704FF4164064
:109D10001049086000208880C880088188810C2054
:109D200048810D4801F040F8012240F225510A48CF
:109D300001F021F80121084800F0F4FF10BD0000F7
:109D400044010020400100204C0100204801002077
:109D50003B010020301000200044004000BF0848B4
:109D60000068084A12689042F9D005480068401C13
:109D7000C0F30A01024801600348405C70470000DC
:109D800044010020400100204010002004480068E9
:109D900004490968884201D0012070470020FCE78F
:109DA000400100204401002070B505460D480068C0
:109DB000401CC0F30A0400BF0B4800688442FBD07B
:109DC0000A48055507480460284600F013F80122A8
:109DD00040F22771064800F0CEFF0121044800F050
:109DE000A1FF70BD480100204C0100204018002058
:109DF0000044004007490988C1F307214140064A51
:109E000032F82110034A127881EA022189B2014A0C
:109E10001160704730010020EC17020810B50446AD
:109E200004F13000C4B2392C01DDE01DC4B220467B
:109E3000FFF7BAFF10BD000010B50446002C02DD8C
:109E40000120044908700348007810B12046FFF74C
:109E5000E5FF10BD3801002070B5044600203E49E2
:109E60000870002C00DA00243C4894FBF0F00A2132
:109E700090FBF1F201FB1200C5B22846FFF7DCFFB0
:109E8000374894FBF0F00A2190FBF1F201FB12003D
:109E9000C5B22846FFF7D0FF324894FBF0F00A2104
:109EA00090FBF1F201FB1200C5B22846FFF7C4FF98
:109EB0002D4894FBF0F00A2190FBF1F201FB120017
:109EC000C5B22846FFF7B8FF284894FBF0F00A21F6
:109ED00090FBF1F201FB1200C5B22846FFF7ACFF80
:109EE00042F2107094FBF0F00A2190FBF1F201FBBA
:109EF0001200C5B22846FFF79FFF4FF47A7094FB1B
:109F0000F0F00A2190FBF1F201FB1200C5B22846E5
:109F1000FFF792FF642094FBF0F00A2190FBF1F22E
:109F200001FB1200C5B22846FFF786FF0A2094FB0A
:109F3000F0F00A2190FBF1F201FB1200C5B22846B5
:109F4000FFF77AFF0A2094FBF0F100FB1140C5B245
:109F50002846FFF763FF70BD3801002000CA9A3B16
:109F600000E1F5058096980040420F00A0860100B0
:109F700010B50446C4F30330FFF750FFC4F30320C9
:109F8000FFF74CFFC4F30310FFF748FF04F00F0086
:109F9000FFF744FF10BD000010B540210248FCF758
:109FA0004CF902F087F910BD000C014010B54021BA
:109FB0000248FCF740F902F07DF910BD000C0140A9
:109FC00010B580210748FCF738F980200649088041
:109FD000032088700420C8700248FCF7A9F802F03A
:109FE00069F910BD000C01405C01002010B5802013
:109FF00007490880032088701420C8700548FCF7C2
:10A0000097F880210348FCF716F902F053F910BDC8
:10A010005C010020000C014070477047704770479A
:10A02000704710B50446204600F00EF810BD70B51C
:10A0300005460E46002403E0285D00F005F8641C88
:10A04000B442F9D3012070BD2DE9F04105462E46FA
:10A050000024002725E006F0800028B94FF4805145
:10A060001248FCF7E8F804E04FF480510F48FCF781
:10A07000E4F87006060E4FF480610C48FCF7DDF83A
:10A080006006040E4FF400610848FCF7C6F808B1FA
:10A0900044F001044FF480610448FCF7CCF8781CCC
:10A0A000C7B2082FD7DB2046BDE8F0810010014081
:10A0B000014609B1102001E04FF48010014A106000
:10A0C000012070471008014070B5024600200023AF
:10A0D00017E000EB40042F4D55F82440944206D180
:10A0E00000EB400405EB840464688C4206D000EB6E
:10A0F0004004284D05EB8404A4680CB9012300E05A
:10A10000401C192801DA002BE3D00BB300EB40040C
:10A11000204D05EB8404A468022C1AD11E4C24683F
:10A12000B4B900EB400445F8242000EB400405EBF3
:10A1300084046160012400EB4005164E06EB8505A2
:10A14000AC60164C2468112C22D10124144D2C70C3
:10A150001EE000EB40040F4D05EB8404A468012CC5
:10A1600016D000EB400445F8242000EB400405EB3A
:10A1700084046160012400EB4005064E06EB850572
:10A18000AC60064C2468112C02D10124044D2C70C3
:10A1900070BD0000540C0020B80000200003002017
:10A1A0006F010020421E024B43F82210704700004E
:10A1B0002C0C002010B50446FEF7F0FCFEF70AFE5A
:10A1C000C4EB04118800FEF7E5FDFEF703FE4AF23A
:10A1D000A5510420F7F7E2FAFEF754FD3C21B0FB4D
:10A1E000F1F00149086010BD3000002070B5044650
:10A1F0000D4600F03AFF04F03F0000F14002A111CB
:10A20000002001F027F800F030FF05F1B802A1119D
:10A21000002001F01FF800F028FFC02200210846AE
:10A2200001F018F8C0220121002001F013F870BDE0
:10A23000421E024B43F8221070470000400F0020DE
:10A240002DE9F04104460F462046FCF7CFF80646BC
:10A250002046FCF75FF900F16C053146284600F016
:10A2600087FFBDE8F0810000421E024B43F8221038
:10A2700070470000180F00202DE9F04107460C46FA
:10A280003846FCF7A8F806463846FCF729F880B9A6
:10A2900014B93846FEF7CCFA00213846FCF776F8B8
:10A2A00004FB1605B54200DA354629463846FFF765
:10A2B00079FFBDE8F08110B5044600212046FFF784
:10A2C00071FF10BD2DE9F05F83460C465846FCF740
:10A2D00082F807466B20FEF791FD82465846FCF750
:10A2E000C3F881461948006848452DDB5846FBF7FE
:10A2F000F7FF48BB00215846FCF755F8804600217F
:10A300005846FCF743F8054609EB0A000F4909686F
:10A31000884202DC04FB17860BE00C480068A0EBC7
:10A320000900A8EB0501484390FBFAF0284404FB20
:10A330001706BE4200DA3E4614B95846FEF778FAD0
:10A3400031465846FFF72EFFBDE8F09F3800002049
:10A350002DE9F35F0C460098FCF73DF807466B20AB
:10A36000FEF74CFD82460098F7F7C2FC8346009842
:10A37000FCF77AF881460BF1010088B319480068B0
:10A3800048452DDB0098FBF7ABFF48BB59460098CA
:10A39000FCF709F8804659460098FBF7F7FF064698
:10A3A00009EB0A000F490968884202DC04FB1785A3
:10A3B0000BE00C480068A0EB0900A8EB060148433D
:10A3C00090FBFAF0304404FB1705BD4200DA3D462D
:10A3D00014B90098FEF72CFA29460098FFF7E2FE20
:10A3E000BDE8FC9F380000202DE9F04180460C4676
:10A3F0004046FBF7F0FF06464046F7F779FC074674
:10A40000781CA0B14046FBF76BFF80B914B94046F9
:10A41000FEF70EFA39464046FBF7B8FF04FB160577
:10A42000B54200DA354629464046FFF7BBFEBDE897
:10A43000F081000070B50025202600216C20FCF77B
:10A4400081F82148006800283DD14FF496701E49DC
:10A45000086000241CE004EB44001C4901EB800070
:10A46000406898B104EB440001EB8000806802284A
:10A4700002D1012D00DA012504EB4400134901EB60
:10A4800080008068012802D1022500E01924641CA4
:10A49000192CE0DB012D02D0022D0ED101E0962611
:10A4A0000BE00B48007820B9962601200849087077
:10A4B00002E000200649087000BF00BF01223146BB
:10A4C0001046FEF7ADF870BDF8020020540C0020D5
:10A4D0003203002010B5FCF7F9FCFCF73BFD00202F
:10A4E0000449087004490870012204A1104600F0D4
:10A4F000A3FF10BD6501002066010020202020443C
:10A5000052414D4D202020200000000070B504462F
:10A510000D46164605490D7005490C7006F1B0014F
:10A520000022104600F034FF70BD000066010020DC
:10A53000650100202DE9F0412048006800283BD14A
:10A540004FF4AF701D4908601D48007818B901200C
:10A550001B49087002E00020194908704FF4BD70D3
:10A56000FEF74CFC0446012C01DA3C2604E03C20BA
:10A5700090FBF4F0801EC6B200251BE0284600F0D8
:10A5800039FD20B10E48007808B9E32700E0DF2745
:10A59000C5EB0510C00090FBF4F000EB06080721A6
:10A5A0004046FBF7CFFF002239461046FEF738F849
:10A5B000681CC5B2A542E1DBBDE8F081680100205E
:10A5C0003403002070B5FCF7C5FC00204249087038
:10A5D00042490870012242A1104600F02DFF1020D0
:10A5E0003D49087004203D490870002240A11046F2
:10A5F00000F022FF062039490870222036490870F1
:10A600006420FEF7FBFB0446002256211046FEF7AD
:10A6100007F83B4894FBF0F03030C5B200222946E1
:10A620001046FDF7FDFF42F2107094FBF0F00A2196
:10A6300090FBF1F201FB12003030C5B20022294636
:10A640001046FDF7EDFF00222E211046FDF7E8FF32
:10A650004FF47A7094FBF0F00A2190FBF1F201FBC9
:10A6600012003030C5B2002229461046FDF7D8FF4F
:10A67000642094FBF0F00A2190FBF1F201FB120040
:10A680003030C5B2002229461046FDF7C9FF00222E
:10A690002E211046FDF7C4FF0A2094FBF0F00A219A
:10A6A00090FBF1F201FB12003030C5B200222946C6
:10A6B0001046FDF7B5FF0A2094FBF0F100FB1140B6
:10A6C0003030C5B2002229461046FDF7A9FF42F2FC
:10A6D00010700C49086070BD650100206601002003
:10A6E0002020204452414D4D202020200000000019
:10A6F0002020204D6973742D54696D652020200041
:10A70000A08601001400002070B5044600256720D3
:10A71000FEF774FB06283FD2DFE800F0030C16209A
:10A720002A3404EB44011E4A52F83100F5F758FF71
:10A73000054631E004EB4401194A02EBC1014868C7
:10A74000F5F74EFF054627E004EB4401144A02EBFF
:10A75000C1018868F5F744FF05461DE004EB44019C
:10A760000F4A02EBC101C868F5F73AFF054613E04E
:10A7700004EB44010A4A02EBC1010869F5F730FF16
:10A78000054609E004EB4401054A02EBC1014869B2
:10A79000F5F726FF054600BF00BF284670BD000044
:10A7A0006C49020810B500F047F810BD4FF0E021E9
:10A7B000012804D0801C06D00020886170470869F9
:10A7C00040F0010002E0086920F0010008617047D4
:10A7D0004FF0E0210028086902D040F0020001E0BB
:10A7E00020F002000861704710B541F66A0000F0E1
:10A7F0000DF80120FFF7ECFF0120FFF7D7FF142031
:10A800000149086010BD0000140000204FF0E02155
:10A810004861704700B506480068064909688842E3
:10A8200004D1FCF79BFC08B1012000BD0020FCE72F
:10A83000DC000020E000002010B54E48006820B188
:10A840004C480068401E4B4908604B48006828B1DE
:10A8500049480068401E4849086003E04FF47A7098
:10A86000454908604548007870B143480068C821F0
:10A8700090FBF1F201FB1200642805DD4FF48071BA
:10A880003F48FBF7DAFC04E04FF480713C48FBF7EB
:10A89000D2FC3C48006820B13A480068401E394963
:10A8A00008603948006820B137480068401E3649C2
:10A8B00008603648006820B134480068401E3349BB
:10A8C00008603348006820B131480068401E3049B4
:10A8D00008603048006820B12E480068401E2D49AD
:10A8E00008602D48007820B12B480078401E2A4986
:10A8F00008702A48007820B128480078401E27496F
:10A9000008702748007820B125480078401E244967
:10A9100008702448007820B122480078401E214960
:10A9200008702148006828B11F480068401E1E4971
:10A93000086002E000201D4908701D48006828B129
:10A940001B480068401E1A49086002E000201949AF
:10A9500008701948006820B117480068401E164961
:10A9600008601648006820B114480068401E13496A
:10A97000086010BD500100201400002008010020D4
:10A980000008014018000020E0030020E803002038
:10A99000EC030020E4030020000000200100002060
:10A9A00002000020030000202C0100203B010020B9
:10A9B000D40300209603002068010020F802002044
:10A9C00070477047704770477047704770477047CF
:10A9D0007047704770477047704770477047000076
:10A9E0002DE9F0477148007808B1FCF789FE002096
:10A9F0006E49087000212820FBF7A4FD01230022E6
:10AA00006B4801681846FDF7B3FA4FF4C170FEF7C2
:10AA1000F5F940B302210320FBF794FD00221F212A
:10AA2000104600F0B5FC63480068FBF754F9814616
:10AA300000231A4649461846FDF7CAFB40F27B1030
:10AA4000FEF7DCF928B900221146104600F0A0FC00
:10AA500004E000221021104600F09AFC0022202180
:10AA60001046FDF7DDFD032631460320FBF76AFDA6
:10AA70005148006818B95148006800283DD04E4838
:10AA80000068C0B10022B621104600F081FC4C489D
:10AA90000078801E4A49087047480068FAF777FA3C
:10AAA000002220211046FDF7BBFD46480068FAF75A
:10AAB0003FFAFBF729F94148006840B3761C31465C
:10AAC0000320FBF73FFD0022B621104600F060FC9A
:10AAD0003B480078801E3A49087038480068FAF709
:10AAE00056FA002220211046FDF79AFD36480068EC
:10AAF000FAF71EFAFBF708F911E03448006838B19C
:10AB00000022BD21104600F043FCFBF7FDF806E0F3
:10AB10000022BE21104600F03BFCFBF7F5F8032EA7
:10AB200005D104210320FBF70DFDFBF7EDF84FF4F1
:10AB3000BD70FEF763F90446092C01DD092700E02A
:10AB4000E7B2012C02DA4FF03C0805E03C2090FB14
:10AB5000F4F0401E00F0FF08002513E0C5EB0510DF
:10AB6000C00090FBF4F000EB080906214846FBF713
:10AB7000E9FC05F13100C1B200221046FDF750FD9D
:10AB8000681CC5B2BD42E9DB0A2C0DD106216E203E
:10AB9000FBF7D8FC002231211046FDF741FD0022D1
:10ABA00030211046FDF73CFDBDE8F0876F01002025
:10ABB00030000020380000203C0000204800002029
:10ABC00065010020400000204C000020A000002073
:10ABD000704770477047000070B540F227711E48FB
:10ABE00000F0AAF8C8B11D4800681D4909688842EC
:10ABF0000CD01B480068401CC0F30A041948015DD2
:10AC0000154800F01BF91648046005E0002240F2E8
:10AC10002771114800F0AFF800BF40F225510E48EF
:10AC200000F08AF8B8B10C4800F004F9C5B20E483B
:10AC30000068401CC0F30A040B4804600B4800681D
:10AC4000844202D101200A4908700A48055564204F
:10AC50000949086000BF70BD004400404801002061
:10AC60004C01002040180020400100204401002039
:10AC70003C010020401000202C01002070B540F263
:10AC800027711F4800F058F8C8B11E4800681E49D7
:10AC9000096888420CD01C480068401C00F01F0462
:10ACA0001A48015D164800F0C9F81748046005E02D
:10ACB000002240F22771124800F05DF800BF40F218
:10ACC00025510F4800F038F8C0B10D4800F0B2F837
:10ACD000C5B20F480068401CC0F308040C4804606B
:10ACE0000C480068844202D101200B4908700B48CF
:10ACF00005554FF47A700A49086000BF70BD000026
:10AD0000004800408C03002090030020CC3100203C
:10AD1000840300208803002097030020CC2F00200C
:10AD2000D40300200029818902D041F4005101E0C0
:10AD300021F400518181704770B501F01F06012296
:10AD40000025C1F3421302FA06F4012B0FD0022BA7
:10AD50000FD0838A4FEA11210088234202FA01F2C0
:10AD600000EA020001D000B10125284670BD8389A8
:10AD7000F0E7038AEEE710B5C1F3421301F01F04B8
:10AD80000121A140012B07D0022B07D01430002A4B
:10AD9000026805D00A4304E00C30F8E71030F6E70B
:10ADA0008A43026010BD000030B50446008A85B0B9
:10ADB0000D464CF6FF710840E98801432182A189C4
:10ADC0004EF6F3100140A8882A8910436A890A4385
:10ADD0001043A081A08A4FF6FF410840A989014392
:10ADE000A1826846FDF7DAFD1148844201D103983B
:10ADF00000E00298642200EBC00101EB001029681A
:10AE00006FF018058900B0FBF1F0B0FBF2F1090119
:10AE10000B096B4300EB8300322303EB0010B0FB04
:10AE2000F2F000F00F000843208105B030BD0000B3
:10AE3000003801408088C0F308007047C1F3080162
:10AE4000818070477047704770470120704700004D
:10AE50002D2802D08D2842D12EE0224909680429EC
:10AE600014DA20490968491C1E4A11601E49096804
:10AE7000126811441D4A02EB01110968491CD1B93D
:10AE800018490968491E174A116014E016490968F3
:10AE9000491C154A116011460968124A126811448A
:10AEA000124A02EB01110968491C21B90E490968CF
:10AEB000491E0D4A116012E00A49096829B1094981
:10AEC0000968491E074A116008E007490968002916
:10AED00004DD05490968491E034A116000BF00BF2F
:10AEE0007047000060010020EC0200209C2C002034
:10AEF0004FF6FF72904216D042F21072904212DB6F
:10AF0000520090420FDA084A1278521CD1B214292A
:10AF100000DB0021054A1278914204D0044A42F82D
:10AF20002100014A117070472500002024000020F4
:10AF30002404002000BFFEE770B502460020002375
:10AF400017E000EB4004174D55F82440944206D119
:10AF500000EB400405EB840464688C4206D000EBEF
:10AF60004004104D05EB8404A4680CB9012300E0F3
:10AF7000401C192801DA002BE3D093B100EB400408
:10AF8000084D05EB8404A468012C0AD1022400EBCF
:10AF90004005044E06EB8505AC604FF49674024DF7
:10AFA0002C6070BD540C0020B800002010B50D4A74
:10AFB00012680D4B1B681A4402EB42020B4B03EB69
:10AFC00082025168074A1268074B1B681A4402EB59
:10AFD0004202064B53F82200FFF7AEFF012004495E
:10AFE000087010BD4C03002060010020540C0020AC
:10AFF0006F010020014607480268481C824204D0C5
:10B0000005480268481C824201D101207047002097
:10B01000FCE700003C0000204800002001460B290E
:10B0200020D2DFE801F006080A0C0E1012141619DF
:10B030001C00002070470220FCE70420FAE70820EB
:10B04000F8E71020F6E72020F4E74020F2E7802020
:10B05000F0E74FF48070EDE74FF40070EAE74FF44B
:10B060008060E7E70020E5E7704770B500BF00218A
:10B070000846FDF757FFC5B201210020FDF752FF3A
:10B08000C4B2802D02D00DB1FBF764FF802C02D03A
:10B090000CB1FBF75FFF05F080000028E7D104F05A
:10B0A00080000028E3D170BD10B515E0FBF76AFA07
:10B0B0000D480068C82190FBF1F201FB12006428E2
:10B0C00005DA4FF480610948FBF7B7F804E04FF464
:10B0D00080610648FBF7AFF80348006818B1FDF738
:10B0E000D9FE0028E2D010BD14000020000C014061
:10B0F0002DE9F04107460D4690461C46069E01206C
:10B100001A490870E2B220210020FDF789FA0420D4
:10B1100016490870E2B220210020FDF781FA012DC6
:10B1200002D0022D0CD105E0E2B2BF21002000F0D8
:10B130002FF905E0E2B2C021002000F029F900BF9C
:10B1400000BF04E0E2B220210020FDF769FA0748C1
:10B1500000787828F6DB772004490870E2B22021D5
:10B160000020FDF75DFABDE8F081000065010020D8
:10B1700070B505460C462846FDF740FEA04209D0B2
:10B180002946204600F0C0F82846FAF7F3FD0646A7
:10B19000FFF7AEFE70BD00002DE9F04105460C46FC
:10B1A00016461548854225DA2846FAF7FFFD074678
:10B1B000FBF766FDA0B12846FBF7A6F80746FDF7AA
:10B1C0001DFEA04216D02846FBF79EF807463946DA
:10B1D000204600F099F86EB12846FFF789FE09E095
:10B1E0002846FAF7E3FDC0EBC000044901EB8000FC
:10B1F00040680460BDE8F08178D403005CEB01088E
:10B200002DE9F04105460F46164640F29310FDF732
:10B21000F5FD0446002C01DB322C00DD002404F592
:10B22000CA702946FFF7A4FF04F5E3703946FFF71B
:10B230009FFF04F5FC703146FFF79AFF641C322C27
:10B2400000DB0024214640F29310FFF791FFBDE898
:10B25000F0810000F8B505460E4617464FF48041D0
:10B260002648FAF7E8FF25B980212548FAF7E3FFD9
:10B2700003E080212248FAF7E0FF26B1402121486F
:10B28000FAF7DBFF04E04FF400411C48FAF7D5FF62
:10B2900020211A48FAF7D1FF4FF47F40ADF80000A3
:10B2A00010208DF8030003208DF802006946144831
:10B2B000FAF73EFF1248FAF7ADFF0446E4B244EA5B
:10B2C0000724A1B20E48FAF7BAFF20210B48FAF77B
:10B2D000B2FF40210B48FAF7AEFF4FF40041074898
:10B2E000FAF7A9FF4FF47F40ADF8000028208DF851
:10B2F000030069460248FAF71BFFF8BD000C014045
:10B3000000180140000801402DE9F0470746884633
:10B310004FEA8806C6F3074AB6B23D464FF0030926
:10B3200003F00AFA00BF00243146504603F046FA03
:10B33000A0B1280E03F0C4FA044624B1C5F30740B7
:10B3400003F0BEFA044624B1C5F3072003F0B8FAAF
:10B3500004461CB1E8B203F0B3FA044603F010F956
:10B3600024B9A9F1010000F0FF0901E04FF0000944
:10B37000B9F1000FD7DC03F0D5F904480068401C90
:10B38000024908602046BDE8F08700005401002013
:10B3900070B505460C4616466720FDF72FFD0628BA
:10B3A00045D2DFE800F0030D18232E3904EB4400EA
:10B3B000204A52F830103246284600F03DF836E078
:10B3C00004EB44001B4A02EBC000324641682846A9
:10B3D00000F032F82BE004EB4400164A02EBC00008
:10B3E00032468168284600F027F820E004EB44004C
:10B3F000104A02EBC0003246C168284600F01CF833
:10B4000015E004EB44000B4A02EBC0003246016930
:10B41000284600F011F80AE004EB4400054A02EB6C
:10B42000C00032464169284600F006F800BF00BF60
:10B4300070BD00006C4902082DE9F04106460C463B
:10B44000174666E0207823285DD1641C2078A0F19F
:10B450003005641C207805EB850100EB4100A0F16C
:10B460003005641C0B2D4DD2DFE805F04C060D14A1
:10B470001B222930373E45003A4640F287113046BC
:10B48000FCF7C9F93EE03A464FF4C4713046FCF788
:10B49000C2F937E03A4640F289113046FCF7BBF971
:10B4A00030E03A464FF4C5713046FCF7B4F929E074
:10B4B0003A4640F28B113046FCF7ADF922E03A46AD
:10B4C0004FF4C6713046FCF7A6F91BE03A4640F24D
:10B4D0008D113046FCF79FF914E03A464FF4C771DE
:10B4E0003046FCF798F90DE03A4640F28F113046AD
:10B4F000FCF791F906E03A464FF4C8713046FCF784
:10B500008AF900BF05E014F8011B3A463046FDF702
:10B5100087F82078002895D1BDE8F0812DE9F04129
:10B5200007460C4615461E461148007838B104F10E
:10B530003000C1B232463846FDF772F816E07CB1F1
:10B5400001200B49087032462D213846FDF768F876
:10B5500004F13000C1B232463846FDF761F805E02B
:10B5600025B1324620210020FDF75AF8BDE8F081D0
:10B570006401002070B504461148AFF30080114902
:10B5800004EBC40001EB8004002620884FF0FF3557
:10B590008107002906D00ADA8006204604D501F08A
:10B5A00076F903E02C4604E000F0F0FE30B126808E
:10B5B00000240348AFF30080204670BD2680F1E7E9
:10B5C000000000008026002010B504460C48AFF3B0
:10B5D00000800C4904EBC40001EB80042088810743
:10B5E00003D0800603D5A46805E0002403E02046CC
:10B5F00000F0C5FE64680248AFF30080204610BD2D
:10B6000000000000802600202DE9F84306460F4682
:10B610006648AFF30080684601F04CFC04004FF030
:10B62000FF3575D00146304601F092FC8146206915
:10B630000028F6D017F00C0004D004280AD00828FF
:10B6400066D103E0208840F0010006E0208840F049
:10B6500004002080208840F00200208017F0060FB0
:10B6600004D0484601F014FC002851D12088DFF8AE
:10B67000408180064FF000064BD52146484600F039
:10B6800019FF012803D02088C00772D133E00021C0
:10B690004848C4461BE000BFB0F800805FEA8872EB
:10B6A00013D0026923699A420FD1A0420DD0C28AF9
:10B6B000E38A9A4209D1026A236A9A4205D15FEA73
:10B6C000887270D4228892076DD4491C2430BCF84B
:10B6D00000209142E0DB208810F0050F06D0B9076A
:10B6E0005AD500BF40F00B00208055E02146484667
:10B6F00000F07BFEE8B3208810F0060F04D021464E
:10B70000484600F047FEA0B3B80745D52088E9E7D2
:10B7100043E0B80741D42146484600F02EFE0128F8
:10B7200003D02088C0073ED130E0002121484246A6
:10B7300017E000BFB0F800C05FEA8C730FD0036958
:10B740002769BB420BD1A04209D0838AA78ABB429A
:10B7500005D15FEA8C7326D423889B0723D4491C28
:10B76000243013889942E5DB2088410705D520461F
:10B7700000E018E000F003FE0EE0C00702D0E06930
:10B78000206209E0204600F0F4FD60B1A682214667
:10B79000484600F0ECFD30B1009D0448AFF3008056
:10B7A0002846BDE8F8832680F7E700000000000087
:10B7B00014490208802600202DE9F04107460E4674
:10B7C00015461348AFF3008045F00044CEB111494F
:10B7D00007EBC70001EB800001888A0711D001F058
:10B7E0000F02022A06D089062A46314605D500F006
:10B7F0006FFF04E04FF0FF3403E000F0C1FD00B143
:10B800002C1A0348AFF300802046BDE8F081000009
:10B81000000000008026002070B504460D460E484A
:10B82000AFF300800D4904EBC40001EB80004FF042
:10B83000FF3401888A070AD08906294602D500F01C
:10B84000E9FF01E000F0A0FD012800D1002402483A
:10B85000AFF30080204670BD00000000802600206D
:10B860002DE9F04107460D4616461148AFF300801A
:10B870004FF0FF34B5B10F4907EBC70001EB800073
:10B8800001888A070ED001F00F02012A0AD089062A
:10B890003246294602D501F075F801E000F078FD46
:10B8A00000B100240248AFF300802046BDE8F081DB
:10B8B000000000008026002030380A2801D2012034
:10B8C00070470020704710B50446B4F5004F01DD05
:10B8D000002010BD2046FFF74DFEFAE700BFFEE74F
:10B8E00010B50446B4F5004F01DD002010BD204620
:10B8F000FFF76AFEFAE70146B1F5004F01DD0120CE
:10B9000070470020FCE7000070B504460D460EA10C
:10B910002046F4F751FF10B948F2010070BD0CA1A8
:10B920002046F4F749FF10B948F20200F6E70AA1F1
:10B930002046F4F741FF10B948F20300EEE729462C
:10B940002046FFF761FEE9E7535444494E000000EA
:10B950005354444F55540000535444455252000030
:10B960002DE9F04104460D4616461F46B4F5004F3A
:10B9700003DD4FF0FF30BDE8F08132462946204616
:10B98000FFF71AFFF7E770B504460D46B4F5004F10
:10B9900002DD4FF0FF3070BD29462046FFF73CFF27
:10B9A000F9E72DE9F04104460D4616461F46B4F569
:10B9B000004F03DD4FF0FF30BDE8F08132462946ED
:10B9C0002046FFF74DFFF7E7704700000021094AC6
:10B9D0001268094B1B68D01800E0491C074A02EBAB
:10B9E00001121268521C002AF7D1884200DB401A6B
:10B9F00070470000EC020020600100209C2C002019
:10BA00002DE9F84F05464FF00009C86900900C4633
:10BA10000127C8464E46284600F0EDF8012808D117
:10BA20002846F4F7DDFD0C300D21B0FBF1F0401C91
:10BA3000C7B22069009901F056FB824600252069B3
:10BA400090F87B1019B1B5F5007F56D02AE0818FB0
:10BA5000A94227D1016C009A0025914200D900919A
:10BA60006946009E02F018FD002847D02069009921
:10BA700001F05EFE88B1009601226946206900F05F
:10BA800048F800283AD02069009900F047F90028CA
:10BA900034D04FF00008009E34E02069009900F097
:10BAA0005FF982460AEB1511206902F07FFB00283E
:10BAB00024D02069C16D05F00F0001EB4010007823
:10BAC00038B1FF2805D0E52803D04FF000096D1CE0
:10BAD000B5E7B9F1000F02D1009E1FFA85F809F110
:10BAE0000101C9B28946E5280AD0206990F87B0097
:10BAF00040B1C7F50070A84204D20020BDE8F88F1D
:10BB0000B942E4D12169A1F8788020694667012013
:10BB1000F4E72DE9F041154607460C460E6801F0A2
:10BB200011FB002818D0384601F05DFA024638466D
:10BB3000216802F053FF00280ED035B13146384657
:10BB4000226802F04BFF002806D00021384600F0A2
:10BB500005F8002800D00120BDE8F08170B504464A
:10BB6000806C0D46A8423ED094F85010012928D18F
:10BB700066697EB1216889060CD5617F022906D0ED
:10BB8000002201463046E36C01F02BFA14E0218CD0
:10BB90004218F6E76268E16CD368012298470028F2
:10BBA00020D0607F022809D16268218CA06CD36804
:10BBB0000844E16C01229847002813D0002084F843
:10BBC000500085B194F85100218C626848432844A4
:10BBD0009368E16C01229847012806D04FF0FF30AE
:10BBE000A064002070BD012070BDA564FBE7034682
:10BBF00002FB013070472DE9F04100270446B846AA
:10BC00003D463E4625E002F06FFD38B320782028FF
:10BC100024D02E2814D0A0F16101192902D9203195
:10BC2000192907D8B8F1000F03D088EA0001890666
:10BC300014D480464FB13046761C02280ED806E058
:10BC400067B9641C0026012703E0082D06D26D1C8D
:10BC5000641C20780028D6D10C2D02D30120BDE829
:10BC6000F0810020FBE7012302F006BBF8B5C169B3
:10BC70000446009100293DD0206900F071F8074684
:10BC800000252069818FA9420FD10025694602F065
:10BC900003FC00282FD02069009901F049FD58BB12
:10BCA0002069009900F05CF8074607EB1511206940
:10BCB00002F07CFA00281ED0206905F00F01C06D4B
:10BCC00000EB411630782E2809D10CA13046F4F74C
:10BCD00073FD68B10DA13046F4F76EFD40B13078C8
:10BCE00050B1E52804D0F07A0F2803D0000701D521
:10BCF0006D1CC6E70020F8BD0120F8BD2E202020D5
:10BD00002020202020202010000000002E2E2020A7
:10BD100020202020202020100000000070B50546C3
:10BD200000F01EF806464FF40071E86DF4F7FAFCD7
:10BD3000002406E03119284602F074FD00280AD0DC
:10BD4000641CA87FA042F5D80021284602F06AFDB5
:10BD5000002800D0012070BD10B5FBF7B7F810BD6A
:10BD6000838E82691A44037F032B01D0C38E1A4449
:10BD7000807F891E00FB012070472DE9F0410446B9
:10BD8000007F0025012806D0022838D0032857D08C
:10BD90000020BDE8F08102262CE03146204601F06B
:10BDA000B8F9804601462046FFF7D8FE002867D044
:10BDB00006EB4600C0F34800B0F5FF7F04D8E16C05
:10BDC000084401F02DFC0CE0E06C08F1010190F852
:10BDD000FF712046FFF7C2FE88B3E06C007847EAA7
:10BDE0000020F10701D0000901E0C0F30B0000B909
:10BDF0006D1C761C206B801CB042CED840E0022126
:10BE0000204601F086F9074601462046FFF7A6FEC8
:10BE1000A8B102260FE016F0FF0F05D17F1C3946AE
:10BE20002046FFF79BFE50B1E06CF1B230F81100F4
:10BE300000B96D1C761C206B801CB042EBD81FE053
:10BE40000221204601F065F9074601462046FFF72A
:10BE500085FEA8B102260FE0700605D17F1C394689
:10BE60002046FFF77BFE58B1E06C06F07F0150F8EA
:10BE7000210000B96D1C761C206B801CB042EBD8F1
:10BE8000284686E72DE9F04389B00E46904699464C
:10BE90000546FFF7B0FE88B301271B4C1CE0424665
:10BEA000314604A8FFF7DFFE28B1A74214D90020CD
:10BEB00009B0BDE8F083694604A800F0ACF9002899
:10BEC000F6D0684601F050FC02463146284600F0A4
:10BED0001DF80028ECD007E03A467F1C04A928464C
:10BEE00001F0BEFA0128DAD04B4642463146684698
:10BEF00000F0B0F80028DBD00120D9E7FFE7694661
:10BF0000284600F088F9E4E73E420F002DE9F74F9C
:10BF1000086982B00C46416F0091B0F878504FF03C
:10BF2000000B0298F4F75CFB81462069009901F050
:10BF3000DAF88246D846464E7DE0206990F87B10BC
:10BF400031B1B5F5007F1DD1002005B0BDE8F08FFF
:10BF5000818FA94216D1016C009A0025914200D927
:10BF6000009101226946FFF7D4FD0028EDD0206939
:10BF70000099FFF7D3FE0028E7D020690099FFF76A
:10BF8000EFFE82460AEB15110191206902F00EF9CD
:10BF90000028DAD0206905F00F010D22C06DBBF139
:10BFA000000F00EB411109F10C00B0FBF2F0C0B240
:10BFB000087001D0002200E0402210430870049A6B
:10BFC0004A73A1F81A800F2200F01F00CA72401EA7
:10BFD00000EB800202EBC000029A4FF0010B131835
:10BFE00000204A1C1F5C4FB116F800C001F80C700D
:10BFF000375C401C0D2807F80280F3D3002305E0CE
:10C00000375CCB55375CBB54FF23401C0D28F7D35E
:10C01000B9F10C0F02D9A9F10D0000E00020814612
:10C02000E843000706D101222069019902F07EFD54
:10C0300000288AD06D1CB9F1000F7FF47EAF216912
:10C04000009848672069A0F8785001207DE700003B
:10C05000365103082DE9FC5F06460D469A46012A33
:10C060000DD0002081462869416F0091B0F87870AA
:10C0700090F87B2042B1B7F5007F02D018E0012094
:10C08000F0E70020BDE8FC9F828FBA4210D1026C1D
:10C0900000278A4200D9009201226946FFF739FD44
:10C0A0000028EFD028690099FFF738FE0028E9D072
:10C0B0002869009901F017F800EB17118B462869E1
:10C0C00002F074F80028DDD0286907F00F01C06D78
:10C0D00000EB41140020315C2154401C0B28FAD3A2
:10C0E0005FEA0A004FF0000837D00646C07AE072D7
:10C0F00084F80C8084F80D80F089E081308A2082F9
:10C1000000F0DBFF014604F1120002F00BFAB08AE6
:10C11000A08201F06DFA014604F1160002F002FA65
:10C12000608A2083708B6083F069E061F0696860E9
:10C13000F069C5E9020806F11A0001F071FA044637
:10C1400006F1140001F06CFA04EB0040E8610122F2
:10C150005946286902F0EAFC56E084F80C8084F81D
:10C160000D8001F045FA014604F10E0002F0DAF903
:10C1700000F0A3FF014604F1100002F0D3F9208A79
:10C180006082E189E1822083C4F81C80C5F80C80BC
:10C19000C5F80480C5F80880B9F1000F1ED0102042
:10C1A000E072009901912869006C884200D90190E1
:10C1B000002201A92869FFF7ACFC00283FF462AF18
:10C1C0000198E861010C04F1140002F0ABF9019848
:10C1D00081B204F11A0002F0A5F907E02020E07214
:10C1E000A4F81480A4F81A80C5F81C8001225946CE
:10C1F000286902F09BFC0028E0D0B9F1000F05D0BF
:10C2000028690199FFF78AFD0028D7D0EF820098AE
:10C210002862012036E72DE9F041002704460D464B
:10C22000384620212954401C0B28FBD300212954D7
:10C2300020786178A2782E2806D111B12E2902D05B
:10C2400002E0287031E0AAB10026207868B32E28D9
:10C2500013D020280AD002F03EFAA0F16101A855BF
:10C26000192902D820F02000A855761C641C082E3D
:10C27000EBD304E02870687017E00127641C0826DF
:10C28000207890B12E2813D020280BD057B102F07F
:10C2900022FAA0F16101A855192902D820F0200046
:10C2A000A855761C641C0B2EEAD30120BDE8F08152
:10C2B0000127F7E70649096809B9052101E04FF4AC
:10C2C000FA61084600BF011EA0F10100FBD17047D2
:10C2D000580100202DE9F8430546006990F87A607E
:10C2E000416F0091B0F8784000F0FDFE07463AE05B
:10C2F000286990F87B1029B1B4F5007F15D1002092
:10C30000BDE8F883818FA1420FD1016C009A00240F
:10C31000914200D90091694602F0BEF80028EFD0A2
:10C3200028690099FFF71CFD074607EB14118846A2
:10C33000286901F03BFF0028E2D0286904F00F01D2
:10C34000761EC06DF6B200EB4110E5210170E043AE
:10C35000000700D036B901224146286902F0E6FB09
:10C360000028CDD0641C002EC2D10120C8E70020D7
:10C3700070470020704700207047002070477047CA
:10C380000020704700207047002070470020704751
:10C390000020704770B505460C460869142100F06E
:10C3A00049FD002820D028785C2800D16D1C287811
:10C3B000002819D00020E06101222146284600F023
:10C3C0009FF8002810D0206921467C30FFF718FB29
:10C3D000002809D0206900237C301A462146FFF747
:10C3E00051FD002800D0012070BD70B505460C46F7
:10C3F0000869142100F01EFD002838D028785C2838
:10C4000000D16D1C2878002831D000200246E06160
:10C410002146284600F074F8002828D0206990F8BA
:10C420007C1029B17C300022214600F01DFC02E086
:10C430002046FFF71BFC002819D02046FFF74AFFD3
:10C44000002814D0E169206902F0A8F800280ED075
:10C450002069017F032909D102F034FB002806D0AE
:10C460000021206902F0DEF9002800D0012070BD13
:10C4700070B504460E4615460421106900F0DAFC3A
:10C48000002816D020785C2800D1641C2078002871
:10C490000FD000200246E8612946204600F030F81F
:10C4A000002806D02946304600F0FAFE002800D0C9
:10C4B000012070BD70B505460C460869042100F0E6
:10C4C000B9FC00281BD028785C2800D16D1C287886
:10C4D000002814D00026324621462846E66100F0A6
:10C4E0000FF800280BD0206900227C30214600F094
:10C4F000BBFB002803D06675E069A061012070BD18
:10C500002DE9F047002706460D469146B84620E043
:10C51000286901227C30294600F0A6FBC0B95FEAF9
:10C5200009002DD00127286929467C30FFF768FAD9
:10C53000002825D0286900237C3001222946FFF7F6
:10C54000A1FC00281CD0284602F0C6F9002817D00C
:10C55000264429697C3100242046325D5C2A06D0BD
:10C56000222A04D04AB10A54401C641CF5E7641C1A
:10C5700001F80080002FD6D1CAE701F80080012021
:10C58000BDE8F0872DE9F0414FF0FF3500F1480498
:10C590008564806860604FF000062672667200F560
:10C5A000007100F58060E560C4E9051026776677C4
:10C5B0004FF00208C4F82480A4F148044FF0300181
:10C5C00004F11800F4F7D0F80021204601F0EEFD48
:10C5D00008B3E06D00F5FF7001F022F8A0F52A41E4
:10C5E000553918D1E06D0178E9290AD0EB2902D13B
:10C5F0008178902905D000F5E37001F016F8A0616C
:10C6000000E0A661204600F000FD38B1E18DB1F5F3
:10C61000007F40D104E00220BDE8F0810320FBE769
:10C62000A07F08280DD006DC01280AD0022808D0F7
:10C63000042830D105E0102803D0202801D040285C
:10C6400029D1B4F822C0BCF1000F24D0627F012AA6
:10C6500001D0022A1FD1238C666AB3421BD8A78D52
:10C6600002FB03C305EB471505F5007595FBF1F1DA
:10C670005A18B21AA262B2FBF0F22263A386E186D4
:10C680004002A0634009A08740F6F570824204D2C0
:10C690000120207716E00420BEE74FF6F5708242B5
:10C6A00002D284F81C800DE003202077204600F0A1
:10C6B000B7FD38B92046FFF760FBA066204602F0C0
:10C6C00001FA08B10020A7E70520A5E7012070477F
:10C6D0002DE9F0470446008889461746C00613D462
:10C6E0000421206900F0A6FB50B1E068A168C219DE
:10C6F0008A4201D90F1A07D0C0F3080600253AE094
:10C70000208840F0100020800020BDE8F087A1695B
:10C710002069FFF725FB627D81182069837F9A1AC3
:10C7200001F0ECFC0028F0D0A7EB050808EB0600B0
:10C73000B0F5007F01D9C6F5007820694246C06D8A
:10C74000811909EB0500F3F776FF06EB0800C60533
:10C75000F60D0FD1607D401CC1B261752069827FEA
:10C76000914207D10021617504F1180101F094FE96
:10C770000028CAD04544BD42C9D3E0682844E060DF
:10C780002846C2E770B506460C46154614211069C6
:10C7900000F050FB002839D030785C2800D1761C9E
:10C7A00020785C2800D1641C307880B3207870B386
:10C7B00000200246E86129463046FFF7A1FE002826
:10C7C00024D0286990F87C0080B1002632462946A2
:10C7D0002046FFF748FA01281AD0286900227C3049
:10C7E000294600F041FA002810D007E00126324621
:10C7F00029462046FFF737FA012809D03246294654
:10C80000204601F0FCFC002800D0012070BDFFE7AD
:10C810000020FBE72DE9F041044600880D46C006E4
:10C8200002D50020BDE8F0810421206900F002FB60
:10C8300040B3A068A84200D205462069690A827FF9
:10C84000B1FBF2F302FB13116175E769A761806B1D
:10C85000B5FBF0F656B104F118084146A769206906
:10C8600001F01AFE0028DDD0761EF6D1A1692069FC
:10C8700000F05EFF18B12069807F6075A76101201C
:10C88000E560CFE7208840F010002080C9E7F0B5D0
:10C890000446008889B0C0065FD41421206900F0E6
:10C8A000C9FA002855D0D4E9010181424CD9491E6A
:10C8B0002046FFF7AFFF002850D0206900F093FB1F
:10C8C0000246A169206902F089F8002846D069462D
:10C8D000204601F050FC002840D0E069000CADF883
:10C8E0001400E069ADF81A00A068079000F080FE1F
:10C8F00001460DF1160001F015FE00F0DEFB0146C9
:10C9000006A801F00FFEBDF81800ADF812006F4642
:10C91000E58A216A206900F0E6FB00EB15110E465E
:10C92000206901F043FCC0B1206905F00F0120220D
:10C93000C06D00EB41103946F3F7C2FE01223146CB
:10C94000206902F0F3F840B12069017F032907D084
:10C950000AE0208840F010002080002009B0F0BDDF
:10C9600002F0B0F80028F9D00021206901F05AFF48
:10C970000028F3D000212069FFF7F0F80028EDD05F
:10C980000120EBE72DE9F74F0446008882B01746F7
:10C99000C00603D5002005B0BDE8F08F1421206942
:10C9A00000F048FA60B121884FF4007909EA811B50
:10C9B00004F11800E1694FF0000A009029B10EE07F
:10C9C000208840F010002080E4E72069009900F002
:10C9D000B9FB0028DFD0A069E06184F815A0E06809
:10C9E0000025C0F308064CE02069617D827F9142FA
:10C9F00018D1E168A2682944914203D2009901F05C
:10CA00004BFD0BE0D4F81880009900F09BFB002848
:10CA1000C1D04146A269206901F0E0FF0028BAD0E8
:10CA200084F815A0A1692069FFF79AF9617D08448F
:10CA300001900EB95F4505D22069019901F0B6FB5E
:10CA40000028A8D0A7EB050808EB0600484501D947
:10CA5000C6F500780398424641192069C06D3044FC
:10CA6000F3F7E9FD2069019901F0DCFE002892D07E
:10CA700006EB0800C605F60D02D1607D401C60750E
:10CA80004544BD42B0D3E0682844E060A1688842D4
:10CA900000D9A06001207EE72DE9F05F05460C4635
:10CAA0006848AFF30080002000F004FA060055D07B
:10CAB0000146284600F04CFA8246306900284DD0E5
:10CAC00000205146024604E0401C5C2B00D1024687
:10CAD000491C0B78002BF7D10AEB020083465AA1C0
:10CAE000F3F76AFE00B32A21584600F06DFA0546B6
:10CAF0005846F3F775FD8046681C1AD04FF00109BF
:10CB00000BEB050051A1F3F757FE18B1A8EB050098
:10CB1000A0F101008046308880060DD532462146BE
:10CB20005046FFF7A5FC0BE000254FF00109A84691
:10CB3000F1E74FF00009EEE731462046FFF71BFC16
:10CB400060B1002084F8FF00B9F1000F08D055EA69
:10CB500008001FD0CDB35946002349E001242EE040
:10CB600023465A4610E05B1C12F8011BA0F1610736
:10CB7000192F01D820F02000A1F16107192F01D849
:10CB800021F020018842C6D118780028EBD1117815
:10CB90000029E8D13088800603D5307D84F806016D
:10CBA00009E0002084F80601F082B4F80401B082A4
:10CBB0003046FFF7E4FB7068C4F800010024214808
:10CBC000AFF300802046BDE8F09F13E011F8012B81
:10CBD000E05CA2F16107192F01D822F02002A0F138
:10CBE0006107192F01D820F02000824293D15B1CED
:10CBF000AB42EBDBB8F1000FCCD02046F3F7F0FCF2
:10CC0000844605EB0801614585DC0BEB05035B1CE5
:10CC1000ACEB080212E000BF13F8010BA15CA0F11D
:10CC20006107192F01D820F02000A1F16107192F09
:10CC300001D821F020018842A5D1521C6245EBDBCE
:10CC4000A8E70000000000002A2E2A002E2A00007B
:10CC50000168002901DCF4F744B8491E016041680D
:10CC60004A1C426008787047002301F005BB0000B1
:10CC7000F0B5044689B01A48AFF3008000F0AAF876
:10CC8000BCB10020ADF8000004906946204600F0D9
:10CC90005FF9049808B3BDF8000000F02001049883
:10CCA00000F0CEFC04460E48AFF3008009B02046E9
:10CCB000F0BD00240B4D26460B4F0AE0E87900F04A
:10CCC0000401286800F0BCFCA04200DD0446761C8C
:10CCD000083538888642F1DBE5E70324E3E7000006
:10CCE0000000000030490208164902088A68002A3C
:10CCF00001DCF4F7E9B9521E8A604A68C0B2531CDD
:10CD00004B60107070470000F0B5044695B00F46B8
:10CD10002F48AFF30080002000F0CCF805004ED083
:10CD20000146204600F014F90646286980B3288899
:10CD300080062ED53046F3F753FC441E06D4305DF2
:10CD40005C2802D0641EFAD500E06CB1621C31464A
:10CD50006846F3F770FC0DEB04010020487039467B
:10CD60006846F3F75CFC07E03846F3F739FC024607
:10CD700039466846F3F75FFC29466846FFF79AFB99
:10CD800001281CD02A4639463046FFF7FBFC14E048
:10CD900015E029463846FFF7F0FA01280FD029465A
:10CDA0003046FFF7EAFA50B1284600F0A7F801280C
:10CDB00005D029463846FFF7E5FA012806D00124B8
:10CDC0000348AFF3008015B02046F0BD0024F7E71C
:10CDD0000000000070B5124C207800281ED100F031
:10CDE00041F800220F4811460F4B05E0C5796D0749
:10CDF00050F8085B521C29601D88AA42F6D3002017
:10CE00000A4B0B4A05E000BF00EBC005401C23F8AD
:10CE100025101588A842F7D30120207070BD0000AE
:10CE20000404002030490208164902088026002028
:10CE30001449020810B504460068814301D000205F
:10CE400010BD000706D4606800214269084690477B
:10CE5000C00701D0012010BD206820F0060020602E
:10CE6000EDE7000007480021A0F58062C0E902213B
:10CE7000054A426000F5C073044A9A60416101822C
:10CE800070470000102B0020184902084C49020886
:10CE900060B1017851B1012100E0491C425C002AD7
:10CEA000FBD1084410F8010C5C2801D00020704729
:10CEB0000120704770B5064600240A4D0A4804E078
:10CEC0002988890706D02435641C01888C42F7DB49
:10CED000002070BD24212846F3F746FC06B13460DB
:10CEE000284670BD8026002014490208004870477B
:10CEF0000101DB074FF440207047000030B50022ED
:10CF00001149124B1AE00C88A40715D0814213D0A6
:10CF10000C690569AC420FD10488A40609D5CC8AF6
:10CF2000C58AAC4208D10C6A056AAC4204D1012022
:10CF300030BD8C8A858AF8E7521C24311C88A242B5
:10CF4000E1DB002030BD00008026002014490208EB
:10CF5000F0B51B4A1B4CE8B10378DBB123F0200687
:10CF600043783A2B03D085783A2D03D012E0302352
:10CF7000801C01E073B1C01C002507E01779B7429F
:10CF800002D157799F420AD06D1C08322788BD42D2
:10CF9000F4DBF0BD00230EE0D579ED0709D013686E
:10CFA0000B61D2795207F4D50A8842F020020A8038
:10CFB000F0BD5B1C08322588AB42EDDBF0BD000004
:10CFC0003049020816490208002205E08B4201D1CF
:10CFD00010467047401C521C0378002BF6D1581E97
:10CFE000704700207047007F012805D0022806D036
:10CFF000032807D00020704740F6FF7070474FF6B7
:10D00000FF7070476FF07040704710B5044681693B
:10D0100001F0CCF8002809D0E06D00F5FF7000F0B9
:10D02000FFFAA0F52A41553901D0002010BDE06D6E
:10D03000417BA1770B3000F0F3FAE085E06D0E3014
:10D0400000F0EEFA6084E06D017C6177113000F051
:10D05000E7FAA085E06D133000F0E2FA6062E06D5F
:10D06000163000F0DDFA2084616AE9B9B8B9E06DE4
:10D07000283000F0D5FAE087E06D2C3000F0D5FACA
:10D080002064E06D303000F0CBFAA4F84400E06D8D
:10D09000323000F0C5FAA4F84600606A20B9E06DAD
:10D0A000203000F0C2FA6062208C20B9E06D24309C
:10D0B00000F0BBFA2084012010BD10B5FFF716FF69
:10D0C00010F01F0100D10121C0F303220C2A00D867
:10D0D00002B9012241EA4211442202EB104041EA26
:10D0E000402080B210BD10B5002280F87B2059B9D5
:10D0F0000267017F032906D0828E816911440122D3
:10D1000080F87B2003E0016CFEF72AFE014608460A
:10D1100010BD027F012A04D0022A06D0032A0AD1B8
:10D1200005E001EB4101890A02E0090A00E0C909B2
:10D13000028C8A4201D8002070478269408C1044DA
:10D14000084470472DE9F04105460E46C46E5CE088
:10D1500021462846FFF7DDFF804601462846FEF7B8
:10D16000FDFC002838D0287F012804D0022823D0D5
:10D17000032830D127E004EB4400C0F34800B0F5A9
:10D18000FF7F04D8E96C084400F04AFA0DE0E86C2F
:10D1900008F1010190F8FF712846FEF7DFFC002836
:10D1A0001AD0E86C007847EA0020E10701D00009B6
:10D1B0000FE0C0F30B000CE0E96C200601EBD0504F
:10D1C00000F02EFA05E0E96C600601EBD05000F0AB
:10D1D0002CFA18B118E00020BDE8F0810E480021BB
:10D1E00002880E4809E003889F0604D59B0702D5F4
:10D1F0008369A34208D02430491C9142F3D33460A0
:10D20000641C0120EC66E7E7641C286B801CA042CC
:10D210009ED8EC66DFE70000144902088026002053
:10D2200010B504468069B4F844100144204600F06B
:10D23000BDFF002829D0E06D00F5FE7000F0F5F983
:10D240001449884220D1E06D00F0EFF9124988427C
:10D250001AD1E06D00F5F27000F0E7F90F4988424D
:10D2600012D1E06D00F5F47000F0DFF9216B81421E
:10D270000AD3A066E06D00F5F67000F0D6F902283A
:10D2800002D3216B814201D2002010BDE066012053
:10D2900010BD0000000055AA5252614172724161F6
:10D2A0002DE9FF5F054600200E4602900190039095
:10D2B000C969814600913069FFF715FFB5F804711F
:10D2C00082464FF0000B306990F87B00E0B1B7F573
:10D2D000007F10D01CE07F1A016C009A914200D9A7
:10D2E0000091694601F0D8F8002805D0306900990E
:10D2F00000F01EFA18B1002004B0BDE8F09F3069BC
:10D300000099FEF72DFD82463069818FB942E2D93E
:10D3100009F101090AEB1711306900F047FF0028F5
:10D32000EAD0306907F00F01C06D00EB411420789E
:10D330000028E1D0E5285AD0E17A0F2902D0080769
:10D3400055D407E0400605D5012003900190607B8D
:10D35000029011E0039878B30F290BD000200390BE
:10D36000204600F001FA0199002975D002998842FF
:10D3700048D001E00198D0B3617B0298814202D08D
:10D380000020019068E02078344B00F01F00401E20
:10D3900000EB800101EBC00805EB080100201A5CDE
:10D3A000A25C0A54401C0D28F9D3207808F10D081E
:10D3B000400601D505F808B0E07A00F03F000F28DC
:10D3C0004AD0072100E0491E605C2028FBD0491CA0
:10D3D000002002E0225C2A54401C8842FAD3217AC1
:10D3E00020290DD02E212954401C082103E033E0D0
:10D3F0002A54491C401C625C202A01D00B29F7D317
:10D4000005F800B005F58275298801EB0900288030
:10D41000E07A307504F11C0000F007F97060B0602C
:10D4200004F1160000F0FCF8C10A2971C0F345119F
:10D43000C0066971800EA87104F1180000F0F0F8C0
:10D4400000F01F01E971C0F34311400A297200F294
:10D45000BC70688101204FE77F1C34E73651030818
:10D460002DE9F84F834660480E4615464FF0000AF6
:10D470004FF6FF78824201DD062713E042F20F707B
:10D48000854201DD05270DE0B5F57A7F01DB042734
:10D4900008E0632D01DD032704E0092D01DD0227EB
:10D4A00000E00127002003E02E2900D18046401C27
:10D4B0001BF800100029F7D105B94F1E4FF00009E5
:10D4C000C7F107004C46009018E000BF1BF809A008
:10D4D000BAF1200F10D0BAF12E0F0DD0BAF1000F13
:10D4E00011D0AAF16100192801D82AF0200A50466B
:10D4F00001F0F1F83055641C09F10109C14502D26F
:10D500000098A042E2D8EDB37E203055641C072F6E
:10D5100046D2DFE807F04542352A1E1204003248A1
:10D520003249401C95FBF0F0414305EB41150928B9
:10D5300000D9092030303055641C42F2107095FB40
:10D54000F0F06FF41C7141433030305505EB01159C
:10D55000641C4FF47A7095FBF0F06FF07C0141434E
:10D560003030305505EBC105641C642095FBF0F0AC
:10D570006FF0180141433030305505EB8105641CD4
:10D580000A2000E00CE095FBF0F04142303001EB66
:10D590008101305505EB4105641C30353555641C5F
:10D5A000BAF1000F1AD02E203055641CA8F57F4127
:10D5B0004046FF3912D0451C071D0DE01BF8050041
:10D5C00060B1A0F16101192901D820F0200001F01B
:10D5D00082F83055641C6D1CBD42EFD300203055DD
:10D5E0000120BDE8F88F00009F860100CBF3FFFF0C
:10D5F00010B5FFF77FFCC0F344011D2900D90021BD
:10D60000C0F305223B2A00D90022C0F3044041EABE
:10D610004211172800D9172041EAC02080B210BD5E
:10D620004178007840EA01207047C1788278090685
:10D6300041EA02414278007841EA022108437047FA
:10D6400010B5044640680022B1B318B12068C00785
:10D6500002D00BE0032010BD22606068016800204A
:10D66000884750B3206840F001012160206820F015
:10D670001E0121606068002142690846904701064A
:10D6800003D5206840F0180106E0C10738D08007B4
:10D6900003D4206840F01001216060680168012017
:10D6A000884750B1206840F0020120462160FEF713
:10D6B00069FF18B1022010BD0AE021E0206840F0A7
:10D6C000040120462160FFF701F8F0B90420F2E7D9
:10D6D00068B12068C0070AD12260D4E90120E1695D
:10D6E0001268904760B1206840F001002060206817
:10D6F00040F004002060616821B1896811B104E044
:10D700000120D8E740F0100020600020D3E700009F
:10D710000246002106E00548405C904201D101200C
:10D720007047491C0A29F6DB0020F9E7280300208E
:10D73000007F012804D0022805D003280FD107E07C
:10D7400040F6F87001E04FF6F870814205D206E02D
:10D7500021F070400349884201D301207047002026
:10D7600070470000F8FFFF0F024600200146C30784
:10D7700000D0802303EB5000535C491C1844C0B216
:10D780000B29F4D370470000FBF7B2F8F9F736FC29
:10D79000F8F720FBF5F7CCFBFCF7ACFAFDF724F823
:10D7A000F3F774FEF8F7DEFEFBF7A4FAF8F704FFD0
:10D7B000F9F7AEFBF4F754FDF4F752FD002063498E
:10D7C00008600520624908604FF4167061490860DE
:10D7D00000206149087061490860012060490860C3
:10D7E000F4F78EFD6820FBF709FB044640F2E732B0
:10D7F0005C4801682046FDF703FD42F6681164208D
:10D80000FDF7B6FCF4F7A0FE4FF42F705649086000
:10D81000FCF7D8FEF4F7DEF9FDF746FCF4F79CFAC6
:10D8200000210A20FDF7A4FC00210B20FDF7A0FC3D
:10D8300000210C20FDF79CFCFBF71AFE01204B4950
:10D8400008604FF42F704A49086048607CE0FBF79D
:10D85000D5FEF3F7F7FE3E48006810B901204549B0
:10D860000870FBF7DBFB3D4800683C490968491C30
:10D870003A4A1160062836D006DC062845D2DFE891
:10D8800000F013161924272F092835D004DC0728A7
:10D890002CD0082839D12CE00A2830D0A0F5985097
:10D8A0008838002831D12DE0F4F72AFD31E0F4F773
:10D8B000EFF92EE0F8F700FE27480078012803D1A1
:10D8C00041F288302549086023E0F4F79BFC20E012
:10D8D0001F48006818B142F210702049086018E033
:10D8E000F4F79EFE15E0F4F70BFB12E0F4F77EFC74
:10D8F0000FE0F4F77DFA0CE0F4F798F809E0F4F79C
:10D90000C9F906E0F4F74CFB03E000201349086076
:10D9100000BF00BF18480068B0F5FA7F05DA4FF481
:10D9200080611648F8F789FC04E04FF480611348E1
:10D93000F8F781FCF5F7E4FCF4F706FEF4F790FC49
:10D94000F4F7C8F8F8F71EFE81E700006800002031
:10D95000C4000020280100206C0100200C000020E1
:10D96000040000203000002038000020600000206B
:10D97000F40B00201000002014000020000C0140D7
:10D98000014A00F05FB80000902C0020014900F02F
:10D9900066B80000902C0020014900F05DB900003D
:10D9A000902C0020014B00F067B90000902C002063
:10D9B000014900F08DB90000902C0020014B00F0CF
:10D9C00093B90000902C00202DE9F041074618493A
:10D9D000184A126831F81200F8F734FD0646F8F7D5
:10D9E00031FC054614481349096850F821002C1AE7
:10D9F000002C00DA64420A2C0EDB10480D4909683D
:10DA0000405C401CC0B20D490A4A12688854642820
:10DA100002DC0B48006848B107480649096840F82D
:10DA2000215000200549034A12688854BDE8F0815E
:10DA3000800D0020D4000020F40B0020D80000202E
:10DA4000C400002018B1022807D000207047906859
:10DA5000C06900B1004780207047506870472DE9C9
:10DA6000F8430C4610B101287DD104E088680068B5
:10DA70008047BDE8F883A068816901208847A068D5
:10DA800041694FF4C87088470025A0688168FF206D
:10DA900088476D1C102DF8D3A06881690020884745
:10DAA000002223461146104600F04CF90546002698
:10DAB000012D07D0A0688168FF208847761C0546A5
:10DAC000642EF5D3A068816901208847012DCBD150
:10DAD000A068416944F62060884700202070A06853
:10DAE00081690020884704268DF8006023466A4635
:10DAF0004FF4D571082000F025F901280FD19DF8C9
:10DB0000000060B99DF8010048B99DF802000128A5
:10DB100005D19DF80300AA2801D103202070A06838
:10DB200081690120884700254CF25038A06881693E
:10DB300000208847002223461146372000F002F9D2
:10DB40000746A06881690120884778071AD4012F09
:10DB500015D1A0688169002088472078032815D056
:10DB60000020810700E06EE023460022292000F01B
:10DB7000E9F80746A06881690120884747B16D1C14
:10DB80004545D3D32078032807D01EE00120E8E7DD
:10DB90002078032801D0022033E0A06881690020AA
:10DBA00088478DF8006023466A4600213A2000F03D
:10DBB000C9F80546A0688169012088472DB99DF8FC
:10DBC0000000400601D526701CE02078D0B9002561
:10DBD0004746A068816900208847002223461146F5
:10DBE000012000F0AFF80646A0688169012088474F
:10DBF000012E01D03EBB03E06D1CBD42E9D322E003
:10DC000001202070A06881690020884723460022F7
:10DC10004FF40071102000F095F80546A068816966
:10DC2000012088477DB9A0688169002088470022CB
:10DC3000234611463B2000F085F80546A06881691F
:10DC4000012088470DB1002013E7204600F002F9BB
:10DC50000028F9D001200CE770B505460C460846AF
:10DC600000F0F8F8002806D02146284600F017F901
:10DC7000002800D0012070BD2DE9F04106469868CB
:10DC80000F46154681691C460020884723462A46D0
:10DC90003946304600F0A6F80646012D0FD900227D
:10DCA000234611460C2000F04DF8084DA06881680D
:10DCB000FF208847FF2802D06D1EF7D10026A068FC
:10DCC0008169012088473046BDE8F08148E80100BD
:10DCD00038B101284FF0000002D1087048600120DF
:10DCE00070478868406800472DE9F041064698680B
:10DCF0000F46154681691C460020884723462A4660
:10DD00003946304600F046F90646012D11D9A06883
:10DD10008168FD208847A0688168FF208847084DFA
:10DD2000A0688168FF208847FF2802D06D1EF7D1C8
:10DD30000026A0688169012088473046BDE8F0814F
:10DD400048E801002DE9FC4140F040008DF800005A
:10DD5000080E8DF80100080C8DF80200080A8DF8F5
:10DD60000300002014461D468DF804106A46014643
:10DD700005234E0707D1B3EBD10F04D902EBD1062F
:10DD8000367846EA0000060401D580F409404000D8
:10DD9000491C3029EDD3000A40F001008DF8050040
:10DDA000A8688168FF208847A8680621C26868467D
:10DDB00090470027A8688168FF2088470646FF280B
:10DDC00002D17F1C082FF5D34CB1277805E0A86855
:10DDD0008168FF20884704F8010B7F1EF7D2F0B25C
:10DDE000BDE8FC812DE9F04111250F4616461C4681
:10DDF000012A00D912252178042900D240020146C7
:10DE000000222846FFF79EFF10BB1CE046F2A81533
:10DE1000A0688168FF208847FE2802D06D1EF7D1D8
:10DE200016E0ADB1A0684FF4007102693846904722
:10DE3000A0688168FF208847A0688168FF20884724
:10DE400007F50077761E002EE0D10120BDE8F081B5
:10DE50000020FBE77FB50446806881690020884781
:10DE60002346102269460A2000F06CF80546A06897
:10DE700081690120884775B12078012868460CD057
:10DE800009300168C07809BA21F0FF01014301207F
:10DE9000616004B070BD0020FBE70A30F1E77FB598
:10DEA000044688680D468169002088472B46102269
:10DEB0006946092000F046F80646A86881690120F5
:10DEC0008847B6B19DF80500012100F00F0001FA66
:10DED00000F0A080BDF80C0040BAC0F38310814070
:10DEE000E1809DF80000800906D0012819D00228A1
:10DEF00002D0002004B070BD9DF806009DF8071008
:10DF0000000440EA01209DF808100843BDF80910FC
:10DF1000C0F38B1049BAC1F3C211401C891C884060
:10DF20000DE09DF807009DF80810000440EA01206C
:10DF30009DF8091008430004800900F58060206006
:10DF40000120D7E72DE9F04117460E4600221C4676
:10DF50001146FFF7F7FED8B946F2A815A068816808
:10DF6000FF208847FE2802D06D1EF7D110E07DB15A
:10DF7000A0683946026930469047A0688168FF2052
:10DF80008847A0688168FF2088470120BDE8F081AC
:10DF90000020FBE72DE9F0411826884615461C466F
:10DFA000012A00D919262178042900D2400201460D
:10DFB00000223046FFF7C6FE38BBFE27012D29D9C7
:10DFC000FC2727E0A068816838468847A0684FF49E
:10DFD0000071C26840469047A0688168FF2088476A
:10DFE000A0688168FF208847A0688168FF20884773
:10DFF00000F00F00052812D10A4EA0688168FF20AA
:10E000008847FF2802D0761EF7D108E03EB108F518
:10E0100000786D1E002DD5D10120BDE8F0810020D3
:10E02000FBE7000020A1070000B50246104600F003
:10E0300003F83030C0B200BD01464D2920D00CDCC1
:10E040002D2923D004DC1D2910D02B2922D11FE03B
:10E050002E2919D04B291DD114E04E290ED08B2921
:10E060000AD08D2906D08E2914D101E000207047F6
:10E070000120FCE70220FAE70320F8E70420F6E796
:10E080000520F4E70620F2E70720F0E70820EEE796
:10E090000920ECE70020EAE770B500248020104951
:10E0A0000880032088700420C8700E48F8F740F8F4
:10E0B000002510E06006040EFBF76EFFFEF7FAF88D
:10E0C00080210848F8F7A9F808B144F00104FBF7EB
:10E0D0006DFF681CC5B2082DECDB204670BD00004A
:10E0E0005C010020000C014010B5FBF77FFFFBF73F
:10E0F00053FFFBF75BFFFBF763FF10BD70B50446F2
:10E10000C0680D46164610B194F8641029B129462E
:10E110002046BDE8704000F049B894F8652082B10F
:10E12000A16DA9420DD80A44AA420AD9206E691AE3
:10E1300000EB41214FF40072E06DF2F77CFA656567
:10E1400017E0B04200D206466068E16D324683684F
:10E1500028469847012806D04FF0FF306065002020
:10E1600084F8650070BD65656D1C761EA56584F834
:10E170006560012070BD70B50E460446C58A016A0F
:10E180000069FEF7B0FF00EB1511206900F00EF8F2
:10E1900000280AD0206905F00F012022C06D00EB95
:10E1A00041113046F2F78CFA012070BD70B504467B
:10E1B000406D0D46A84201D1012070BDA06DA8425E
:10E1C0000ED894F864100144A94209D9216E281A86
:10E1D00001EB40214FF40072E06DF2F72CFA0CE0F5
:10E1E0006068E16D0122836828469847012804D0C1
:10E1F0004FF0FF306065002070BD6565DCE72DE9FC
:10E20000F0410746086988B00C4690F87A6090465D
:10E2100000253846FDF7EFFC60B1012E09D03846E5
:10E22000F2F7DEF90C300D21B0FBF1F0401CB042EA
:10E2300000D9012569462046FFF79DFF002817D029
:10E240002046FEF747F8002812D045B12069214644
:10E25000406FE0613846FDF7D3FB002808D06B46DD
:10E26000424621463846FDF70DFE002800D0012029
:10E2700008B0BDE8F08100002DE9FF4F97B00C46D3
:10E28000012A19D00020129001204FF0000ACDE998
:10E290000E0A0390E06900901798F2F7A1F9049034
:10E2A0000020109021698346E06908671798FDF700
:10E2B000A2FC012802D009E00120E4E704980D2126
:10E2C0000C30B0FBF1F0401CC0B20E9009A91798B9
:10E2D000FDF7A1FF129808B1092000E00D2007907A
:10E2E00020690099FEF7FFFE81460026206990F81C
:10E2F0007B1019B1B6F5007F13D01BE0818FB142BE
:10E3000018D1016C009A0026914200D9009169460B
:10E3100000F0C2F8002805D020690099FFF708FA3C
:10E3200018B100201BB0BDE8F08F20690099FDF7FF
:10E3300017FD814609EB16112069FFF737FF00280A
:10E34000F0D0206906F00F01C06D00EB4115287870
:10E350000028E7D0E5286FD095F80B80B8F10F0FB3
:10E3600003D05FEA087067D431E0410609D500990F
:10E370001091697B0F9120F04001491CC9B2B3464E
:10E3800003916A7B0F998A4256D100F01F00401E0C
:10E3900000EB800101EBC0001799DFF8F8C00A1804
:10E3A000002000BF1CF80010135C695C81EA0307C1
:10E3B00037F0200708D103B911B1401C0D28F1D363
:10E3C0000AF1010000F0FF0AB8F10F0F34D00398F2
:10E3D00001280ED029D9A0F1010050451BD12846B3
:10E3E000FFF7C2F90F99884215D10AF10100C0B2B6
:10E3F0001AE00E98012803D007990498884214D295
:10E4000000981090B34609A9284600F097F878B113
:10E410004FF0010A12E00E98012806D109A92846FA
:10E4200000F08CF808B1039882460398504505D057
:10E4300001204FF0000A0390761C57E7E87AC0F3FA
:10E44000001112988142F3D11A9808BBE87A20751E
:10E4500005F11A00FFF7E4F8074605F11400FFF78D
:10E46000DFF807EB0040E061E68200982062216956
:10E470001098486721690020A1F878B0216981F8D7
:10E480007AA0E06005F11C00FFF7CFF86060A060A3
:10E49000012047E7365103082DE9F0410D680E468B
:10E4A00004462946FEF735FE804601462046FDF724
:10E4B00055FB002807D0207F012806D0022825D050
:10E4C000032828D00020BDE8F08105EB4500C0F30B
:10E4D0004800B0F5FF7F04D8E16C0844FFF7A0F8CE
:10E4E0000DE0E06C08F1010190F8FF712046FDF7A6
:10E4F00035FB0028E7D0E06C007847EA0020E90708
:10E5000001D000090BE0C0F30B0008E0E16C280625
:10E51000C00D085A03E06806E16CC00D0858306071
:10E520000120D0E70A0A4270017070470A0EC270DB
:10E530000A0C82700A0A42700170704730B50022DE
:10E54000835C8C5C83EA040535F0200501D0002053
:10E5500030BD04B913B1521C0B2AF1D3012030BDD8
:10E5600010B5FBF72DFDFBF717FDFDF7A3FEFBF73D
:10E570003DFDFDF79FFEFBF719FDFDF79BFE10BD6E
:10E5800010B5FBF733FDFDF795FEFBF705FDFDF735
:10E5900091FEFBF715FDFDF78DFE10BD2DE9F0474F
:10E5A0000026012704460D4602297DD379E0E06E5E
:10E5B000A84200D9E56629462046FEF7AAFD814615
:10E5C00001462046FDF7CAFA00287AD0207F0128AC
:10E5D00004D0022846D0032872D14DE005EB450057
:10E5E000C0F34808B8F5FF7F16D8E16C01EB0800CE
:10E5F000FFF716F8E90703D000F00F01000903E068
:10E6000000F47041C0F30B00E26C814602EB08009D
:10E6100089B2FFF787FF3BE0E06CEA0790F8FF1153
:10E62000884604D001F00F0180F8FF1101E080F866
:10E63000FF6184F8507009F101012046FDF78EFA60
:10E6400000283ED0E06CEB07017848EA012202D0B6
:10E650000670100904E001F0F0010170C2F30B0034
:10E66000814615E02806C50DE06C2844FEF7D8FF6A
:10E670008146E06C46530BE06806C50DE06C28440B
:10E68000FEF7D3FF8146E06C4651A06E401CA066A9
:10E6900084F8507049462046FFF74AF8012812D006
:10E6A0004D46206B801C02E013E00AE008E0A8421F
:10E6B0003FF67DAF00212046FDF750FA002800D03C
:10E6C0000020BDE8F08700212046FDF747FA00282A
:10E6D000F7D00120F5E710B5044600F005F808B1C1
:10E6E000204610BD582010BDA0F12001012917D9E6
:10E6F000C91E062914D92D2812D02E2810D00D3964
:10E7000009290DD940280BD01139192908D91D39EB
:10E710001D2905D97D2803D07E2801D0002070470F
:10E720000120704710B501210248F7F786FDFDF77B
:10E73000C1FD10BD0018014010B501210248F7F7D6
:10E740007AFDFDF7B7FD10BD0018014070B5044615
:10E75000254600260FE005F0800010B1FBF730FCE5
:10E7600001E0FBF743FC6806050EFBF715FCFBF721
:10E770001DFC701CC6B2082EEDDB70BD70B5012506
:10E78000FBF71EFCFBF708FC80210A48F7F745FD64
:10E7900000B10025FBF70AFC07480068012806D1F4
:10E7A000002402E0FDF786FD641C0A2CFADB2846F3
:10E7B00070BD0000000C0140580100202DE9F0411F
:10E7C00007460C460A201649086000BFFFF7C8FE3E
:10E7D000A02101EB4701C8B200F072F805460DB95F
:10E7E000FFF7CEFE1DB90E4800680028EED145B1F6
:10E7F0002646E11704EB1161C1F3072000F060F831
:10E80000054655B12646E11704EB11610912A4EB48
:10E810000121C8B200F054F805462846BDE8F08151
:10E82000500100202DE9F0410D46C1680446E1B1D8
:10E8300000261DB3656594F864204FF400779AB301
:10E84000A06D8318AB4227D18A4225D204F15C0423
:10E850006068216800EB42203A46F1F7ECFE207A2E
:10E86000401C20720120BDE8F081002DFAD000226A
:10E87000294600F05BF90028F5D0F3E794F864200E
:10E88000002AEFD06368216EA06DDB6898470028EE
:10E89000E9D084F86460E5E76368216EDB68984737
:10E8A0000028E0D084F8646004F158043A46D4E9C2
:10E8B0000110F1F7C0FE0120256020736673D1E7D7
:10E8C00010B504462046FFF741FFFFF757FF08B198
:10E8D000012010BD0020FCE72DE9F0410446C76986
:10E8E000FEF786FE0646FEF7E8FB804620694FF4F9
:10E8F0000071C06DF1F716FF20690B2234A1C56DC0
:10E900002846F1F7DDFE1020E872314605F10E00D1
:10E91000FFF708FE414605F11000FFF703FE4146F0
:10E9200005F11200FFF7FEFD314605F11600FFF775
:10E93000F9FD414605F11800FFF7F4FD05F120004F
:10E94000202229460646F1F7BBFEE069010C05F1DD
:10E950001400FFF7E7FDE06981B205F11A00FFF747
:10E96000E1FD2E2070702069006F010C06F114008B
:10E97000FFF7D8FD2069006F81B206F11A00FFF79A
:10E98000D1FD2169E069086739462069FDF7E8F99A
:10E99000064601223146206900F0C8F8002814D04C
:10E9A00020694021C06DF1F7BDFE012506E0711917
:10E9B000002200F0BBF8002807D06D1C2069817F81
:10E9C000A942F4D80220E0820120BDE8F0810000D5
:10E9D0002E20202020202020202020002DE9F0477C
:10E9E000154604460E46FEF794FB81460146204636
:10E9F000FDF7B4F8002809D0207F4FF00108012866
:10EA000006D0022844D0032848D00020BDE8F08773
:10EA100006EB4600C0F34807C5F30B05B7F5FF7FCB
:10EA200013D8E06C3844FEF7FBFDF10702D065F324
:10EA30001F1002E000F470402843E16CCA1981B253
:10EA40004FEA0200FFF76EFD38E0F007E06C06D0F9
:10EA500090F8FF1165F31F1180F8FF1101E080F8B5
:10EA6000FF5184F8508009F101012046FDF776F846
:10EA70000028CBD0F00703D0E16C280908701DE016
:10EA8000E06C017801F0F00141EA1521017015E018
:10EA9000E16C300601EBD050A9B2D3E77006C60D89
:10EAA000E06C3044FEF7C1FD18B9A06E08B1401EFD
:10EAB000A066E06C29463044FFF738FD84F85080AA
:10EAC0000120A3E710B50446C06D4FF40071F1F7C3
:10EAD00029FE1449E06DFFF729FDE06D124900F5AC
:10EAE000F270FFF723FDE06DA16E00F5F470FFF703
:10EAF0001DFDE06DE16E00F5F670FFF717FDE06DAE
:10EB00004AF6552100F5FF70FFF70CFDB4F84410EC
:10EB1000A06901442046FFF785FE002800D00120AF
:10EB200010BD0000525261417272416170B50446DD
:10EB30000D464069E16D08B1012A09D060680122E3
:10EB4000C36828469847002801D00120656570BD3C
:10EB50000B4600222946FEF744FAF4E700000000C5
:10EB60003000002000000000000000009F050000B1
:10EB70000000000040480000010000001C000020D0
:10EB8000670000000000000003000000000000001B
:10EB900002E80000020000001C00002068000000E5
:10EBA00065000000280C00006500000002A80000BD
:10EBB000030000001C00002069000000D0070000D6
:10EBC000B80B0000DE070000022000000400000077
:10EBD0001C0000206A00000001000000E8030000A3
:10EBE0000100000002200000050000001C000020C1
:10EBF000650000000100000040420F00010000001D
:10EC00000220000006000000340000200000000088
:10EC1000000000003B0000000000000000000000B9
:10EC2000640000001C0000206B0000000A000000CF
:10EC30006400000028000000129000006500000041
:10EC4000380000200000000000000000D007000095
:10EC5000BC02000011580000660000001C000020EB
:10EC60007A010000010000000A0000000A00000014
:10EC700002200000670000003C00002000000000AF
:10EC8000000000000A000000000000000120000059
:10EC9000680000001C0000207B0100000000000054
:10ECA0000100000000000000026800006900000090
:10ECB0001C0000207C01000000000000010000009A
:10ECC00000000000026800006A0000001C00002034
:10ECD0007D01000000000000780000000500000039
:10ECE000C24800006B0000001C0000207E010000F4
:10ECF00000000000D0070000D007000013580000FB
:10ED00006C0000001C0000207F01000000000000DB
:10ED10009F05000000000000434800006D00000057
:10ED20001C0000208001000000000000D00700004F
:10ED300000000000135800006E0000001C000020BE
:10ED400081010000000000009F050000000000009D
:10ED5000434800006F0000001C00002082010000FA
:10ED60000000000001000000000000000268000038
:10ED7000700000001C000020830100000100000062
:10ED800006000000010000000220000071000000E9
:10ED90001C00002084010000000000009F0500000E
:10EDA0000000000042480000720000001C0000202B
:10EDB00085010000000000000100000001000000CB
:10EDC00002680000730000001C00002086010000A3
:10EDD00000000000010000000000000002680000C8
:10EDE0007400000048000020000000000000000047
:10EDF0000A00000000000000012000007500000073
:10EE00001C00002091010000010000000200000031
:10EE10000100000002200000C80000007000002077
:10EE20000000000000000000D0070000000000000B
:10EE300011580000C900000074000020000000000C
:10EE400000000000D0070000000000001158000082
:10EE5000CA00000078000020000000000000000050
:10EE6000010000000000000001680000CB0000006D
:10EE70007C000020000000000000000001000000F5
:10EE80000000000001680000CC00000080000020AD
:10EE90000000000000000000010000000000000071
:10EEA00001680000CD000000840000200000000088
:10EEB00000000000010000000000000001680000E8
:10EEC000CE000000880000200000000000000000CC
:10EED0000A0000000000000000200000CF00000039
:10EEE0008C00002000000000000000000100000075
:10EEF0000000000000680000D0000000900000202A
:10EF00000000000000000000D0070000000000002A
:10EF100031290000D1000000940000200000000012
:10EF20000000000001000000000000000068000078
:10EF3000D200000098000020000000000000000047
:10EF4000010000000000000000680000E80300006D
:10EF50001C0000206C000000000000000500000004
:10EF60000000000002000000E90300001C00002077
:10EF70006D000000BC020000B0040000840300002B
:10EF800012580000EA0300001C0000208600000068
:10EF900001000000100E00000A000000C24800003E
:10EFA000EB0300001C0000206E00000000000000C9
:10EFB0007F51010000000000D2500000EC0300006F
:10EFC0001C0000206F000000000000007F510100C5
:10EFD00000000000D2500000ED0300001C000020E3
:10EFE000700000000A000000C0A80000100E000021
:10EFF000D2500000EE0300001C0000207100000051
:10F000000A000000C0A8000008070000D25000005D
:10F01000EF0300001C000020720000000000000050
:10F020007F51010000000000D2500000F0030000FA
:10F030001C00002073000000000000007F51010050
:10F0400000000000D2500000F10300001C0000206E
:10F05000740000000A000000C0A80000100E0000AC
:10F06000D2500000F20300001C00002075000000D8
:10F070000A000000C0A8000008070000D2500000ED
:10F08000F30300001C0000207600000000000000D8
:10F090007F51010000000000D2500000F403000086
:10F0A0001C00002077000000000000007F510100DC
:10F0B00000000000D2500000F50300001C000020FA
:10F0C000780000000A000000C0A80000100E000038
:10F0D000D2500000F60300001C0000207900000060
:10F0E0000A000000C0A8000008070000D25000007D
:10F0F000F70300001C0000207A0000000000000060
:10F100007F51010000000000D2500000F803000011
:10F110001C0000207B000000000000007F51010067
:10F1200000000000D2500000F90300001C00002085
:10F130007C0000000A000000C0A80000100E0000C3
:10F14000D2500000FA0300001C0000207D000000E7
:10F150000A000000C0A8000008070000D25000000C
:10F16000FB0300001C0000207E00000000000000E7
:10F170007F51010000000000D2500000FC0300009D
:10F180001C0000207F000000000000007F510100F3
:10F1900000000000D2500000FD0300001C00002011
:10F1A000800000000A000000C0A80000100E00004F
:10F1B000D2500000FE0300001C000020810000006F
:10F1C0000A000000C0A8000008070000D25000009C
:10F1D000FF0300001C00002082000000000000006F
:10F1E0007F51010000000000D25000000004000028
:10F1F0001C00002083000000000000007F5101007F
:10F2000000000000D2500000010400001C0000209B
:10F21000840000000A000000C0A80000100E0000DA
:10F22000D2500000020400001C00002085000000F5
:10F230000A000000C0A8000008070000D25000002B
:10F24000030400001C000020870100002020202073
:10F25000FFFFFF7F31302D5602500100D007000024
:10F260001C000020870000000000000005000000D6
:10F270000000000002000000D10700001C00002078
:10F2800088000000BC020000B004000084030000FD
:10F2900012580000D20700001C000020A10000004E
:10F2A00001000000100E00000A000000C24800002B
:10F2B000D30700001C0000208900000000000000AF
:10F2C0007F51010000000000D2500000D407000070
:10F2D0001C0000208A000000000000007F51010097
:10F2E00000000000D2500000D50700001C000020E4
:10F2F0008B0000000A000000C0A80000100E0000F3
:10F30000D2500000D60700001C0000208C00000036
:10F310000A000000C0A8000008070000D25000004A
:10F32000D70700001C0000208D0000000000000036
:10F330007F51010000000000D2500000D8070000FB
:10F340001C0000208E000000000000007F51010022
:10F3500000000000D2500000D90700001C0000206F
:10F360008F0000000A000000C0A80000100E00007E
:10F37000D2500000DA0700001C00002090000000BE
:10F380000A000000C0A8000008070000D2500000DA
:10F39000DB0700001C0000209100000000000000BE
:10F3A0007F51010000000000D2500000DC07000087
:10F3B0001C00002092000000000000007F510100AE
:10F3C00000000000D2500000DD0700001C000020FB
:10F3D000930000000A000000C0A80000100E00000A
:10F3E000D2500000DE0700001C0000209400000046
:10F3F0000A000000C0A8000008070000D25000006A
:10F40000DF0700001C000020950000000000000045
:10F410007F51010000000000D2500000E007000012
:10F420001C00002096000000000000007F51010039
:10F4300000000000D2500000E10700001C00002086
:10F44000970000000A000000C0A80000100E000095
:10F45000D2500000E20700001C00002098000000CD
:10F460000A000000C0A8000008070000D2500000F9
:10F47000E30700001C0000209900000000000000CD
:10F480007F51010000000000D2500000E40700009E
:10F490001C0000209A000000000000007F510100C5
:10F4A00000000000D2500000E50700001C00002012
:10F4B0009B0000000A000000C0A80000100E000021
:10F4C000D2500000E60700001C0000209C00000055
:10F4D0000A000000C0A8000008070000D250000089
:10F4E000E70700001C0000209D0000000000000055
:10F4F0007F51010000000000D2500000E80700002A
:10F500001C0000209E000000000000007F51010050
:10F5100000000000D2500000E90700001C0000209D
:10F520009F0000000A000000C0A80000100E0000AC
:10F53000D2500000EA0700001C000020A0000000DC
:10F540000A000000C0A8000008070000D250000018
:10F55000EB0700001C000020880100002020202074
:10F56000FFFFFF7F32302D5602500100B80B000024
:10F570001C000020A20000000000000005000000A8
:10F580000000000002000000B90B00001C00002079
:10F59000A3000000BC020000B004000084030000CF
:10F5A00012580000BA0B00001C000020BC00000034
:10F5B00001000000100E00000A000000C248000018
:10F5C000BB0B00001C000020A40000000000000095
:10F5D0007F51010000000000D2500000BC0B000071
:10F5E0001C000020A5000000000000007F51010069
:10F5F00000000000D2500000BD0B00001C000020E5
:10F60000A60000000A000000C0A80000100E0000C4
:10F61000D2500000BE0B00001C000020A70000001C
:10F620000A000000C0A8000008070000D250000037
:10F63000BF0B00001C000020A8000000000000001C
:10F640007F51010000000000D2500000C00B0000FC
:10F650001C000020A9000000000000007F510100F4
:10F6600000000000D2500000C10B00001C00002070
:10F67000AA0000000A000000C0A80000100E000050
:10F68000D2500000C20B00001C000020AB000000A4
:10F690000A000000C0A8000008070000D2500000C7
:10F6A000C30B00001C000020AC00000000000000A4
:10F6B0007F51010000000000D2500000C40B000088
:10F6C0001C000020AD000000000000007F51010080
:10F6D00000000000D2500000C50B00001C000020FC
:10F6E000AE0000000A000000C0A80000100E0000DC
:10F6F000D2500000C60B00001C000020AF0000002C
:10F700000A000000C0A8000008070000D250000056
:10F71000C70B00001C000020B0000000000000002B
:10F720007F51010000000000D2500000C80B000013
:10F730001C000020B1000000000000007F5101000B
:10F7400000000000D2500000C90B00001C00002087
:10F75000B20000000A000000C0A80000100E000067
:10F76000D2500000CA0B00001C000020B3000000B3
:10F770000A000000C0A8000008070000D2500000E6
:10F78000CB0B00001C000020B400000000000000B3
:10F790007F51010000000000D2500000CC0B00009F
:10F7A0001C000020B5000000000000007F51010097
:10F7B00000000000D2500000CD0B00001C00002013
:10F7C000B60000000A000000C0A80000100E0000F3
:10F7D000D2500000CE0B00001C000020B70000003B
:10F7E0000A000000C0A8000008070000D250000076
:10F7F000CF0B00001C000020B8000000000000003B
:10F800007F51010000000000D2500000D00B00002A
:10F810001C000020B9000000000000007F51010022
:10F8200000000000D2500000D10B00001C0000209E
:10F83000BA0000000A000000C0A80000100E00007E
:10F84000D2500000D20B00001C000020BB000000C2
:10F850000A000000C0A8000008070000D250000005
:10F86000D30B00001C000020890100002020202074
:10F87000FFFFFF7F33302D5602500100A00F000024
:10F880001C000020BD00000000000000050000007A
:10F890000000000002000000A10F00001C0000207A
:10F8A000BE000000BC020000B004000084030000A1
:10F8B00012580000A20F00001C000020D70000001A
:10F8C00001000000100E00000A000000C248000005
:10F8D000A30F00001C000020BF000000000000007B
:10F8E0007F51010000000000D2500000A40F000072
:10F8F0001C000020C0000000000000007F5101003B
:10F9000000000000D2500000A50F00001C000020E5
:10F91000C10000000A000000C0A80000100E000096
:10F92000D2500000A60F00001C000020C200000002
:10F930000A000000C0A8000008070000D250000024
:10F94000A70F00001C000020C30000000000000002
:10F950007F51010000000000D2500000A80F0000FD
:10F960001C000020C4000000000000007F510100C6
:10F9700000000000D2500000A90F00001C00002071
:10F98000C50000000A000000C0A80000100E000022
:10F99000D2500000AA0F00001C000020C60000008A
:10F9A0000A000000C0A8000008070000D2500000B4
:10F9B000AB0F00001C000020C7000000000000008A
:10F9C0007F51010000000000D2500000AC0F000089
:10F9D0001C000020C8000000000000007F51010052
:10F9E00000000000D2500000AD0F00001C000020FD
:10F9F000C90000000A000000C0A80000100E0000AE
:10FA0000D2500000AE0F00001C000020CA00000011
:10FA10000A000000C0A8000008070000D250000043
:10FA2000AF0F00001C000020CB0000000000000011
:10FA30007F51010000000000D2500000B00F000014
:10FA40001C000020CC000000000000007F510100DD
:10FA500000000000D2500000B10F00001C00002088
:10FA6000CD0000000A000000C0A80000100E000039
:10FA7000D2500000B20F00001C000020CE00000099
:10FA80000A000000C0A8000008070000D2500000D3
:10FA9000B30F00001C000020CF0000000000000099
:10FAA0007F51010000000000D2500000B40F0000A0
:10FAB0001C000020D0000000000000007F51010069
:10FAC00000000000D2500000B50F00001C00002014
:10FAD000D10000000A000000C0A80000100E0000C5
:10FAE000D2500000B60F00001C000020D200000021
:10FAF0000A000000C0A8000008070000D250000063
:10FB0000B70F00001C000020D30000000000000020
:10FB10007F51010000000000D2500000B80F00002B
:10FB20001C000020D4000000000000007F510100F4
:10FB300000000000D2500000B90F00001C0000209F
:10FB4000D50000000A000000C0A80000100E000050
:10FB5000D2500000BA0F00001C000020D6000000A8
:10FB60000A000000C0A8000008070000D2500000F2
:10FB7000BB0F00001C0000208A0100002020202074
:10FB8000FFFFFF7F34302D56025001008813000024
:10FB90001C000020D800000000000000050000004C
:10FBA0000000000002000000891300001C0000207B
:10FBB000D9000000BC020000B00400008403000073
:10FBC000125800008A1300001C000020F200000000
:10FBD00001000000100E00000A000000C2480000F2
:10FBE0008B1300001C000020DA0000000000000061
:10FBF0007F51010000000000D25000008C13000073
:10FC00001C000020DB000000000000007F5101000C
:10FC100000000000D25000008D1300001C000020E6
:10FC2000DC0000000A000000C0A80000100E000068
:10FC3000D25000008E1300001C000020DD000000E8
:10FC40000A000000C0A8000008070000D250000011
:10FC50008F1300001C000020DE00000000000000E8
:10FC60007F51010000000000D250000090130000FE
:10FC70001C000020DF000000000000007F51010098
:10FC800000000000D2500000911300001C00002072
:10FC9000E00000000A000000C0A80000100E0000F4
:10FCA000D2500000921300001C000020E100000070
:10FCB0000A000000C0A8000008070000D2500000A1
:10FCC000931300001C000020E20000000000000070
:10FCD0007F51010000000000D2500000941300008A
:10FCE0001C000020E3000000000000007F51010024
:10FCF00000000000D2500000951300001C000020FE
:10FD0000E40000000A000000C0A80000100E00007F
:10FD1000D2500000961300001C000020E5000000F7
:10FD20000A000000C0A8000008070000D250000030
:10FD3000971300001C000020E600000000000000F7
:10FD40007F51010000000000D25000009813000015
:10FD50001C000020E7000000000000007F510100AF
:10FD600000000000D2500000991300001C00002089
:10FD7000E80000000A000000C0A80000100E00000B
:10FD8000D25000009A1300001C000020E90000007F
:10FD90000A000000C0A8000008070000D2500000C0
:10FDA0009B1300001C000020EA000000000000007F
:10FDB0007F51010000000000D25000009C130000A1
:10FDC0001C000020EB000000000000007F5101003B
:10FDD00000000000D25000009D1300001C00002015
:10FDE000EC0000000A000000C0A80000100E000097
:10FDF000D25000009E1300001C000020ED00000007
:10FE00000A000000C0A8000008070000D25000004F
:10FE10009F1300001C000020EE0000000000000006
:10FE20007F51010000000000D2500000A01300002C
:10FE30001C000020EF000000000000007F510100C6
:10FE400000000000D2500000A11300001C000020A0
:10FE5000F00000000A000000C0A80000100E000022
:10FE6000D2500000A21300001C000020F10000008E
:10FE70000A000000C0A8000008070000D2500000DF
:10FE8000A31300001C0000208B0100002020202074
:10FE9000FFFFFF7F35302D56025001007017000024
:10FEA0001C000020F300000000000000050000001E
:10FEB0000000000002000000711700001C0000207C
:10FEC000F4000000BC020000B00400008403000045
:10FED00012580000721700001C0000200D010000E5
:10FEE00001000000100E00000A000000C2480000DF
:10FEF000731700001C000020F50000000000000047
:10FF00007F51010000000000D25000007417000073
:10FF10001C000020F6000000000000007F510100DE
:10FF200000000000D2500000751700001C000020E7
:10FF3000F70000000A000000C0A80000100E00003A
:10FF4000D2500000761700001C000020F8000000CE
:10FF50000A000000C0A8000008070000D2500000FE
:10FF6000771700001C000020F900000000000000CE
:10FF70007F51010000000000D250000078170000FF
:10FF80001C000020FA000000000000007F5101006A
:10FF900000000000D2500000791700001C00002073
:10FFA000FB0000000A000000C0A80000100E0000C6
:10FFB000D25000007A1700001C000020FC00000056
:10FFC0000A000000C0A8000008070000D25000008E
:10FFD0007B1700001C000020FD0000000000000056
:10FFE0007F51010000000000D25000007C1700008B
:10FFF0001C000020FE000000000000007F510100F6
:020000040802F0
:1000000000000000D25000007D1700001C000020FE
:10001000FF0000000A000000C0A80000100E000051
:10002000D25000007E1700001C00002000010000DC
:100030000A000000C0A8000008070000D25000001D
:100040007F1700001C0000200101000000000000DC
:100050007F51010000000000D25000008017000016
:100060001C00002002010000000000007F51010080
:1000700000000000D2500000811700001C0000208A
:10008000030100000A000000C0A80000100E0000DC
:10009000D2500000821700001C0000200401000064
:1000A0000A000000C0A8000008070000D2500000AD
:1000B000831700001C000020050100000000000064
:1000C0007F51010000000000D250000084170000A2
:1000D0001C00002006010000000000007F5101000C
:1000E00000000000D2500000851700001C00002016
:1000F000070100000A000000C0A80000100E000068
:10010000D2500000861700001C00002008010000EB
:100110000A000000C0A8000008070000D25000003C
:10012000871700001C0000200901000000000000EB
:100130007F51010000000000D2500000881700002D
:100140001C0000200A010000000000007F51010097
:1001500000000000D2500000891700001C000020A1
:100160000B0100000A000000C0A80000100E0000F3
:10017000D25000008A1700001C0000200C01000073
:100180000A000000C0A8000008070000D2500000CC
:100190008B1700001C0000208C0100002020202074
:1001A000FFFFFF7F36302D5602500100581B000024
:1001B0001C0000200E0100000000000005000000EF
:1001C0000000000002000000591B00001C0000207D
:1001D0000F010000BC020000B00400008403000016
:1001E000125800005A1B00001C00002028010000CB
:1001F00001000000100E00000A000000C2480000CC
:100200005B1B00001C00002010010000000000002B
:100210007F51010000000000D25000005C1B000074
:100220001C00002011010000000000007F510100AF
:1002300000000000D25000005D1B00001C000020E8
:10024000120100000A000000C0A80000100E00000B
:10025000D25000005E1B00001C00002013010000B3
:100260000A000000C0A8000008070000D2500000EB
:100270005F1B00001C0000201401000000000000B3
:100280007F51010000000000D2500000601B000000
:100290001C00002015010000000000007F5101003B
:1002A00000000000D2500000611B00001C00002074
:1002B000160100000A000000C0A80000100E000097
:1002C000D2500000621B00001C000020170100003B
:1002D0000A000000C0A8000008070000D25000007B
:1002E000631B00001C00002018010000000000003B
:1002F0007F51010000000000D2500000641B00008C
:100300001C00002019010000000000007F510100C6
:1003100000000000D2500000651B00001C000020FF
:100320001A0100000A000000C0A80000100E000022
:10033000D2500000661B00001C0000201B010000C2
:100340000A000000C0A8000008070000D25000000A
:10035000671B00001C0000201C01000000000000C2
:100360007F51010000000000D2500000681B000017
:100370001C0000201D010000000000007F51010052
:1003800000000000D2500000691B00001C0000208B
:100390001E0100000A000000C0A80000100E0000AE
:1003A000D25000006A1B00001C0000201F0100004A
:1003B0000A000000C0A8000008070000D25000009A
:1003C0006B1B00001C00002020010000000000004A
:1003D0007F51010000000000D25000006C1B0000A3
:1003E0001C00002021010000000000007F510100DE
:1003F00000000000D25000006D1B00001C00002017
:10040000220100000A000000C0A80000100E000039
:10041000D25000006E1B00001C00002023010000D1
:100420000A000000C0A8000008070000D250000029
:100430006F1B00001C0000202401000000000000D1
:100440007F51010000000000D2500000701B00002E
:100450001C00002025010000000000007F51010069
:1004600000000000D2500000711B00001C000020A2
:10047000260100000A000000C0A80000100E0000C5
:10048000D2500000721B00001C0000202701000059
:100490000A000000C0A8000008070000D2500000B9
:1004A000731B00001C0000208D0100002020202074
:1004B000FFFFFF7F37302D5602500100401F000024
:1004C0001C000020290100000000000005000000C1
:1004D0000000000002000000411F00001C0000207E
:1004E0002A010000BC020000B004000084030000E8
:1004F00012580000421F00001C00002043010000B1
:1005000001000000100E00000A000000C2480000B8
:10051000431F00001C0000202B0100000000000011
:100520007F51010000000000D2500000441F000075
:100530001C0000202C010000000000007F51010081
:1005400000000000D2500000451F00001C000020E9
:100550002D0100000A000000C0A80000100E0000DD
:10056000D2500000461F00001C0000202E01000099
:100570000A000000C0A8000008070000D2500000D8
:10058000471F00001C0000202F0100000000000099
:100590007F51010000000000D2500000481F000001
:1005A0001C00002030010000000000007F5101000D
:1005B00000000000D2500000491F00001C00002075
:1005C000310100000A000000C0A80000100E000069
:1005D000D25000004A1F00001C0000203201000021
:1005E0000A000000C0A8000008070000D250000068
:1005F0004B1F00001C000020330100000000000021
:100600007F51010000000000D25000004C1F00008C
:100610001C00002034010000000000007F51010098
:1006200000000000D25000004D1F00001C00002000
:10063000350100000A000000C0A80000100E0000F4
:10064000D25000004E1F00001C00002036010000A8
:100650000A000000C0A8000008070000D2500000F7
:100660004F1F00001C0000203701000000000000A8
:100670007F51010000000000D2500000501F000018
:100680001C00002038010000000000007F51010024
:1006900000000000D2500000511F00001C0000208C
:1006A000390100000A000000C0A80000100E000080
:1006B000D2500000521F00001C0000203A01000030
:1006C0000A000000C0A8000008070000D250000087
:1006D000531F00001C0000203B0100000000000030
:1006E0007F51010000000000D2500000541F0000A4
:1006F0001C0000203C010000000000007F510100B0
:1007000000000000D2500000551F00001C00002017
:100710003D0100000A000000C0A80000100E00000B
:10072000D2500000561F00001C0000203E010000B7
:100730000A000000C0A8000008070000D250000016
:10074000571F00001C0000203F01000000000000B7
:100750007F51010000000000D2500000581F00002F
:100760001C00002040010000000000007F5101003B
:1007700000000000D2500000591F00001C000020A3
:10078000410100000A000000C0A80000100E000097
:10079000D25000005A1F00001C000020420100003F
:1007A0000A000000C0A8000008070000D2500000A6
:1007B0005B1F00001C0000208E0100002020202074
:1007C000FFFFFF7F38302D56025001002823000024
:1007D0001C00002044010000000000000500000093
:1007E0000000000002000000292300001C0000207F
:1007F00045010000BC020000B004000084030000BA
:10080000125800002A2300001C0000205E01000096
:1008100001000000100E00000A000000C2480000A5
:100820002B2300001C0000204601000000000000F7
:100830007F51010000000000D25000002C23000076
:100840001C00002047010000000000007F51010053
:1008500000000000D25000002D2300001C000020EA
:10086000480100000A000000C0A80000100E0000AF
:10087000D25000002E2300001C000020490100007F
:100880000A000000C0A8000008070000D2500000C5
:100890002F2300001C0000204A010000000000007F
:1008A0007F51010000000000D25000003023000002
:1008B0001C0000204B010000000000007F510100DF
:1008C00000000000D2500000312300001C00002076
:1008D0004C0100000A000000C0A80000100E00003B
:1008E000D2500000322300001C0000204D01000007
:1008F0000A000000C0A8000008070000D250000055
:10090000332300001C0000204E0100000000000006
:100910007F51010000000000D2500000342300008D
:100920001C0000204F010000000000007F5101006A
:1009300000000000D2500000352300001C00002001
:10094000500100000A000000C0A80000100E0000C6
:10095000D2500000362300001C000020510100008E
:100960000A000000C0A8000008070000D2500000E4
:10097000372300001C00002052010000000000008E
:100980007F51010000000000D25000003823000019
:100990001C00002053010000000000007F510100F6
:1009A00000000000D2500000392300001C0000208D
:1009B000540100000A000000C0A80000100E000052
:1009C000D25000003A2300001C0000205501000016
:1009D0000A000000C0A8000008070000D250000074
:1009E0003B2300001C000020560100000000000016
:1009F0007F51010000000000D25000003C230000A5
:100A00001C00002057010000000000007F51010081
:100A100000000000D25000003D2300001C00002018
:100A2000580100000A000000C0A80000100E0000DD
:100A3000D25000003E2300001C000020590100009D
:100A40000A000000C0A8000008070000D250000003
:100A50003F2300001C0000205A010000000000009D
:100A60007F51010000000000D25000004023000030
:100A70001C0000205B010000000000007F5101000D
:100A800000000000D2500000412300001C000020A4
:100A90005C0100000A000000C0A80000100E000069
:100AA000D2500000422300001C0000205D01000025
:100AB0000A000000C0A8000008070000D250000093
:100AC000432300001C0000208F0100002020202074
:100AD000FFFFFF7F39302D56025001001027000024
:100AE0001C0000205F010000000000000500000065
:100AF0000000000002000000112700001C00002080
:100B000060010000BC020000B0040000840300008B
:100B100012580000122700001C000020790100007C
:100B200001000000100E00000A000000C248000092
:100B3000132700001C0000206101000000000000DD
:100B40007F51010000000000D25000001427000077
:100B50001C00002062010000000000007F51010025
:100B600000000000D2500000152700001C000020EB
:100B7000630100000A000000C0A80000100E000081
:100B8000D2500000162700001C0000206401000065
:100B90000A000000C0A8000008070000D2500000B2
:100BA000172700001C000020650100000000000065
:100BB0007F51010000000000D25000001827000003
:100BC0001C00002066010000000000007F510100B1
:100BD00000000000D2500000192700001C00002077
:100BE000670100000A000000C0A80000100E00000D
:100BF000D25000001A2700001C00002068010000ED
:100C00000A000000C0A8000008070000D250000041
:100C10001B2700001C0000206901000000000000EC
:100C20007F51010000000000D25000001C2700008E
:100C30001C0000206A010000000000007F5101003C
:100C400000000000D25000001D2700001C00002002
:100C50006B0100000A000000C0A80000100E000098
:100C6000D25000001E2700001C0000206C01000074
:100C70000A000000C0A8000008070000D2500000D1
:100C80001F2700001C0000206D0100000000000074
:100C90007F51010000000000D2500000202700001A
:100CA0001C0000206E010000000000007F510100C8
:100CB00000000000D2500000212700001C0000208E
:100CC0006F0100000A000000C0A80000100E000024
:100CD000D2500000222700001C00002070010000FC
:100CE0000A000000C0A8000008070000D250000061
:100CF000232700001C0000207101000000000000FC
:100D00007F51010000000000D250000024270000A5
:100D10001C00002072010000000000007F51010053
:100D200000000000D2500000252700001C00002019
:100D3000730100000A000000C0A80000100E0000AF
:100D4000D2500000262700001C0000207401000083
:100D50000A000000C0A8000008070000D2500000F0
:100D6000272700001C000020750100000000000083
:100D70007F51010000000000D25000002827000031
:100D80001C00002076010000000000007F510100DF
:100D900000000000D2500000292700001C000020A5
:100DA000770100000A000000C0A80000100E00003B
:100DB000D25000002A2700001C000020780100000B
:100DC0000A000000C0A8000008070000D250000080
:100DD0002B2700001C000020900100002020202074
:100DE000FFFFFF7F30312D5602500100FFFF000052
:100DF00000000000000000000000000000000000F3
:100E000000000000000000000000000054220E005E
:100E1000010000000A0000002A070D000200000087
:100E200014000000E7030C00030000001E00000097
:100E300064160B000400000028000000AF3C0A000C
:100E400005000000320000000475090007000000E2
:100E50003C000000CBBD0800080000004600000078
:100E6000911508000A00000050000000077B0700F1
:100E70000B0000005A000000FCEC06000D00000012
:100E8000640000005A6A06000F0000006E000000B7
:100E900028F2050011000000780000007F830500A3
:100EA0001300000082000000921D050016000000E3
:100EB0008C000000A2BF0400180000009600000093
:100EC000046904001B000000A00000001B190400BE
:100ED0001D000000AA00000058CF03002100000000
:100EE000B40000003A8B030024000000BE000000A4
:100EF000494C030027000000C80000001A1203003C
:100F00002B000000D20000004ADC02002F0000008D
:100F1000DC0000007DAA020033000000E6000000B3
:100F2000637C020037000000F0000000AE510200B8
:100F30003C000000FA0000001A2A020041000000F4
:100F40000401000069050200460000000E010000D7
:100F50005FE301004C00000018010000C8C301005D
:100F6000520000002201000073A60100580000009A
:100F70002C010000348B01005F00000036010000EE
:100F8000E17101006600000040010000565A0100B6
:100F90006E0000004A0100006F440100760000006E
:100FA000540100000D3001007E0000005E010000D1
:100FB000131D01008700000068010000660B01009E
:100FC0009000000072010000EDFA00009A0000009D
:100FD0007C01000091EB0000A400000086010000ED
:100FE0003EDD0000AF00000090010000E0CF0000F7
:100FF000BA0000009A01000066C30000C6000000AD
:10100000A4010000BFB70000D3000000AE01000043
:10101000DCAC0000E0000000B8010000AFA200005E
:10102000EE000000C20100002B990000FC0000004F
:10103000CC010000449000000C010000D60100002B
:10104000EF8700001B010000E0010000228000008B
:101050002C010000EA010000D47800003D010000EE
:10106000F4010000FC7100004F010000FE010000CF
:10107000916B000062010000080200008D65000015
:101080007601000012020000E85F00008B01000002
:101090001C0200009C5A0000A00100002602000073
:1010A000A3550000B601000030020000F850000017
:1010B000CD0100003A020000944C0000E501000060
:1010C0004402000075480000FE0100004E020000CE
:1010D000944400001702000058020000EE40000097
:1010E0003202000062020000803D00004D0200005C
:1010F0006C020000453A0000690200007602000020
:101100003A37000087020000800200005D340000D2
:10111000A50200008A020000AA310000C4020000FB
:10112000940200001E2F0000E40200009E02000056
:10113000B82C000005030000A8020000752A00007A
:1011400026030000B20200005228000049030000FC
:10115000BC0200004E2600006C030000C602000026
:101160006724000090030000D00200009B220000D2
:10117000B5030000DA020000E8200000DB030000F5
:10118000E40200004D1F000002040000EE02000017
:10119000C91D000029040000F8020000591C0000CD
:1011A0005104000002030000FD1A00007A04000050
:1011B0000C030000B4190000A40400001603000092
:1011C0007D180000CD040000200300005617000029
:1011D000F80400002A0300003F1600002305000069
:1011E00034030000361500004F0500003E030000E8
:1011F0003B1400007B050000480300004D13000075
:10120000A8050000520300006B120000D505000085
:101210005C03000095110000020600006603000058
:10122000CA1000002F060000700300000910000023
:101230005D0600007A030000520F00008B060000DC
:1012400084030000A40E0000B90600008E03000015
:10125000FF0D0000E806000098030000620D00008A
:1012600016070000A2030000CD0C00004407000098
:10127000AC0300003F0C000072070000B603000042
:10128000B80B0000A0070000C0030000380B0000EE
:10129000CE070000CA030000BD0A0000FC070000E2
:1012A000D4030000490A00002A080000DE03000001
:1012B000DA09000057080000E80300007109000087
:1012C00084080000F20300000C090000B1080000CF
:1012D000FC030000AC080000DD080000060400006C
:1012E000510800000909000010040000FA0700007E
:1012F000350900001A040000A7070000600900007B
:1013000024040000580700008A0900002E04000091
:101310000C070000B409000038040000C4060000F7
:10132000DE090000420400007F060000070A0000FA
:101330004C0400003D0600002F0A00005604000087
:10134000FF050000560A000060040000C30500000D
:101350007D0A00006A04000089050000A40A00005C
:101360007404000053050000CA0A00007E04000057
:101370001E050000EF0A000088040000EC040000D5
:10138000130B000092040000BC040000370B0000A7
:101390009C0400008E0400005A0B0000A60400000C
:1013A000630400007C0B0000B0040000390400005E
:1013B0009E0B0000BA04000010040000BE0B0000E9
:1013C000C4040000EA030000DF0B0000CE040000AC
:1013D000C5030000FE0B0000D8040000A2030000BB
:1013E0001D0C0000E2040000800300003B0C000024
:1013F000EC0400005F030000580C0000F60400003D
:1014000040030000750C00000005000023030000ED
:10141000910C00000A05000006030000AC0C00005F
:1014200014050000EB020000C70C00001E050000C0
:10143000D0020000E00C000028050000B702000008
:10144000FA0C0000320500009F020000120D00009F
:101450003C050000880200002A0D0000460500003F
:1014600071020000420D0000500500005C02000007
:10147000580D00005A050000470200006E0D0000E4
:101480006405000033020000840D00006E050000BA
:1014900020020000990D0000780500000E020000F7
:1014A000AD0D000082050000FC010000C10D000030
:1014B0008C050000EC010000D40D00009605000032
:1014C000DB010000E70D0000A0050000CC010000DA
:1014D000F90D0000AA050000BD0100000B0E000080
:1014E000B4050000AE0100001C0E0000BE050000A7
:1014F000A00100002D0E0000C805000093010000AF
:101500003D0E0000D2050000860100004D0E0000D7
:10151000DC050000790100005C0E0000E60500001B
:101520006E0100006B0E0000F0050000620100007B
:10153000790E0000FA05000057010000870E000038
:10154000040600004C010000950E00000E0600008D
:1015500042010000A20E0000180600003801000041
:10156000AF0E0000220600002E010000BB0E00009E
:101570002C06000025010000C70E00003606000002
:101580001C010000D30E0000400600001301000003
:10159000DE0E00004A0600000B010000E90E00000C
:1015A0005406000003010000F40E00005E06000077
:1015B000FB000000FE0E000068060000F4000000C2
:1015C000080F000072060000ED000000120F00007E
:1015D0007C060000E60000001C0F000086060000EC
:1015E000DF000000250F000090060000D900000079
:1015F0002E0F00009A060000D2000000360F0000F7
:10160000A4060000CC0000003F0F0000AE06000062
:10161000C6000000470F0000B8060000C10000002F
:101620004F0F0000C2060000BB000000570F000073
:10163000CC060000B60000005E0F0000D6060000D9
:10164000B1000000650F0000E0060000AC000000E3
:101650006D0F0000EA060000A7000000730F0000F5
:10166000F4060000A20000007A0F0000FE06000051
:101670009E000000800F0000080700009A00000094
:10168000860F000012070000950000008D0F00007B
:101690001C07000091000000930F000026070000C7
:1016A0008D000000980F0000300700008A00000045
:1016B0009E0F00003A07000086000000A30F000004
:1016C0004407000082000000A80F00004E07000041
:1016D0007F000000AE0F0000580700007C000000F3
:1016E000B20F00006207000078000000B70F000092
:1016F0006C07000075000000BC0F000076070000BA
:1017000072000000C10F0000800700006F000000A1
:10171000C50F00008A0700006C000000C90F000020
:101720009407000069000000CD0F00009E07000034
:1017300067000000D10F0000A8070000640000004F
:10174000D50F0000B207000062000000D90F0000B2
:10175000BC0700005F000000DD0F0000C6070000AE
:101760005D000000E00F0000D00700005A000000FC
:10177000E40F0000DA07000058000000E70F000047
:10178000E407000056000000EB0F0000EE07000029
:1017900054000000EE0F0000F807000052000000A7
:1017A000F10F00000208000050000000F40F0000DC
:1017B0000C0800004E000000F70F000016080000A3
:1017C0004C000000FA0F0000200800004A00000052
:1017D000FD0F00002A08000048000000FF0F000075
:1017E0003408000047000000021000000000000064
:1017F00021100000422000006330000084400000FF
:10180000A5500000C6600000E770000008810000DD
:10181000299100004AA100006BB100008CC10000BA
:10182000ADD10000CEE10000EFF100003112000068
:10183000100200007332000052220000B552000076
:1018400094420000F7720000D66200003993000055
:10185000188300007BB300005AA30000BDD3000032
:101860009CC30000FFF30000DEE3000062240000E0
:10187000433400002004000001140000E66400006E
:10188000C7740000A4440000855400006AA500004D
:101890004BB500002885000009950000EEE500002A
:1018A000CFF50000ACC500008DD500005336000018
:1018B000722600001116000030060000D7760000E6
:1018C000F666000095560000B44600005BB70000C5
:1018D0007AA700001997000038870000DFF70000A2
:1018E000FEE700009DD70000BCC70000C448000010
:1018F000E558000086680000A77800004008000056
:10190000611800000228000023380000CCC9000044
:10191000EDD900008EE90000AFF900004889000011
:10192000699900000AA900002BB90000F55A0000CF
:10193000D44A0000B77A0000966A0000711A0000CD
:10194000500A0000333A0000122A0000FDDB0000BC
:10195000DCCB0000BFFB00009EEB0000799B000089
:10196000588B00003BBB00001AAB0000A66C0000C7
:10197000877C0000E44C0000C55C0000222C0000C5
:10198000033C0000600C0000411C0000AEED0000B4
:101990008FFD0000ECCD0000CDDD00002AAD000081
:1019A0000BBD0000688D0000499D0000977E00007F
:1019B000B66E0000D55E0000F44E0000133E00003D
:1019C000322E0000511E0000700E00009FFF00002C
:1019D000BEEF0000DDDF0000FCCF00001BBF0000F9
:1019E0003AAF0000599F0000788F000088910000F6
:1019F000A9810000CAB10000EBA100000CD10000D9
:101A00002DC100004EF100006FE1000080100000C9
:101A1000A1000000C2300000E320000004500000DC
:101A2000254000004670000067600000B983000098
:101A300098930000FBA30000DAB300003DC3000050
:101A40001CD300007FE300005EF30000B102000041
:101A500090120000F3220000D23200003542000054
:101A6000145200007762000056720000EAB50000D0
:101A7000CBA50000A8950000898500006EF5000048
:101A80004FE500002CD500000DC50000E234000039
:101A9000C3240000A014000081040000667400004C
:101AA000476400002454000005440000DBA7000048
:101AB000FAB7000099870000B89700005FE70000C0
:101AC0007EF700001DC700003CD70000D3260000B1
:101AD000F236000091060000B016000057660000C4
:101AE0007676000015460000345600004CD9000000
:101AF0006DC900000EF900002FE90000C899000030
:101B0000E98900008AB90000ABA900004458000030
:101B1000654800000678000027680000C018000033
:101B2000E108000082380000A32800007DCB0000FF
:101B30005CDB00003FEB00001EFB0000F98B0000A7
:101B4000D89B0000BBAB00009ABB0000754A0000A8
:101B5000545A0000376A0000167A0000F10A0000AB
:101B6000D01A0000B32A0000923A00002EFD0000B7
:101B70000FED00006CDD00004DCD0000AABD00009F
:101B80008BAD0000E89D0000C98D0000267C0000A0
:101B9000076C0000645C0000454C0000A23C0000A3
:101BA000832C0000E01C0000C10C00001FEF0000AF
:101BB0003EFF00005DCF00007CDF00009BAF000017
:101BC000BABF0000D98F0000F89F0000176E000018
:101BD000367E0000554E0000745E0000932E00001B
:101BE000B23E0000D10E0000F01E00000000000018
:101BF0000000000000005F00000000000007000778
